:100000000C9462080C9481080C9481080C94980A52
:100010000C94CE0A0C9481080C9481080C948108ED
:100020000C9481080C9481080C9481080C9481082C
:100030000C9481080C9481080C9481080C94280E6F
:100040000C9481080C9481080C9481080C9481080C
:100050000C9413580C941F4F0C9481080C94810835
:100060000C9481080C94F54F0C9481080C94E94F82
:100070000C9481080C9481080C9481080C948108DC
:100080000C94D6630C9481080C9481080C9481081C
:100090000C9433500C9481080C9427500C948108D4
:1000A0000C9481080C9481080C9481080C948108AC
:1000B0000C9481080C9481080C9481080C9481089C
:1000C0000C9481080C9481080C9481080C9481088C
:1000D0000C9481080C9481080C9481080C9481087C
:1000E0000C9481080C94CC570C94D6570C94C2579E
:1000F0000C947C570C9407580C94F8570C94EC57BC
:100100000C94E0570C9481080C9481080C9481089D
:100110000C9481080C9481080C9481080C9481083B
:10012000084AD73B3BCE016E84BCBFFDC12F3D6C5E
:1001300074319ABD56833DDA3D00C77F11BED9E4C4
:10014000BB4C3E916BAAAABE000000803F076342F1
:1001500036B79BD8A71A39685618AEBAAB558C1D5E
:100160003CB7CC5763BD6DEDFD753EF6177231BFE0
:10017000000000803F08000000BE922449123EAB00
:10018000AAAA2ABECDCCCC4C3E00000080BEABAAB1
:10019000AAAA3E00000000BF000000803F0000004F
:1001A0000000084178D3BB4387D1133D190E3CC3EF
:1001B000BD4282AD2B3E68EC8276BED98FE1A93E6E
:1001C0004C80EFFFBE01C4FF7F3F000000000050E5
:1001D0003A20256C642050612020252D372E326670
:1001E000206D0A002563002563004932433A200050
:1001F000256300256C642050612020252D372E3288
:1002000066206D00256C6420432000256300545F48
:1002100052483D252D342E3166200052483D252D73
:10022000342E31662000256300256300507772313B
:100230003D25730A0044656275673D3078252D7849
:100240000A00496E7075742050313D25730A0048CC
:10025000554D5F5057525F414C574159533D25739F
:100260000A0025730A006175746F0A004C6F6720DD
:100270006D6F64653D00496E74722E205365633A5C
:1002800020202050303D252D372E33662050313D23
:10029000252D372E33660A00496E74722E20546F56
:1002A00074616C3A2050303D252D6C642050313DF6
:1002B000252D6C640A005553425F5057523D2573FB
:1002C0000A00565F4D43553D252D352E32660A00F6
:1002D000565F494E3D252D352E32660A0052657017
:1002E0006F7274204D61736B3D3078252D6C7820D2
:1002F000005265706F727420496E74657276616C1D
:100300003D252D640A0052494D4520616464723DCB
:10031000252D642E252D640A004E65696768626F7D
:1003200072207461626C652073697A653D25640A88
:1003300000545820506F7765723D25640A00493299
:10034000433A200049443D0053797374656D20534E
:10035000756D6D6172790A00256300256300437530
:100360007272656E74207265706F727420696E743B
:10037000657276616C3D252D64207365630A004EBD
:100380006577207265706F727420696E746572761D
:10039000616C3D252D64207365630A00256300555B
:1003A00073696E67207265706F72743D3078252DA9
:1003B0006C7820004E6577207265706F72743D30E6
:1003C00078252D6C782000256300256300256300C7
:1003D000256300204F534343414C3D2564200020BA
:1003E000467573653A2065653D253032782068662C
:1003F0003D25303278206C663D25303278206C62A5
:100400003D25303278004D43553D2530366C78001F
:10041000256300252D31306C7520252D31306C750C
:1004200020252D31306C7520252D31306C75200A3A
:10043000007478206C656E20202020207268206D6A
:10044000697373202020207268207374616C6520AA
:1004500020207268206D6973630A002563004F4B8A
:100460000A00256300256300256300256300445FBF
:10047000434F4D504153533D307825780A00445F37
:10048000414343454C3D307825780A00445F505243
:1004900045533D307825780A00445F5057525F310C
:1004A0003D307825780A00445F4145533D3078253A
:1004B000780A00445F50315F4C45443D30782578E0
:1004C0000A00445F50305F4C45443D307825780A3F
:1004D00000445F4556454E543D307825780A004427
:1004E0005F504F5745523D307825780A00445F4CA5
:1004F00045443D307825780A00445F4F573D3078B9
:1005000025780A00445F504B543D6E307825780AB8
:1005100000445F54583D307825780A00445F5258B3
:100520003D307825780A00445F4F5045523D307881
:1005300025780A0043757272656E74206465627571
:10054000673D307825580A004E65772064656275EE
:10055000673D307825580A0025730A0025372E3369
:10056000662025372E33660025352E32662000455D
:1005700072726F72203020566F6C74004E6F742050
:10058000737570706F727465640A004572726F7271
:10059000203020566F6C74004572726F72203020CC
:1005A000566F6C740025730A00545820506F77659D
:1005B000723D25640A005465737420352025730A42
:1005C000005465737420342025730A0054657374D5
:1005D00020332025730A005465737420322025735C
:1005E0000A005465737420312025730A0025730AAC
:1005F0000025730A0025730A0025730A0058544128
:100600004C5F5452494D3D25640025730A00525FEA
:1006100050413D09093078256C7800525F503D0902
:10062000093078256C7800525F41333D09093078F4
:10063000257800525F41323D090930782578005213
:100640005F41313D09093078257800525F565F4996
:100650004E3D09093078257800525F52483D09091E
:100660003078257800525F555054494D453D09304A
:1006700078257800525F50315F543D090930782564
:100680007800525F50313D09093078257800525F7B
:1006900050305F543D09093078257800525F503062
:1006A0003D09093078257800525F565F4D43553D2E
:1006B000093078257800525F545F4D43553D09302D
:1006C00078257800525F54313D090930782578004B
:1006D000525F543D09093078257800525F45363421
:1006E0003D09093078257800525F49443D090930B9
:1006F00078257800525F50412000525F5020005210
:100700005F41332000525F41322000525F4131206F
:1007100000525F565F494E2000525F5248200052FF
:100720005F555054494D452000525F50315F542071
:1007300000525F50312000525F50305F5420005211
:100740005F50302000525F565F4D43552000525F8E
:10075000545F4D43552000525F54312000525F5486
:100760002000525F4536342000525F494420002566
:100770003032780025372E33662025372E33662019
:1007800025352E30660025352E32662000204E6538
:100790007665722D7573656420737461636B203E9A
:1007A0002025642062797465730A00557074696D40
:1007B0006520256420646179732C20253032643AE9
:1007C000253032643A253032640A0074657374202F
:1007D0005B6F66667C317C327C337C347C355D209B
:1007E000202020202020202D2074657374206D6F20
:1007F0006465730A0D00776474205B6F6E7C6F66AE
:10080000667C746573745D202020202020202020C9
:1008100020202D207761746368646F670A0D00756E
:1008200070677220202020202020202020202020DF
:1008300020202020202020202020202D20726562D2
:100840006F6F742076696120626F6F746C6F616482
:1008500065720A0D00626F6F742020202020202016
:100860002020202020202020202020202020202088
:10087000202D207265626F6F740A0D00707772739D
:10088000205B646565707C666F7263655F69646C2C
:10089000655D2020202020202D206D637520736C45
:1008A000656570206D6F64650A0D00726573742054
:1008B000656570726F6D2020202020202020202070
:1008C000202020202020202D20726573746F7265F7
:1008D00020656570726F6D0A0D007031205B6F6E60
:1008E0007C6F66665D202020202020202020202094
:1008F0002020202020202D2064697361626C6520F7
:1009000070756C736520703120746F20736176652B
:1009100020706F7765720A0D0070777231205B6FFF
:100920006E7C6F66665D2020202020202020202005
:1009300020202020202D2070696E31207077720ACF
:100940000D0074787077205B31352D305D202020CC
:1009500020202020202020202020202020202D208A
:100960005458205077722E20486967686573742048
:100970003020283364426D290A0D00737320202033
:100980002020202020202020202020202020202067
:10099000202020202020202D2073797374656D2065
:1009A00073756D6D6172790A0D00727320202020BD
:1009B0002020202020202020202020202020202037
:1009C0002020202020202D20726164696F20737404
:1009D0006174730A0D007269205B696E745D20207A
:1009E0002020202020202020202020202020202007
:1009F00020202D207265706F727420696E7465728C
:100A000076616C0A0D007265205B6D61736B5D2011
:100A100020202020202020202020202020202020D6
:100A200020202D206D6F7465207265706F727420A8
:100A300073657474696E670A0D006F77202020203B
:100A400020202020202020202020202020202020A6
:100A50002020202020202D206F6E652D7769726563
:100A60002073656E736F72730A0D006C6F67205B85
:100A70006175746F7C6F6E7C6F66665D20202020D0
:100A8000202020202020202D206D6F74657320648D
:100A9000617461206F6E205553420A0D006E65200F
:100AA0005B666C7573685D2020202020202020204C
:100AB0002020202020202020202D206E65696768BE
:100AC000626F72207461626C650A0D00657272203B
:100AD0002020202020202020202020202020202016
:100AE00020202020202020202D206572726F72206F
:100AF000696E666F0A0D006D63752020202020202E
:100B000020202020202020202020202020202020E5
:100B10002020202D206D637520696E666F0A0D0000
:100B20006964205B72657365745D2020202020203D
:100B30002020202020202020202020202D2069641B
:100B40002068616E646C696E670A0D0068756D706F
:100B5000205B6F6E7C6F66665D2020202020202049
:100B600020202020202020202D2068756D696469B8
:100B70007479207065726D2073656E736F7220706A
:100B800077720A0D0068756D20202020202020201B
:100B90002020202020202020202020202020202055
:100BA000202D2068756D69646974792073656E7392
:100BB0006F720A0D006465205B6D61736B5D2020B0
:100BC0002020202020202020202020202020202025
:100BD000202D2064656275670A0D0063616C6920D1
:100BE0005B5B765F696E7C61317C61325D20766F24
:100BF0006C747C72657365747C6E6F6E655D202DA0
:100C00002063616C6962726174650A0D00616463DE
:100C100020202020202020202020202020202020D4
:100C20002020202020202020202D2073686F772076
:100C3000765F696E2C2061312C20613220766F6CDA
:100C400074616765730A0D00616573205B6F6E7C6C
:100C50006F66665D2020202020202020202020207C
:100C6000202020202D20696E746567726574790AD2
:100C70000D00752020202020202020202020202052
:100C800020202020202020202020202020202D2057
:100C9000757074696D650A0D007620202020202073
:100CA0002020202020202020202020202020202044
:100CB00020202020202D2076657273696F6E0A0D2A
:100CC00000682020202020202020202020202020FC
:100CD000202020202020202020202020202D2068BF
:100CE000656C700A0D00256300756E6B6E6F776E14
:100CF00020636D640A004E48444330323136200090
:100D00004C334734323030442000484D4335383876
:100D10003320004144584C3334352000424D50308C
:100D200038352000484948363133302000415432AC
:100D3000344D41432000202573002025362E326695
:100D400020002530327800202573002025362E32F1
:100D500066204F6E2D426F6172640025303278003C
:100D60000A00452025642E256420636C6F636B2088
:100D7000256C752063707520256C75206C706D2056
:100D8000256C752069727120256C7520676C65640F
:100D900020256C7520796C656420256C7520726C3B
:100DA000656420256C7520747820256C75206C692D
:100DB0007374656E20256C752073656E736F727326
:100DC00020256C752073657269616C20256C750A2D
:100DD00000532025642E256420636C6F636B2025EF
:100DE0006C7520747820256C7520727820256C75C0
:100DF0002072747820256C752072727820256C75AD
:100E0000207265786D697420256C752061636B7440
:100E10007820256C75206E6F61636B747820256C6B
:100E2000752061636B727820256C752074696D651F
:100E3000646F757420256C752062616461636B72E8
:100E40007820256C7520746F6F6C6F6E6720256C31
:100E50007520746F6F73686F727420256C752062D3
:100E6000616473796E636820256C752062616463C8
:100E7000726320256C7520636F6E74656E74696F84
:100E80006E64726F7020256C752073656E64696E78
:100E90006764726F7020256C75206C6C74782025E7
:100EA0006C75206C6C727820256C750A0025732592
:100EB000730A004F6E6C696E650A000A002C20638D
:100EC0006865636B207261746520257520487A001F
:100ED00025732025732C206368616E6E656C202558
:100EE0007520706F776572202575000A0025783AA5
:100EF000004D414320616464726573732000526148
:100F00006E646F6D204555493634206164647265A6
:100F100073732067656E6572617465640A000A2ADE
:100F20002A2A2A2A2A2A426F6F74696E672025733B
:100F30002A2A2A2A2A2A2A0A00020000FFFE000082
:100F40000141544D45474131323872666131006C80
:100F50006F63616C686F737400454550524F4D204C
:100F6000697320636F72727570742C20726577726A
:100F70006974696E67207769746820646566617555
:100F80006C74732E0A006E616E00696E660000401C
:100F90007A10F35A00A0724E18090010A5D4E80088
:100FA00000E87648170000E40B54020000CA9A3BA0
:100FB000000000E1F5050000809698000000404226
:100FC0000F000000A08601000000102700000000B4
:100FD000E803000000006400000000000A000000B8
:100FE00000000100000000002C76D888DC674F0864
:100FF00023DFC1DFAE59E1B1B796E5E3E453C63A6A
:10100000E651997696E8E6C28426EB898C9B62EDE0
:10101000407C6FFCEFBC9C9F40F2BAA56FA5F4909A
:10102000055A2AF75C936B6CF9676DC11BFCE0E411
:101030000D47FEF520E6B500D0ED902E0300943567
:1010400077050080841E080000204E0A000000C8BA
:101050000C333333330F986E12831141EF8D21140B
:10106000893BE65516CFFEE6DB18D1844B381BF7DB
:101070007C1D901DA4BBE424203284725E2281007A
:10108000C9F124ECA1E53D27494E46494E49545942
:101090004E414ECDCCCC3D0AD7233C17B7D1387743
:1010A000CC2B329595E6241FB14F0A000020410059
:1010B00000C84200401C4620BCBE4CCA1B0E5AAEA3
:1010C000C59D740011241FBECFEFD1E4DEBFCDBF9C
:1010D00016E0A0E0B2E0E2EEFEEF00E00BBF02C0DF
:1010E00007900D92AE3CB107D9F71DE2AEECB6E029
:1010F00001C01D92A837B107E1F70E94D94D0C94A9
:101100006F7F0C94000029E0FC0120935700C895E4
:10111000802D0895E0919D17F0E0EF71F070EE5092
:10112000F84E808380919D178F5F80939D178091EB
:10113000B22488608093B2244FED54E0CA0161E18B
:101140000E94213F80E090E008954F925F926F925D
:101150007F928F929F92AF92BF92CF92DF92EF9247
:10116000FF920F931F93DF93CF93CDB7DEB76097B6
:101170000FB6F894DEBF0FBECDBF3B018091CE0607
:101180009091CF0681FD74980E94E9454C0183EF50
:1011900096E00E9418400AC0C8010296B3010E945E
:1011A000EE3C009701F5C8010E94DE40082F192F80
:1011B0000115110589F721C1C8010296B3010E94EA
:1011C000E53CD4018C918150F801808780E091E06A
:1011D000A0E0B0E081879287A387B48783EF96E091
:1011E000B8010E949F40C8010D9660E074E64FE18F
:1011F0005AE098010E94DD4284E00E941D47D80118
:1012000015969C938E93149783E00E941D472C01A2
:10121000F80197838683D401AC908085A81ABB24FB
:10122000CC24DD2486E0AA0CBB1CCC1CDD1C8A95DA
:10123000D1F7618572858385948520EC30E040E0AC
:1012400050E00E949078672F782F892F9927A60E5B
:10125000B71EC81ED91EF801A186B286C386D486E1
:10126000D4018C9180878091CE069091CF0681FD2C
:1012700008C08091B90480FD04C081FFB6C01D9BE9
:10128000B4C0EDB7FEB772970FB6F894FEBF0FBEAD
:10129000EDBFEDB6FEB60894E11CF11C80E092E0D3
:1012A00092838183C4010196D70113969C938E93F8
:1012B0001297F301808114968C93149715961C92C3
:1012C0001597818116968C93169717961C92D401C8
:1012D0008C91F70180871186D80114968D919C918D
:1012E00015979387828755864486BB27AD2D9C2D05
:1012F0008B2D97878687C601B50124E630E040E054
:1013000050E00E949078672F782F892F99270E94AC
:10131000D678F701718B608B0E94477C20919C04EA
:101320008DB79EB742960FB6F8949EBF0FBE8DBF85
:101330002223A9F000D000D0EDB7FEB7319687EE9A
:1013400091E0ADB7BEB712969C938E93119722830E
:1013500013820E94597C0F900F900F900F908091F4
:101360003B1C86FF42C00E94CF4BC40104960E94E2
:101370008E4BEDB7FEB73C970FB6F894FEBF0FBE8D
:10138000EDBF31967E010894E11CF11CADB7BEB7EC
:101390001296FC92EE92119780E190E09383828303
:1013A0008CE392E095838483D80114968D919C916F
:1013B00015979783868316968D919C9117979187A1
:1013C0008087D4018C91828713860E94B77CEDB709
:1013D000FEB73C960FB6F894FEBF0FBEEDBF82E09D
:1013E0000E94AB4BC7010E948E4B8091CE0690911C
:1013F000CF0681FF0DC0749A0BC088E495E00E946F
:10140000AC3F082F192F0115110509F0D5CEEDCFEE
:1014100060960FB6F894DEBF0FBECDBFCF91DF91BF
:101420001F910F91FF90EF90DF90CF90BF90AF9002
:101430009F908F907F906F905F904F900895EF9264
:10144000FF92CF93DF93E82EE7017E01F92EE701AB
:101450008091CE069091CF0687FF2FC08DB79EB7A3
:101460000C970FB6F8949EBF0FBE8DBFEDB7FEB7B9
:1014700031968FE492E0ADB7BEB712969C938E93EF
:1014800011978A81828313828B8184831582888558
:10149000868317828C819D81918780878E819F8131
:1014A000938782870E94477C2DB73EB7245F3F4FCA
:1014B0000FB6F8943EBF0FBE2DBF83EF96E0BE017E
:1014C0000E94664088E495E0BE010E94D23FDF9111
:1014D000CF91FF90EF90089587EE93E081159105ED
:1014E00011F00197F1F708958823E9F052985A987E
:1014F0001DBA80916900806280936900EA9A8091A8
:10150000B9049091BA0492FF12C053985B98EB9A79
:101510008091690080688093690080916800816093
:10152000809368000895109269005A9AEA98089585
:101530001F920F920FB60F9211248F939F93AF9328
:10154000BF938091680080FF20C080919224909189
:101550009324A0919424B09195240196A11DB11DCE
:101560008093922490939324A0939424B0939524F1
:101570008091CE069091CF0690FF07C0749882E0CC
:1015800090E090938F0480938E04BF91AF919F91D0
:101590008F910F900FBE0F901F9018951F920F9272
:1015A0000FB60F9211248F939F93AF93BF938091A7
:1015B000680080FF20C08091962490919724A0918C
:1015C0009824B09199240196A11DB11D8093962471
:1015D00090939724A0939824B09399248091CE0659
:1015E0009091CF0691FF07C0739882E090E09093AE
:1015F0008F0480938E04BF91AF919F918F910F9034
:101600000FBE0F901F90189580937C0080917B00F7
:10161000877F80937B0080917C00806C80937C002E
:1016200085E080937A0080917A00806880937A00C8
:1016300080917B0087FFFCCF80917B0085FFFCCFF2
:1016400080917A00806480937A0080917A0086FD90
:10165000FCCF109279001092780084E090E060E076
:1016600070E020917A00206420937A0020917A0023
:1016700026FDFCCF2091780030917900620F731F16
:10168000019779F710927C0080917A008F77809390
:101690007A00769567957695679580E090E00E9450
:1016A0001376089580E00E94040B209190043091FD
:1016B000910440919204509193040E94F17621EE9E
:1016C0003AE744E95EE30E94E174089580E1809383
:1016D0005101809351019091510195FF03C08F5F9B
:1016E0008F31B9F76BE4869FB0011124882777FD0D
:1016F0008095982F0E94157620E030E64FE954E45B
:101700000E94E17420E030E04AE754E40E94AB75A7
:1017100008958091B30484FF4BC080917B00886062
:1017200080937B0089EC80937C0085E080937A0035
:1017300080917A00806880937A0080917B0087FF97
:10174000FCCF80917B0085FFFCCF80917A00806484
:1017500080937A0080917A0086FDFCCF80917A0098
:10176000806480937A0080917A0086FDFCCF60913E
:1017700078007091790080E090E00E94137627ED68
:1017800033EA40E95FE30E94F17626E636E648E870
:1017900053E40E94E07460939217709393178093C0
:1017A00094179093951780917A008F7780937A00A1
:1017B00008956F927F928F929F92AF92BF92CF9235
:1017C000DF92EF92FF920F931F93DF93CF93CDB7EA
:1017D000DEB72A970FB6F894DEBF0FBECDBF3C012F
:1017E0001092D6068FEF89835EEAC52E57E1D52E7B
:1017F00000E010E042E0E42EF12CEC0EFD1E4E0164
:101800000894811C911C3AE0A32EB12CAC0EBD1E95
:101810003FC00830110509F441C0C401B7012A874F
:101820000E94DB4889812A858F3F11F08E3F19F491
:101830008093D60634C06114710479F4C7010E9404
:10184000F5488093AF24F701A7EAB4E281918D9324
:10185000EA15FB05D9F721E022C0C7010E94F5482F
:10186000F6018083D701F80123E0EE0FFF1F2A95D0
:10187000E1F7E00FF11FEA55F84E8D918193AA151B
:10188000BB05D9F70F5F1F4F89E090E0C80ED91E46
:10189000202F8981882309F0BCCF01C028E0822F46
:1018A0002A960FB6F894DEBF0FBECDBFCF91DF9161
:1018B0001F910F91FF90EF90DF90CF90BF90AF906E
:1018C0009F908F907F906F90089500D080E69DE06C
:1018D000EDB7FEB7928381830E94597C0F900F90E1
:1018E00008952F923F924F925F926F927F928F92C4
:1018F0009F92AF92BF92CF92DF92EF92FF920F939F
:101900001F93DF93CF9300D000D0CDB7DEB78C010B
:10191000009741F489E290E06BE270E04AE250E027
:1019200027E00AC08130910549F489E290E06BE23A
:1019300070E04AE250E026E00E94B747C8010E94EA
:10194000D90BF801EC52F94F808301151105A1F074
:101950001EEAC12E17E1D12E00E010E04F01B2E4E3
:101960006B2EBDE07B2EAAE34A2EADE05A2EF6E3A5
:101970002F2EFDE03F2EFAC087EA94E20E94274A0C
:101980009C01B901882777FD8095982F0E941576D4
:10199000C82EE92EE7EAAE2EE4E2BE2E0BE51DE0EE
:1019A000D5018D915D0100D000D0EDB7FEB7319625
:1019B000ADB7BEB712961C930E9311978283138214
:1019C0006B837C830E94597C0F900F900F900F9037
:1019D0006B817C81BFEAAB16B4E2BB0609F700D08D
:1019E00000D000D00DB71EB70F5F1F4F2BE43DE0B6
:1019F000EDB7FEB7328321838C2D9E2D20E030E0A1
:101A000048EC52E40E94AB75D80112966D937D9319
:101A10008D939C9315970E94597CEDB7FEB736962F
:101A20000FB6F894FEBF0FBEEDBF8091AF248823A0
:101A300019F08EE792E002C087E892E000D000D073
:101A400027E43DE0ADB7BEB712963C932E931197B5
:101A500014969C938E9313970E94597C0F900F902D
:101A60000F900F900E94650C88C0780163E0EE0C27
:101A7000FF1C6A95E1F7E00EF11EE6EAF7E1EE0ED3
:101A8000FF1EC7010E94274A9C01B901882777FDE4
:101A90008095982F0E9415765C0120E030E0D701F8
:101AA0008D917D0100D000D0EDB7FEB73196ADB776
:101AB000BEB712967C926E9211978283138229830D
:101AC0003A836B837C830E94597C29813A812F5F02
:101AD0003F4F0F900F900F900F906B817C812830BB
:101AE0003105E9F600D000D000D0EDB6FEB608947E
:101AF000E11CF11CEDB7FEB7528241828A2D9B2D6D
:101B000020E030E048EC52E40E94AB75D701129619
:101B10006D937D938D939C9315970E94597CEDB79F
:101B2000FEB736960FB6F894FEBF0FBEEDBFD601D6
:101B30008C91882319F08EE792E002C087E892E04A
:101B400000D000D0EDB7FEB7328221829483838328
:101B50000E94597C0F900F900F900F900E94650C7F
:101B60000F5F1F4F29E030E0C20ED31ED4018C91CD
:101B700090E0081719070CF478CF0F900F900F9092
:101B80000F90CF91DF911F910F91FF90EF90DF9019
:101B9000CF90BF90AF909F908F907F906F905F900D
:101BA0004F903F902F900895DF93CF9300D0CDB703
:101BB000DEB78091A82489838091AE248A83CE01E8
:101BC00001960E94003D0F900F90CF91DF910895F4
:101BD000CF93DF93EC018091A7248F3FB1F58091E3
:101BE000A8248F3F91F58091A9248F3F71F58091B2
:101BF000AA248F3F51F58091AB248F3F31F580911E
:101C0000AC248F3F11F58091AD248F3FF1F480918A
:101C1000AE248F3FD1F489E290E06BE270E04AE2BB
:101C200050E027E00E94B74780E090E00E94D90B87
:101C3000CC52D94F888387EA94E267E170E049E0AB
:101C400050E00E94A97D0E94D40DDF91CF910895AC
:101C50001F920F920FB60F920BB60F9211242F9373
:101C60003F934F935F936F937F938F939F93AF9324
:101C7000BF93EF93FF938091B22482608093B2244C
:101C80008091B90486FD2B9A8091B90487FD2B9A27
:101C900080918E0490918F041816190614F4749A8A
:101CA000739A8091CE069091CF0685FF02C07498FA
:101CB000739880915005909151050197909351052B
:101CC00080935005009709F068C0809102079091B9
:101CD00003070196909303078093020720913D200C
:101CE00030913E2040913F20509140202F5F3F4F48
:101CF0004F4F5F4F20933D2030933E2040933F2035
:101D00005093402020E130E030935105209350055E
:101D10002091B90420FD02C01D9B05C01092D2067F
:101D20001092D10606C021E030E03093D206209315
:101D3000D1066091B7047091B8046115710599F0EE
:101D400001960E94AF78009771F477988091CE0643
:101D50009091CF0693FF07C0749884E090E0909331
:101D60008F0480938E046091B7047091B80461155C
:101D7000710579F080910207909103070E94AF7876
:101D8000009739F48BEF94E062E140E050E00E946C
:101D9000213F8091B90486FD2B988AE695E060E0AA
:101DA00040E050E00E94213FFF91EF91BF91AF9141
:101DB0009F918F917F916F915F914F913F912F9163
:101DC0000F900BBE0F900FBE0F901F901895809133
:101DD0009D1790915120891B08950E94E70E88233A
:101DE00079F0E0915120F0E0EF71F070EE50F84E94
:101DF000208130E0809151208F5F8093512002C07C
:101E00002FEF3FEFC9010895CF93DF93EC011092BC
:101E1000F6061092F50688819981009731F022E04C
:101E2000833C920709F0B9C009C00E94E70E8823DD
:101E300041F483EC92E099838883B3C0613109F067
:101E4000B0C0F89478940E94ED0E90E09093FA065A
:101E50008093F9068D3009F47CC08F3F31F38231D5
:101E6000910569F18F37910521F08830910509F0CE
:101E700053C08091FD069091FE06181619060CF0CD
:101E800060C06091722D7091732D88E090E00E9487
:101E90001B7C6091722D7091732D80E290E00E9406
:101EA0001B7C6091722D7091732D88E090E00E94F0
:101EB0001B7C8091FD069091FE0601973EC06091CB
:101EC000722D7091732D8DE090E00E941B7C10921A
:101ED000FC061092FB0614C08E5A9F4DFC018081B7
:101EE0006091722D7091732D90E00E941B7C809107
:101EF000FB069091FC0601969093FC068093FB06EE
:101F00008091FB069091FC062091FD063091FE0623
:101F1000821793070CF315C06091722D7091732D89
:101F20000E941B7C8091FD069091FE062091F9068F
:101F3000FC01EE5AFF4D208301969093FE0680939C
:101F4000FD068091FD069091FE068F33910509F004
:101F50006CCF109251208091512080939D178091D9
:101F6000FD069091FE06FC01EE5AFF4D1082909303
:101F7000F6068093F5061092FE061092FD068091FB
:101F8000B0249091B124009709F44FCF6091F706E7
:101F900040E050E00E94213F48CF1982188283E040
:101FA00001C081E0DF91CF91089578948091D106AE
:101FB0009091D206009731F08091B9049091BA04C3
:101FC00091FF03C083B7817F03C083B7817F8660A1
:101FD00083BFF89483B7816083BF7894889583B773
:101FE0008E7F83BF78940895CF93DF93EC0188812F
:101FF0009981009721F02AE08635920799F40E9492
:1020000030510E94D50F8091880E9091890E65E81D
:1020100040E050E00E94213F86E59AE09983888362
:1020200081E003C01982188283E0DF91CF91089587
:10203000CF93DF930E94305180EB0E94A74A882300
:10204000B1F40E940D4B80913B1C90913C1C81602F
:1020500090933C1C80933B1C00D08DE29DE0EDB73B
:10206000FEB7928381830E94597C0F900F908EB1AE
:10207000C82FD0E0C470D070729A0E9430518EE4A4
:102080000E94A74A8823B1F40E940D4B80913B1C0B
:1020900090913C1C826090933C1C80933B1C00D030
:1020A00084E29DE0EDB7FEB7928381830E94597C64
:1020B0000F900F90209709F472980E9430518EEE85
:1020C0000E94A74A8823B1F40E940D4B80913B1CCB
:1020D00090913C1C846090933C1C80933B1C00D0EE
:1020E0008CE19DE0EDB7FEB7928381830E94597C1D
:1020F0000F900F9086EA0E94A74A8823B1F40E94AD
:102100000D4B80913B1C90913C1C886090933C1C33
:1021100080933B1C00D083E19DE0EDB7FEB7928336
:1021200081830E94597C0F900F900E9430518CE364
:102130000E94A74A8823B1F40E940D4B80913B1C5A
:1021400090913C1C806190933C1C80933B1C00D080
:102150008AE09DE0EDB7FEB7928381830E94597CAF
:102160000F900F900E94305182ED0E94A74A882361
:10217000B1F40E940D4B80913B1C90913C1C8062FD
:1021800090933C1C80933B1C00D080E09DE0EDB719
:10219000FEB7928381830E94597C0F900F90C7E015
:1021A000D0E00E9430518CE70E94A74A8823B9F4FE
:1021B0000E940D4B80913B1C90913C1C806490933D
:1021C0003C1C80933B1C00D086EF9CE0EDB7FEB733
:1021D000928381830E94597C0F900F9002C02197B7
:1021E00001F70E940D4B0E94650CDF91CF9108957D
:1021F000DF93CF9300D0CDB7DEB74A8369830E94C7
:10220000E34A6981862F0E94154B4A81842F0E94E0
:10221000154B0E940D4B0F900F90CF91DF910895B9
:10222000AF92BF92DF92EF92FF920F931F93DF93D3
:10223000CF9300D00F92CDB7DEB7082FD22E4A83AE
:102240005B8369830E94E34A6981862F0E94154B54
:10225000802F81600E940A4B4A815B81042F152FD9
:10226000AA24BB24ED2CFF240894E108F1080FC038
:10227000AE14BF0419F40E94304B02C00E94264BDA
:10228000F80180830894A11CB11C0F5F1F4FAD148F
:1022900078F30E940D4B0F900F900F90CF91DF912C
:1022A0001F910F91FF90EF90DF90BF90AF90089536
:1022B000AF92BF92CF92DF92EF92FF920F931F9354
:1022C000DF93CF93CDB7DEB760970FB6F894DEBF3C
:1022D0000FBECDBFB82EA42E662309F455C0AE01A3
:1022E0004F5F5F4F80E1DA011D928A95E9F780EB3D
:1022F00068E928E00E941011BB2059F000D088E85E
:1023000092E0EDB7FEB7928381830E94477C0F90E5
:102310000F908E010F5F1F4F38E0E32EF12CEC0E73
:10232000FD1E2FE8C22E22E0D22ED8018D918D0104
:1023300000D000D0EDB7FEB73196ADB7BEB712965C
:10234000DC92CE921197828313820E94477C0F9079
:102350000F900F900F900E151F0539F700D000D089
:10236000EDB7FEB7319684E992E0ADB7BEB71296ED
:102370009C938E9311978885828313820E94477C59
:102380000F900F900F900F90AA2009F457C0AE0144
:102390004F5F5F4F80E1FA0111928A95E9F780EB78
:1023A00060E828E00E941011BB2069F000D08AE9A3
:1023B00092E0ADB7BEB712969C938E9311970E9490
:1023C000477C0F900F908E010F5F1F4F90E1E92E19
:1023D000F12CEC0EFD1E8FE8C82E82E0D82EF801FD
:1023E00081918F0100D000D0EDB7FEB73196ADB727
:1023F000BEB71296DC92CE921197828313820E940E
:10240000477C0F900F900F900F900E151F0539F716
:1024100000D000D0EDB7FEB7319684E992E0ADB7B9
:10242000BEB712969C938E931197888582831382F0
:102430000E94477C0F900F900F900F9060960FB600
:10244000F894DEBF0FBECDBFCF91DF911F910F91EA
:10245000FF90EF90DF90CF90BF90AF9008950F93D3
:102460001F93DF93CF9300D0CDB7DEB71A821982C6
:102470008EEE6AEA8E010F5F1F4FA80122E00E94D4
:102480001011398120E08A8190E0822B932B909368
:102490001318809312188EEE6CEAA80122E00E94B5
:1024A0001011398120E08A8190E0822B932B909348
:1024B0001518809314188EEE6EEAA80122E00E948F
:1024C0001011398120E08A8190E0822B932B909328
:1024D0001718809316188EEE60EBA80122E00E9478
:1024E0001011398120E08A8190E0822B932B909308
:1024F0002518809324188EEE62EBA80122E00E943A
:102500001011398120E08A8190E0822B932B9093E7
:102510002718809326188EEE64EBA80122E00E9413
:102520001011398120E08A8190E0822B932B9093C7
:102530002918809328188EEE66EBA80122E00E94ED
:102540001011398120E08A8190E0822B932B9093A7
:102550001918809318188EEE68EBA80122E00E94EB
:102560001011398120E08A8190E0822B932B909387
:102570001B1880931A188EEE6AEBA80122E00E94C5
:102580001011398120E08A8190E0822B932B909367
:102590001F1880931E188EEE6CEBA80122E00E949B
:1025A0001011398120E08A8190E0822B932B909347
:1025B0002118809320188EEE6EEBA80122E00E9475
:1025C0001011398120E08A8190E0822B932B909327
:1025D0002318809322180F900F90CF91DF911F91B5
:1025E0000F9108952F923F924F925F926F927F9238
:1025F0008F929F92AF92BF92CF92DF92EF92FF9213
:102600000F931F93DF93CF93CDB7DEB76C970FB6C1
:10261000F894DEBF0FBECDBFA82E4A8B2B8FFE01D4
:10262000319683E0DF011D928A95E9F78091361893
:10263000882339F46C8F0E942F1281E08093361822
:102640006C8D662309F475C08EEE64EF4EE20E9435
:10265000F81069E07AE180E090E00E94944A8EEE02
:1026600066EFAE014F5F5F4F22E00E94101169815B
:1026700070E080E090E0982F872F762F66272A81E0
:1026800030E040E050E0622B732B842B952B20919F
:1026900028183091291840E050E0621B730B840B1E
:1026A000950B209126183091271840E050E00E94A9
:1026B00090787B018C013FE015950795F794E7949E
:1026C0003A95D1F76091201870912118882777FDED
:1026D0008095982F2BE0660F771F881F991F2A95EA
:1026E000D1F72091221830912318442737FD4095C7
:1026F000542F2E0D3F1D401F511F0E94F8782E0DA4
:102700003F1D30931D1820931C18285F3F4F14E085
:10271000359527951A95E1F779010027F7FC009583
:10272000102FE0922A18F0922B1800932C18109377
:102730002D18BA2DB295BB0FBB0FB07CBC5CB9870E
:102740002A2D30E03E8B2D8B63E070E00A2C02C016
:10275000660F771F0A94E2F7882777FD8095982FF8
:1027600025E335E040E050E00E949078DC01CB01A9
:102770000296A11DB11D8A879B87AC87BD8720E586
:1027800033EC40E050E004C05595479537952795C8
:10279000AA94D2F72E873F87488B598B18861C82C4
:1027A0001D821E821F8248E050E08D899E89481B51
:1027B000590B5C8B4B8B69C18EEE64EF49850E948F
:1027C000F8106A857B858C859D850E94944A8EEEE3
:1027D00066EFAE014F5F5F4F23E00E9410118091C2
:1027E0001C1890911D18805A9F401C01442437FCEE
:1027F0004094542CC201B101A20191010E94907831
:102800006F8B788F898F9A8F2091161830911718B7
:10281000442737FD4095542FC201B1010E949078A2
:102820007B018C01BDE015950795F794E794BA9567
:10283000D1F722E030E040E050E0E20EF31E041F4A
:10284000151F6F89788D898D9A8DACE09595879548
:1028500077956795AA95D1F7209118183091191896
:10286000442737FD4095542F0E949078BC0199274A
:1028700077FD9095892FE60EF71E081F191FE2E0DD
:1028800015950795F794E794EA95D1F780E090E8DD
:10289000A0E0B0E0E80EF91E0A1F1B1F20912418CB
:1028A0003091251840E050E0C801B7010E949078AF
:1028B0003B014C017FE096948794779467947A95D6
:1028C000D1F7A980BB24CC24DD246501BB24AA2434
:1028D0008A8190E0A0E0B0E0BA2FA92F982F882736
:1028E000A82AB92ACA2ADB2A8B8190E0A0E0B0E0AE
:1028F000A82AB92ACA2ADB2A0B8804C0D594C7940F
:10290000B794A7940A94D2F720911418309115180F
:10291000442737FD4095542FC201B1010E949078A1
:102920007B018C014BE015950795F794E7944A9548
:10293000D1F78091121890911318AA2797FDA095AE
:10294000BA2F32E0880F991FAA1FBB1F3A95D1F703
:10295000E80EF91E0A1F1B1F20911A1830911B1830
:10296000442737FD4095542F6F89788D898D9A8D36
:102970000E94907827E195958795779567952A9598
:10298000D1F7E60EF71E081F191F0D8804C0EE0CC4
:10299000FF1C001F111F0A94D2F722E030E040E034
:1029A00050E0E20EF31E041F151F82E015950795F7
:1029B000F794E7948A95D1F7AE18BF08C00AD10AF8
:1029C000C601B5012E853F85488959890E949078B6
:1029D00097FD0BC0660F771F881F991FA4019301F5
:1029E0000E94D67879018A010AC0A40193010E944D
:1029F000D67879018A01EE0CFF1C001F111F5527A4
:102A000017FD5A95412F302F2F2DCA01B9010E9471
:102A100090782EED3BE040E050E00E9490785B0122
:102A20006C01C801B70123E433EE4FEF5FEF0E9462
:102A30009078BC01992777FD9095892F6153714F4C
:102A40008F4F9F4F5601DD24B7FCD094CD2C6A0DDB
:102A50007B1D8C1D9D1D44E0959587957795679509
:102A60004A95D1F76E0D7F1D801F911F2C813D81EE
:102A70004E815F81260F371F481F591F2C833D83CE
:102A80004E835F8338853F5F388748855A8945176D
:102A900008F492CE552391F0252F30E040E050E02D
:102AA0006C817D818E819F810E94D67820932E1823
:102AB00030932F1840933018509331188B8D882302
:102AC000C9F160912E1870912F1880913018909153
:102AD0003118611571058105910561F10E94157626
:102AE00020E836EE45EC57E40E94AB7521E03EED60
:102AF00042E45EE30E945477562F472F382F292F48
:102B000060E070E080E89FE3DA01F9012B2F3A2FB3
:102B10004F2F5E2F0E94E0742BE43AE34DEB57E316
:102B20000E94AB75609332187093331880933418F9
:102B3000909335186C960FB6F894DEBF0FBECDBFDC
:102B4000CF91DF911F910F91FF90EF90DF90CF9089
:102B5000BF90AF909F908F907F906F905F904F90BD
:102B60003F902F900895DF93CF9300D000D000D0F6
:102B7000CDB7DEB7FE01319686E0DF011D928A9562
:102B8000E9F780919C17882399F486EA61E340E095
:102B90000E94F81086EA6CE24AE00E94F81081E098
:102BA00080939C176CE77EE380E090E00E94944A5B
:102BB00086EA6DE248E00E94F8106CE77EE380E070
:102BC00090E00E94944A86EA62E3AE014F5F5F4F55
:102BD00026E00E94101186EA6DE247E00E94F8109C
:102BE0009A8180E0498150E0482B592B50939717E8
:102BF000409396179C8180E02B8130E0282B392B65
:102C000030939917209398177E8160E08D8190E032
:102C1000862B972B90939B1780939A176DB77EB74F
:102C2000685070400FB6F8947EBF0FBE6DBFEDB711
:102C3000FEB731966EE972E0ADB7BEB712967C93DF
:102C40006E931197538342833583248397838683BE
:102C50000E94477C6DB77EB7685F7F4F0FB6F894D0
:102C60007EBF0FBE6DBF26960FB6F894DEBF0FBEB7
:102C7000CDBFCF91DF910895CF92DF92EF92FF9277
:102C80000F931F93DF93CF9300D000D000D0CDB728
:102C9000DEB78E010F5F1F4F86E0F80111928A9513
:102CA000E9F78CE362E041E00E94F8108CE360E019
:102CB00048E50E94F81062E174E380E090E00E9431
:102CC000944A8CE363E0A80126E00E9410118CE393
:102CD00062E043E00E94F810998180E00A8110E0F0
:102CE000082B192B10937D1700937C179B8180E094
:102CF0006C8170E0682B792B70937F1760937E173F
:102D00003D8120E08E8190E0822B932B9093811760
:102D100080938017882777FD8095982F0E941576DD
:102D20006B017C01B801882777FD8095982F0E9460
:102D300015769B01AC01C701B6010E9454752DB7F1
:102D40003EB72C5030400FB6F8943EBF0FBE2DBF9B
:102D50000DB71EB70F5F1F4F2CEA32E0EDB7FEB77D
:102D60003283218320917C1730917D17F8013383C2
:102D7000228320917E1730917F1735832483209101
:102D80008017309181173783268320EE3EE245E697
:102D900052E40E94F17620E030E044E353E40E94E4
:102DA000E174F80160877187828793870E94477C6E
:102DB0002DB73EB7245F3F4F0FB6F8943EBF0FBE0E
:102DC0002DBF26960FB6F894DEBF0FBECDBFCF91B4
:102DD000DF911F910F91FF90EF90DF90CF900895BA
:102DE000CF93DF93EC0188819981009731F02AE03D
:102DF0008F33920709F071C00BC087ED96E060E851
:102E000070E00E94D7418FE39AE09983888369C07C
:102E100087ED96E00E940242009709F462C080911B
:102E2000CE069091CF0694FF3FC080913B1C82FF5D
:102E30003BC083E061E048E021E00E94F2128DB7E0
:102E40009EB70A970FB6F8949EBF0FBE8DBFEDB721
:102E5000FEB731968FEC91E0ADB7BEB712969C935A
:102E60008E93119780912E1890912F18A091301861
:102E7000B091311882839383A483B58380913218F3
:102E800090913318A0913418B091351886839783A8
:102E9000A087B1870E94597C8DB79EB70A960FB65E
:102EA000F8949EBF0FBE8DBF8091CE069091CF0645
:102EB00095FF06C080913B1C83FF02C00E94B315A2
:102EC0008091CE069091CF0696FF97CF80913B1CC4
:102ED00084FF93CF0E943C1690CF1982188283E022
:102EE00001C081E0DF91CF910895CF92DF92FF92F0
:102EF0000F931F93CF93DF93729A8091B90483FD50
:102F000006C0C0E5D0E00E946C0A2197E1F78EE48C
:102F10000E94A74A8823B1F08091412090914220DD
:102F2000A0914320B09144200196A11DB11D809332
:102F3000412090934220A0934320B093442021E06D
:102F400030E084C0C0E5D0E00E946C0A2197E1F730
:102F50008FE40E94A74A0E94264BF82E8295869500
:102F6000869583708130A9F42091452030914620C8
:102F700040914720509148202F5F3F4F4F4F5F4F68
:102F8000209345203093462040934720509348207B
:102F900016C08230A0F02091492030914A20409103
:102FA0004B2050914C202F5F3F4F4F4F5F4F20934E
:102FB000492030934A2040934B2050934C200E944C
:102FC000264B1F2D1F7300E0080F111D0E94264B7A
:102FD0000E94304B20E0E901C80FD11DD695C7955E
:102FE000D695C7950E940D4B8091B90483FF7298C6
:102FF000B80180E090E00E94137620E134E048ECD4
:103000005BE30E94F17660933718709338188093D1
:10301000391890933A18BE0180E090E00E94137630
:1030200024EA3CEF44E25CE30E94F17620E030E0E9
:1030300040E252E40E94E0746093B3247093B4249D
:103040008093B5249093B62420E030E0C901DF914D
:10305000CF911F910F91FF90DF90CF9008957298BC
:10306000729A8EE40E94A74A80EA0E94154B80E083
:103070000E94154B80E00E94154B8FE40E94A74AE6
:103080000E94264B82958695869583708130A9F49F
:103090002091452030914620409147205091482072
:1030A0002F5F3F4F4F4F5F4F209345203093462077
:1030B000409347205093482016C08230A0F02091C2
:1030C000492030914A2040914B2050914C202F5F55
:1030D0003F4F4F4F5F4F2093492030934A204093FA
:1030E0004B2050934C2000D000D0EDB7FEB7319666
:1030F00021EC32E0ADB7BEB712963C932E931197F8
:10310000828313820E94477C0F900F900F900F9044
:103110008EE40E94A74A80E80E94154B80E00E943E
:10312000154B80E00E94154B0E940D4B80E090E013
:10313000089500D089EE9CE0ADB7BEB712969C937F
:103140008E9311970E94597C20919C040F900F90B0
:103150002223A9F000D000D0EDB7FEB7319686EE5D
:103160009CE0ADB7BEB712969C938E9311972283C5
:1031700013820E94597C0F900F900F900F9008952A
:1031800000D081EC9CE0EDB7FEB7928381830E9472
:10319000597C89E99CE0EDB7FEB7928381830E9458
:1031A000597C82E79CE0EDB7FEB7928381830E9451
:1031B000597C88E49CE0EDB7FEB7928381830E943E
:1031C000597C8DE09CE0EDB7FEB7928381830E942D
:1031D000597C8BED9BE0EDB7FEB7928381830E9413
:1031E000597C85EB9BE0EDB7FEB7928381830E940B
:1031F000597C85E89BE0EDB7FEB7928381830E94FE
:10320000597C8CE49BE0EDB7FEB7928381830E94EA
:10321000597C80E29BE0EDB7FEB7928381830E94E8
:10322000597C87EF9AE0EDB7FEB7928381830E94C5
:10323000597C8CEC9AE0EDB7FEB7928381830E94B3
:10324000597C8DE99AE0EDB7FEB7928381830E94A5
:10325000597C8BE69AE0EDB7FEB7928381830E949A
:10326000597C8AE39AE0EDB7FEB7928381830E948E
:10327000597C86E09AE0EDB7FEB7928381830E9485
:10328000597C86ED99E0EDB7FEB7928381830E9469
:10329000597C8AEA99E0EDB7FEB7928381830E9458
:1032A000597C8BE799E0EDB7FEB7928381830E944A
:1032B000597C82E499E0EDB7FEB7928381830E9446
:1032C000597C89E199E0EDB7FEB7928381830E9432
:1032D000597C8AED98E0EDB7FEB7928381830E9416
:1032E000597C8BEA98E0EDB7FEB7928381830E9408
:1032F000597C8CE798E0EDB7FEB7928381830E94FA
:10330000597C85E598E0EDB7FEB7928381830E94F2
:10331000597C8FE198E0EDB7FEB7928381830E94DC
:10332000597C86EF97E0EDB7FEB7928381830E94C8
:10333000597C8BEC97E0EDB7FEB7928381830E94B6
:10334000597C0F900F90089581ED92E00E94807C4F
:1033500008952F923F924F925F926F927F928F9239
:103360009F92AF92BF92CF92DF92EF92FF920F9314
:103370001F93CF93DF9360913D2070913E20809109
:103380003F2090914020A0903D20B0903E20C090E2
:103390003F20D090402060903D2070903E20809053
:1033A0003F209090402020903D2030903E20409043
:1033B0003F20509040202DB73EB72A5030400FB6E6
:1033C000F8943EBF0FBE2DBFCDB7DEB721962BEAD6
:1033D00037E0EDB7FEB732832183A0E8EA2EA1E5FE
:1033E000FA2EA1E00A2F112DA80197010E94D6788C
:1033F0003B832A83C601B501A80197010E94D678B4
:10340000F0E1EF2EFEE0FF2E012D112DA801970116
:103410000E94D678332727FD30953D832C83C40145
:10342000B301A80197010E94D678ECE3EE2EF12CAF
:10343000012D112DA80197010E94D678332727FD71
:1034400030953F832E83C201B101A80197010E94EC
:10345000D678772767FD7095798768870E94597CB1
:103460002DB73EB7265F3F4F0FB6F8943EBF0FBE55
:103470002DBFDF91CF911F910F91FF90EF90DF90C3
:10348000CF90BF90AF909F908F907F906F905F9004
:103490004F903F902F900895E8E7FDE28081918161
:1034A00022E482349207B9F000D000D08DE897E092
:1034B000ADB7BEB712969C938E931197E857FD4215
:1034C0001496FC93EE9313970E94597C0F900F90E3
:1034D0000F900F9008953A96B1E4E53FFB07F0F2A4
:1034E00008958F929F92AF92BF92CF92DF92EF9208
:1034F000FF920F931F938C9A0E94520B00D000D022
:1035000000D026E837E0ADB7BEB712963C932E93B5
:103510001197EDB7FEB763837483858396830E940A
:10352000597C8DB79EB706960FB6F8949EBF0FBE16
:103530008DBF81E00E94040B20919404309195048A
:1035400040919604509197040E94F1767B018C0182
:1035500082E00E94040B20919804309199044091DC
:103560009A0450919B040E94F176B62EC72ED82E55
:10357000A92E83E00E94040B9B01AC01ADB7BEB73E
:103580001E970FB6F894BEBF0FBEADBFEDB7FEB726
:10359000319684E797E012969C938E931197C7011A
:1035A000A02FB12F82839383A483B5830B2D1C2D71
:1035B000C801AD2DBA2D86839783A087B187228756
:1035C0003387448755870E94597C8C98EDB7FEB7A6
:1035D0003E960FB6F894FEBF0FBEEDBF0E94650C7D
:1035E0001F910F91FF90EF90DF90CF90BF90AF9021
:1035F0009F908F9008950F931F93CF93DF9388230D
:1036000089F087EA94E26FEF70E049E050E00E94B1
:10361000D17B87EA94E267E170E049E050E00E94E4
:10362000A97D1CC0C7EAD4E20FE617E0899100D05B
:1036300000D0EDB7FEB73196ADB7BEB712961C936A
:103640000E931197828313820E94597C0F900F90E2
:103650000F900F90B4E2CF3ADB0741F70E94650C60
:10366000DF91CF911F910F910895EF92FF920F93E9
:103670001F936091A1047091A20480E090E00E94E9
:10368000C37B65EF72E00E94D87B009709F08BC086
:1036900086E294E9A0E0B0E08093B3049093B40490
:1036A000A093B504B093B60483EB94E06EE070E0B1
:1036B00044E050E00E94A97D8CE390E09093B80430
:1036C0008093B70487EB94E062E170E042E050E061
:1036D0000E94A97D8AE090E09093BA048093B90497
:1036E00089EB94E064E170E042E050E00E94A97D43
:1036F0001092CF061092CE068EEC96E060E070E05D
:1037000042E050E00E94A97D0F2EF2E2EF2EFFEF83
:10371000FF2EFCEC0F2FFBE31F2FF02DE092940403
:10372000F0929504009396041093970484E994E032
:1037300066E070E044E050E00E94A97DE0929804C9
:10374000F092990400939A0410939B0488E994E002
:103750006AE070E044E050E00E94A97D87ED94E3C8
:10376000AFEEBCE38093900490939104A0939204F5
:10377000B093930480E994E062E070E044E050E0AC
:103780000E94A97D1092D30683ED96E066E170E079
:1037900041E050E00E94A97D81E00E94FB1A80E098
:1037A00090E00E94E80D1F910F91FF90EF90089517
:1037B000882309F44BC18091B30480FF0BC000D073
:1037C00089E697E0EDB7FEB7928381830E94597C2A
:1037D0000F900F908091B30481FF0BC000D082E660
:1037E00097E0EDB7FEB7928381830E94597C0F90DA
:1037F0000F908091B30482FF0BC000D08DE597E05D
:10380000EDB7FEB7928381830E94597C0F900F9091
:103810008091B30483FF0BC000D087E597E0EDB73C
:10382000FEB7928381830E94597C0F900F90809104
:10383000B30484FF0BC000D08EE497E0EDB7FEB771
:10384000928381830E94597C0F900F908091B304E2
:1038500085FF0BC000D085E497E0EDB7FEB79283FB
:1038600081830E94597C0F900F908091B30486FF52
:103870000BC000D08FE397E0EDB7FEB79283818352
:103880000E94597C0F900F908091B30487FF0BC06A
:1038900000D087E397E0EDB7FEB7928381830E9463
:1038A000597C0F900F908091B3049091B404A09133
:1038B000B504B091B60490FF0BC000D081E397E04F
:1038C000EDB7FEB7928381830E94597C0F900F90D1
:1038D0008091B3049091B404A091B504B091B60462
:1038E00091FF0BC000D089E297E0EDB7FEB792835D
:1038F00081830E94597C0F900F908091B304909126
:10390000B404A091B504B091B60492FF0BC000D0EE
:103910008FE197E0EDB7FEB7928381830E94597CD7
:103920000F900F908091B3049091B404A091B504CE
:10393000B091B60493FF0BC000D089E197E0EDB7DA
:10394000FEB7928381830E94597C0F900F908091E3
:10395000B3049091B404A091B504B091B60494FF5F
:103960000BC000D081E197E0EDB7FEB79283818371
:103970000E94597C0F900F908091B3049091B404F1
:10398000A091B504B091B60495FF0BC000D08BE0B8
:1039900097E0EDB7FEB7928381830E94597C0F9028
:1039A0000F908091B3049091B404A091B504B091AC
:1039B000B60496FF0BC000D085E097E0EDB7FEB7E8
:1039C000928381830E94597C0F900F908091B30461
:1039D0009091B404A091B504B091B60497FF0BC0C8
:1039E00000D08FEF96E0EDB7FEB7928381830E94FF
:1039F000597C0F900F908091B3049091B404A091E2
:103A0000B504B091B604A0FF0BC000D08AEF96E0D9
:103A1000EDB7FEB7928381830E94597C0F900F907F
:103A20008091B3049091B404A091B504B091B60410
:103A3000A1FF14C200D084EF96E0EDB7FEB79283E9
:103A400081830E94597C0F900F9008C200D000D053
:103A500000D088EE96E0EDB7FEB79283818381E0D7
:103A600090E0A0E0B0E083839483A583B6830E94B6
:103A7000597C8DB79EB706960FB6F8949EBF0FBEC1
:103A80008DBF0E94650C00D000D000D08BED96E079
:103A9000EDB7FEB79283818382E090E0A0E0B0E0D2
:103AA00083839483A583B6830E94597C8DB79EB788
:103AB00006960FB6F8949EBF0FBE8DBF0E94650C90
:103AC00000D000D000D080ED96E0EDB7FEB7928335
:103AD000818384E090E0A0E0B0E083839483A583B9
:103AE000B6830E94597C8DB79EB706960FB6F894A0
:103AF0009EBF0FBE8DBF0E94650C00D000D000D0CD
:103B000084EC96E0EDB7FEB79283818388E090E085
:103B1000A0E0B0E083839483A583B6830E94597CA0
:103B20008DB79EB706960FB6F8949EBF0FBE8DBF99
:103B30000E94650C00D000D000D086EB96E0EDB777
:103B4000FEB79283818380E190E0A0E0B0E08383C0
:103B50009483A583B6830E94597C8DB79EB7069641
:103B60000FB6F8949EBF0FBE8DBF0E94650C00D0AB
:103B700000D000D088EA96E0EDB7FEB7928381834B
:103B800080E290E0A0E0B0E083839483A583B683D5
:103B90000E94597C8DB79EB706960FB6F8949EBFCB
:103BA0000FBE8DBF0E94650C00D000D000D08CE904
:103BB00096E0EDB7FEB79283818380E490E0A0E0C9
:103BC000B0E083839483A583B6830E94597C8DB72C
:103BD0009EB706960FB6F8949EBF0FBE8DBF0E948B
:103BE000650C00D000D000D08EE896E0EDB7FEB7AF
:103BF0009283818380E890E0A0E0B0E083839483A7
:103C0000A583B6830E94597C8DB79EB706960FB6E2
:103C1000F8949EBF0FBE8DBF0E94650C00D000D0EF
:103C200000D082E896E0EDB7FEB79283818380E012
:103C300091E0A0E0B0E083839483A583B6830E94E3
:103C4000597C8DB79EB706960FB6F8949EBF0FBEEF
:103C50008DBF0E94650C00D000D000D084E796E0B4
:103C6000EDB7FEB79283818380E092E0A0E0B0E000
:103C700083839483A583B6830E94597C8DB79EB7B6
:103C800006960FB6F8949EBF0FBE8DBF0E94650CBE
:103C900000D000D000D085E696E0EDB7FEB7928365
:103CA000818380E094E0A0E0B0E083839483A583E7
:103CB000B6830E94597C8DB79EB706960FB6F894CE
:103CC0009EBF0FBE8DBF0E94650C00D000D000D0FB
:103CD00089E596E0EDB7FEB79283818380E098E0B6
:103CE000A0E0B0E083839483A583B6830E94597CCF
:103CF0008DB79EB706960FB6F8949EBF0FBE8DBFC8
:103D00000E94650C00D000D000D08BE496E0EDB7A7
:103D1000FEB79283818380E090E1A0E0B0E08383EE
:103D20009483A583B6830E94597C8DB79EB706966F
:103D30000FB6F8949EBF0FBE8DBF0E94650C00D0D9
:103D400000D000D08FE396E0EDB7FEB79283818379
:103D500080E090E2A0E0B0E083839483A583B68303
:103D60000E94597C8DB79EB706960FB6F8949EBFF9
:103D70000FBE8DBF0E94650C00D000D000D083E341
:103D800096E0EDB7FEB79283818380E090E4A0E0F7
:103D9000B0E083839483A583B6830E94597C8DB75A
:103DA0009EB706960FB6F8949EBF0FBE8DBF0E94B9
:103DB000650C00D000D000D087E296E0EDB7FEB7EA
:103DC0009283818380E090E8A0E0B0E083839483D5
:103DD000A583B6830E94597C8DB79EB706960FB611
:103DE000F8949EBF0FBE8DBF0E94650C00D000D01E
:103DF00000D08BE196E0EDB7FEB79283818380E03F
:103E000090E0A1E0B0E083839483A583B6830E9411
:103E1000597C8DB79EB706960FB6F8949EBF0FBE1D
:103E20008DBF0E94650C00D000D000D08EE096E0DF
:103E3000EDB7FEB79283818380E090E0A2E0B0E02E
:103E400083839483A583B6830E94597C8DB79EB7E4
:103E500006960FB6F8949EBF0FBE8DBF0E94650CEC
:103E600008952F923F924F925F926F927F928F921E
:103E70009F92AF92BF92CF92DF92EF92FF920F93F9
:103E80001F93DF93CF9300D0CDB7DEB79A8389839A
:103E9000DC018D919C911197009711F00C94513297
:103EA0006091A1047091A20482E590E20E94C37B1C
:103EB00082E590E260E470E00E94E17B009759F4B3
:103EC0006091722D7091732D8AE090E00E941B7CAE
:103ED00081E00C9456328130910549F420905220B3
:103EE000332444245524662477244301BFC18230FF
:103EF000910599F43091522020915320932F80E026
:103F0000820F911D1C01892F880F880B482E582E77
:103F1000682E782E882E982EA9C18330910509F03D
:103F20009CC020915220A09053208090542030E0DB
:103F300040E050E060E070E080E090E000E10E944E
:103F40007D70F22E132FE42ED52EC62EB72E282EDE
:103F5000992E2A2D30E040E050E060E070E080E0F3
:103F600090E008E00E947D702F0DB1E02F1508F061
:103F7000B0E0310FE1E0311708F0E0E0B30FF1E01D
:103F8000B31708F0F0E0EF2B4E0D31E04E1508F0BE
:103F900030E0E40FF1E0E41708F0F0E03F2B5D0DB6
:103FA00041E05D1508F040E0A32FA50F31E0A51713
:103FB00008F030E0432B6C0D31E06C1508F030E078
:103FC000F42FF60F41E0F61708F040E0342B7B0D9C
:103FD00041E07B1508F040E0532F570F31E05717B1
:103FE00008F030E0432B820D31E0821508F030E01C
:103FF000480F61E0481708F060E0362B990D930FE9
:10400000022F080D11E0021708F010E01B0F81E0ED
:104010001B1708F080E0B82FBE0F71E0BE1708F044
:1040200070E07A0F61E07A1708F060E06F0F31E01E
:104030006F1708F030E0350F21E0351708F020E069
:10404000240F81E0241708F080E018014B2E572E32
:10405000662E732E822E982EFEC0843091050CF4AD
:10406000FCC020915220A09053207090542080904A
:10407000552030E040E050E060E070E080E090E00B
:1040800008E10E947D70F22E132FE42ED52EC62E4D
:10409000B72E282E992E2A2D30E040E050E060E027
:1040A00070E080E090E000E10E947D702F0DF1E073
:1040B0002F1508F0F0E0310FE1E0311708F0E0E0F3
:1040C000F30FA1E0F31708F0A0E0EA2B4E0D31E06A
:1040D0004E1508F030E0E40FA1E0E41708F0A0E08E
:1040E0003A2B5D0D41E05D1508F040E0B32FB50FB0
:1040F00031E0B51708F030E0432B6C0D31E06C1562
:1041000008F030E0A42FA60F41E0A61708F040E029
:10411000342B7B0D41E07B1508F040E0532F570F07
:1041200031E0571708F030E0432B820D31E0821563
:1041300008F030E0480F61E0481708F060E0362BE7
:10414000990E930E122F180D81E0121708F080E0DF
:10415000282E2F0E81E02F1608F080E0F82EFE0E9C
:1041600081E0FE1608F080E0E82EEB0E81E0EB1611
:1041700008F080E0D82EDA0E81E0DA1608F080E050
:10418000C82EC50E81E0C51608F080E0B82EB40E2A
:1041900081E0B41608F080E0980E272D30E040E072
:1041A00050E060E070E080E090E008E00E947D7008
:1041B000210FE1E0211708F0E0E0320DF1E03215C7
:1041C00008F0F0E0E30FA1E0E31708F0A0E0FA2B1D
:1041D0004F0D31E04F1508F030E0F40FA1E0F41777
:1041E00008F0A0E03A2B5E0D41E05E1508F040E0DB
:1041F000A32FA50F31E0A51708F030E0432B6D0D7C
:1042000031E06D1508F030E0542F560F41E056179D
:1042100008F040E0342B7C0D41E07C1508F040E0D4
:10422000632F670F31E0671708F030E0432B8B0DE9
:1042300031E08B1508F030E0480F71E0481708F0C6
:1042400070E0372B990D222E3E2E4F2E5A2E652EC2
:10425000762E842E932E990E09C00AE0202E332448
:104260004424552466247724882499240E94650CCC
:10427000B22DB33689F4E32DE23371F4F42DF9361F
:1042800059F4552049F4662039F4772029F4882020
:1042900019F4992009F451C59101A201B301C40197
:1042A00013E6A12EB2E3BB2EA9E6CA2EDD24EE242E
:1042B000FF2400E010E00E94EE70823008F074C22B
:1042C000822D853689F4932D923771F4442061F460
:1042D000552051F4662041F4772031F4882021F4F0
:1042E000992011F40C940F2E9101A201B301C40185
:1042F000F5E6AF2EE2E7BE2ECC24DD24EE24FF242B
:1043000000E010E00E94EE70823008F009C1A22D9A
:10431000A53681F4B32DB43669F4442059F4552000
:1043200049F4662039F4772029F4882019F499207B
:1043300009F4CEC69101A201B301C40105E6A02E85
:1043400014E6B12ECC24DD24EE24FF2400E010E09E
:104350000E94EE70823008F063C0E22DE53781F4F0
:10436000332071F4442061F4552051F4662041F467
:10437000772031F4882021F4992011F40C94CB2972
:104380009101A201B301C401B5E7AB2EBB24CC243B
:10439000DD24EE24FF2400E010E00E94EE70823065
:1043A00010F5F22DF83611F00C944F32332011F045
:1043B0000C944F32442011F00C944F32552011F0E0
:1043C0000C944F32662011F00C944F32772011F08C
:1043D0000C944F32882011F00C944F32992011F038
:1043E0000C944F3293C7822D863779F4332069F4C9
:1043F000442059F4552049F4662039F4772029F4F3
:10440000882019F4992009F4D6C7922D943611F01A
:104410000C944F32A32DA13611F00C944F327BC077
:10442000B22DB73789F4E32DEF3671F4442061F4EF
:10443000552051F4662041F4772031F4882021F48E
:10444000992011F40C94992C9101A201B301C4019B
:10445000A7E7AA2EFFE6BF2ECC24DD24EE24FF24FE
:1044600000E010E00E94EE708230B8F5F22DF436D4
:1044700081F4832D893669F4442059F4552049F498
:10448000662039F4772029F4882019F4992009F45A
:1044900058C7922D953611F00C944F32A32DAE369D
:1044A00011F00C944F32442011F00C944F325520EF
:1044B00011F00C944F32662011F00C944F3277209B
:1044C00011F00C944F32882011F00C944F32992047
:1044D00011F00C944F320C94F32CB22DB13389F4BB
:1044E000E32DE03771F4442061F4552051F4662047
:1044F00041F4772031F4882021F4992011F40C94B0
:10450000842DF22DF33311F00C944F32832D81372B
:1045100011F00C944F32442011F00C944F3295C09E
:10452000922D983789F4A32DA43671F4B42DB136A9
:1045300059F4552049F4662039F4772029F488206D
:1045400019F4992009F4F5C39101A201B301C40142
:10455000E8E7AE2E04E6B02E11E6C12EDD24EE24EF
:10456000FF2400E010E00E94EE70823008F083C06B
:10457000E22DE33789F4F32DF23771F4442061F42E
:10458000552051F4662041F4772031F4882021F43D
:10459000992011F40C94DB2E9101A201B301C40106
:1045A000B3E7AB2EA2E7BA2ECC24DD24EE24FF2401
:1045B00000E010E00E94EE70823020F5822D8936F6
:1045C00011F00C944F32932D923711F00C944F321E
:1045D000442011F00C944F32552011F00C944F32BE
:1045E000662011F00C944F32772011F00C944F326A
:1045F000882011F00C944F32992011F00C944F3216
:104600000C94882EA22DA33789F4B32DB33771F4FF
:10461000442061F4552051F4662041F4772031F4B0
:10462000882021F4992011F40C94EA2EE22DE3362F
:1046300011F00C944F32F32DF43611F00C944F32EC
:10464000842D813611F00C944F32552011F00C94CA
:104650004F32662011F00C944F32772011F00C94F9
:104660004F32882011F00C944F32992011F00C94A5
:104670004F320C94EE30922D923791F4A32DA23745
:1046800079F4B42DB53661F4552051F4662041F427
:10469000772031F4882021F4992011F40C94BC2B5C
:1046A0009101A201B301C401F2E7AF2EE2E7BE2EF1
:1046B00005E6C02EDD24EE24FF2400E010E00E9479
:1046C000EE708230C0F5E22DE33789F4F32DF53634
:1046D00071F4842D813659F4552049F4662039F45B
:1046E000772029F4882019F4992009F474C6922DB2
:1046F000923611F00C944F32A32DA53611F00C9484
:104700004F32B42DB43611F00C944F32552011F0C5
:104710000C944F32662011F00C944F32772011F038
:104720000C944F32882011F00C944F32992011F0E4
:104730000C944F32CDC4E22DE33689F4F32DFD36CF
:1047400071F4842D883659F4552049F4662039F4E3
:10475000772029F4882019F4992009F4F2C2922DC7
:104760009D3611F00C944F32A32DA53711F00C9407
:104770004F32B42DB83611F00C944F32552011F051
:104780000C944F32662011F00C944F32772011F0C8
:104790000C944F32882011F00C944F32992011F074
:1047A0000C944F320C94FD30E22DE03791F4F32D50
:1047B000FC3679F4842D853661F4952D983649F4CC
:1047C000662039F4772029F4882019F4992009F417
:1047D0009DC59101A201B301C40110E7A12EBCE661
:1047E000BB2EA5E6CA2EF8E6DF2EEE24FF2400E05D
:1047F00010E00E94EE70823008F049C1A22DA13372
:1048000091F4B32DB13379F4E42DE13761F45520FF
:1048100051F4662041F4772031F4882021F4992066
:1048200011F40C941F2C9101A201B301C401E1E326
:10483000AE2E01E3B02E11E7C12EDD24EE24FF24BD
:1048400000E010E00E94EE70823008F083C0F22D8C
:10485000F73689F4832D8F3671F4942D9C3659F4F4
:10486000552049F4662039F4772029F4882019F47A
:10487000992009F42EC79101A201B301C401B7E642
:10488000AB2EAFE6BA2EFCE6CF2EDD24EE24FF24BD
:1048900000E010E00E94EE70823020F5A22DA436D8
:1048A00011F00C944F32B32DB33611F00C944F32FB
:1048B000E42DEC3611F00C944F32552011F00C948D
:1048C0004F32662011F00C944F32772011F00C9487
:1048D0004F32882011F00C944F32992011F00C9433
:1048E0004F32F4C6F22DF53789F4832D833671F4F7
:1048F000942D9D3659F4552049F4662039F47720DB
:1049000029F4882019F4992009F499C7A22DA0331D
:1049100011F00C944F32B32DB13311F00C944F328F
:10492000E42DE13711F00C944F32552011F00C9426
:104930004F32662011F00C944F32772011F00C9416
:104940004F32882011F00C944F32992011F00C94C2
:104950004F3212C7F22DF43791F4832D8F3679F44C
:10496000942D9F3661F4A52DA23649F4662039F4C2
:10497000772029F4882019F4992009F485C591013C
:10498000A201B301C401E4E7AE2E0FE6B02E1FE68C
:10499000C12EB2E6DB2EEE24FF2400E010E00E94E0
:1049A000EE708230D0F5B22DB03791F4E32DE536BC
:1049B00079F4F42DF23761F4552051F4662041F476
:1049C000772031F4882021F4992011F40C940F2ED3
:1049D000822D843711F00C944F32932D943611F0C0
:1049E0000C944F32A42DA73711F00C944F32552060
:1049F00011F00C944F32662011F00C944F32772056
:104A000011F00C944F32882011F00C944F32992001
:104A100011F00C944F320C94DE31B22DB93691F472
:104A2000E32DEC3679F4F42DF13661F4852D8336DF
:104A300049F4662039F4772029F4882019F4992064
:104A400009F4ABC1922D963311F00C944F32A32D83
:104A5000A93611F00C944F32B42DB53711F00C94E7
:104A60004F32E52DE53611F00C944F32662011F0EF
:104A70000C944F32772011F00C944F32882011F0B3
:104A80000C944F32992011F00C944F3243C4F22D04
:104A9000F33799F4832D823781F4942D973769F495
:104AA000A52DA03751F4662041F4772031F48820F9
:104AB00021F4992011F40C94D12D9101A201B3019C
:104AC000C401A3E7AA2EF2E7BF2EE7E7CE2E00E748
:104AD000D02EEE24FF2400E010E00E94EE70823021
:104AE00008F089C0B22DB03791F4E32DED3679F49A
:104AF000F42DF53761F4852D883649F4662039F4B4
:104B0000772029F4882019F4992009F438C79101F5
:104B1000A201B301C40110E7A12EBDE6BB2EA5E79B
:104B2000CA2EF8E6DF2EEE24FF2400E010E00E94FB
:104B3000EE70823028F5922D913611F00C944F32A0
:104B4000A32DAD3611F00C944F32B42DB53711F0C2
:104B50000C944F32E52DE83611F00C944F3266205C
:104B600011F00C944F32772011F00C944F328820C2
:104B700011F00C944F32992011F00C944F32EEC684
:104B8000F22DF33799F4832D853681F4942D9237E5
:104B900069F4A52DA03751F4662041F4772031F453
:104BA000882021F4992011F40C944731B22DB133AF
:104BB00011F00C944F32E32DE23711F00C944F3288
:104BC000F42DF73711F00C944F32852D803711F00A
:104BD0000C944F32662011F00C944F32772011F074
:104BE0000C944F32882011F00C944F32992011F020
:104BF0000C944F32AAC0922D973791F4A32DA03771
:104C000079F4B42DB83761F4E52DE43749F4662022
:104C100039F4772029F4882019F4992009F40AC47A
:104C20009101A201B301C401E7E7AE2E00E7B02E67
:104C300018E7C12EB4E7DB2EEE24FF2400E010E0DD
:104C40000E94EE708230D0F5F22DF43791F4832D6E
:104C5000833779F4942D953661F4A52DA23749F464
:104C6000662039F4772029F4882019F4992009F472
:104C700048C7B22DB43711F00C944F32E32DE3370F
:104C800011F00C944F32F42DF53611F00C944F3294
:104C9000852D843711F00C944F32662011F00C945E
:104CA0004F32772011F00C944F32882011F00C9481
:104CB0004F32992011F00C944F32EAC3922D923763
:104CC00091F4A32DA73679F4B42DB03761F4E52D16
:104CD000E53749F4662039F4772029F4882019F45F
:104CE000992009F4C2C4F22DFC3611F00C944F3215
:104CF000832D813611F00C944F32942D943711F09E
:104D00000C944F32A52DA83711F00C944F32662029
:104D100011F00C944F32772011F00C944F32882010
:104D200011F00C944F32992011F00C944F320C94E6
:104D3000A2310E94B3150C9451320E9418100C94A9
:104D400051320E943C160C9451326091A104709132
:104D5000A20480E090E00E94C37B8C016CEF72E0C3
:104D60000E94D87B009719F477980C945132C801AF
:104D70006FEF72E00E94D87B009719F4779A0C9439
:104D80005132779903C08CEF92E002C08FEF92E02E
:104D900000D000D028E535E01FC66091A1047091D5
:104DA000A20480E090E00E94C37B8C0166E173E086
:104DB0000E94D87B009709F052C06091A1047091C5
:104DC000A20480E090E00E94C37B8C01009711F464
:104DD0000C94513269E173E00E94D87B009729F46A
:104DE00082E29FEFACECBBE30BC0C8016FE173E064
:104DF0000E94D87B009789F482E29FEFACECBAE383
:104E00008093940490939504A0939604B093970490
:104E100084E994E066E070E0DEC0C8010E94B67AE2
:104E20007B018C0120E030E0A9010E94A775882356
:104E300091F081E00E94040B9B01AC01C801B70115
:104E40000E94AB75609394047093950480939604CC
:104E500090939704DDCF00D088E995E08CC0C8011D
:104E600064E273E00E94D87B009709F052C0609121
:104E7000A1047091A20480E090E00E94C37B8C01A9
:104E8000009711F40C94513269E173E00E94D87BD1
:104E9000009729F482E29FEFACECBBE30BC0C801A2
:104EA0006FE173E00E94D87B009769F482E29FEF84
:104EB000ACECBAE38093980490939904A0939A047D
:104EC000B0939B041DC0C8010E94B67A7B018C017F
:104ED00020E030E0A9010E94A7758823B1F082E0AC
:104EE0000E94040B9B01AC01C801B7010E94AB7585
:104EF000609398047093990480939A0490939B0410
:104F000088E994E06AE070E066C000D08BE895E044
:104F100069C0C80167E273E00E94D87B009709F07E
:104F20006BC06091A1047091A20480E090E00E94A7
:104F3000C37B8C01009711F40C94513269E173E04A
:104F40000E94D87B009769F487ED94E3AFEEBCE351
:104F50008093900490939104A0939204B09393044F
:104F600036C0C8016FE173E00E94D87B009751F40E
:104F700000D08CE795E0ADB7BEB712969C938E93A8
:104F8000119734C0C8010E94B67A1B012C0120E0A1
:104F900030E0A9010E94A775882309F180E00E94F2
:104FA000040B7B018C01C201B10121EE3AE744E917
:104FB0005EE30E94E074A80197010E94AB756093C4
:104FC000900470939104809392049093930480E9E9
:104FD00094E062E070E044E050E00C94213200D0B4
:104FE0008FE695E0EDB7FEB7928381830E94597CEE
:104FF0000F900F900C9451320E94520B00D000D0B1
:1050000000D028E635E0ADB7BEB712963C932E939C
:105010001197EDB7FEB763837483858396830E94EF
:10502000597C8DB79EB706960FB6F8949EBF0FBEFB
:105030008DBF81E00E94040B20919404309195046F
:1050400040919604509197040E94F1767B018C0167
:1050500082E00E94040B9B01AC01ADB7BEB71A976A
:105060000FB6F894BEBF0FBEADBFCDB6DEB6089486
:10507000C11CD11C8CE595E012969C938E931197E0
:105080008E2D9F2DA02FB12FF60182839383A483B1
:10509000B583CA01B90120919804309199044091D7
:1050A0009A0450919B040E94F176D60116966D9356
:1050B0007D938D939C9319970E94597CEDB7FEB711
:1050C0003A960FB6F894FEBF0FBEEDBF0C94DB31DD
:1050D0006091A1047091A20480E090E00E94C37BE3
:1050E000009761F160E070E040E150E00E94A87933
:1050F0002091CE063091CF062617370799F170938D
:10510000CF066093CE068EEC96E060E070E042E061
:1051100050E00E94A97D8091CE069091CF0600D0EC
:1051200000D028E435E0ADB7BEB712963C932E937D
:10513000119714969C938E9313970EC08091CE0670
:105140009091CF0600D000D024E335E0EDB7FEB754
:1051500032832183948383830E94597C0F900F9024
:105160000F900F900E94650C00D000D087E295E070
:10517000ADB7BEB712969C938E93119781E090E0E5
:1051800014969C938E9313970E94597C8CE195E022
:10519000EDB7FEB79283818382E090E094838383AE
:1051A0000E94597C81E195E0ADB7BEB712969C9301
:1051B0008E93119784E090E014969C938E931397AE
:1051C0000E94597C84E095E0EDB7FEB7928381831D
:1051D00088E090E0948383830E94597C89EF94E077
:1051E000ADB7BEB712969C938E93119780E190E075
:1051F00014969C938E9313970E94597C8DEE94E0A5
:10520000EDB7FEB79283818380E290E0948383833D
:105210000E94597C8FED94E0ADB7BEB712969C9377
:105220008E93119780E490E014969C938E9313973D
:105230000E94597C81ED94E0EDB7FEB792838183A3
:1052400080E890E0948383830E94597C82EC94E010
:10525000ADB7BEB712969C938E93119780E091E004
:1052600014969C938E9313970E94597C83EB94E041
:10527000EDB7FEB79283818380E092E094838383CD
:105280000E94597C87EA94E0ADB7BEB712969C9312
:105290008E93119780E094E014969C938E931397CD
:1052A0000E94597C89E994E0EDB7FEB7928381832F
:1052B00080E098E0948383830E94597C8CE894E09A
:1052C000ADB7BEB712969C938E93119780E090E194
:1052D00014969C938E9313970E94597C8EE794E0CA
:1052E000EDB7FEB79283818380E090E2948383835D
:1052F0000E94597C8EE694E0ADB7BEB712969C939F
:105300008E93119780E090E40C9444320E94C01870
:105310000C94513280915620843329F480E061E06E
:1053200040E00E94581120919C04222311F40C9417
:10533000513200D000D0EDB7FEB731968BE694E045
:1053400020C06091A1047091A20480E090E00E94CE
:10535000C37B69E173E00E94D87B009711F481E080
:1053600001C080E00E94FB1A20919C04222311F4CA
:105370000C94513200D000D0EDB7FEB7319688E6DC
:1053800094E0ADB7BEB712969C938E93119722838B
:1053900013820C9448320E94A91920919C04222364
:1053A00011F40C94513200D000D0EDB7FEB7319615
:1053B00085E694E0E6CF0E94A41920919C04222364
:1053C00011F40C94513200D000D0EDB7FEB73196F5
:1053D00082E694E0D6CF6091A1047091A20480E0AF
:1053E00090E00E94C37B8C016CEF72E00E94D87B3E
:1053F000009739F48091B9049091BA0484600C94B8
:105400001732C8016FEF72E00E94D87B4091B90457
:105410005091BA04009711F44B7FE4C342FF03C0DC
:105420008CEF92E002C08FEF92E000D000D025EA2E
:1054300035E0D2C26091A1047091A20480E090E0B6
:105440000E94C37B0E94BA7A803168F48093D306AD
:1054500090E00E94895583ED96E066E170E041E0BE
:1054600050E00C94213200D000D0EDB7FEB7319659
:1054700089EA95E0ADB7BEB712969C938E931197CB
:105480008091D306828384CF0C9400000C94513217
:105490006091A1047091A20480E090E00E94C37B1F
:1054A0008C016CE273E00E94D87B009739F4219A5A
:1054B0008091B9049091BA048061B9C7C8016EE2C5
:1054C00073E00E94D87B009739F4229A8091B90446
:1054D0009091BA048062ABC7C80160E373E00E9498
:1054E000D87B009739F4239A8091B9049091BA043B
:1054F00080649DC7C80162E373E00E94D87B009777
:1055000039F4239A8091B9049091BA0480688FC7C6
:10551000C80164E373E00E94D87B0097C9F48091CE
:10552000B9049091BA0491609093BA048093B9043D
:1055300089EB94E064E170E042E050E00E94A97DD4
:105540008BEF94E062E140E050E00E94213FA9C768
:10555000C8016FEF72E00E94D87B4091B90450916E
:10556000BA04009741F44F705E7F5093BA044093A1
:10557000B9042B9A60C744FF03C08CEF92E002C0CD
:105580008FEF92E000D000D022EE35E0EDB7FEB70D
:1055900032832183948383830E94597C8091B90450
:1055A0000F900F900F900F9085FF03C08CEF92E04B
:1055B00002C08FEF92E000D000D027ED35E0ADB70C
:1055C000BEB712963C932E93119714969C938E938C
:1055D00013970E94597C8091B9040F900F900F90FF
:1055E0000F9086FF03C08CEF92E002C08FEF92E035
:1055F00000D000D02CEC35E0EDB7FEB7328321832C
:10560000948383830E94597C8091B9040F900F90FA
:105610000F900F9087FF03C08CEF92E002C08FEFD6
:1056200092E000D000D021EC35E0ADB7BEB71296C5
:105630003C932E93119714969C938E9313970E94EC
:10564000597C8091B9049091BA040F900F900F90FB
:105650000F9090FF03C08CEF92E002C08FEF92E0BA
:1056600000D000D026EB35E0B7C100D08EE594E045
:10567000ADB7BEB712969C938E9311970E94597C3A
:1056800020919C040F900F902223A9F000D000D00D
:10569000EDB7FEB731968BE594E0ADB7BEB7129685
:1056A0009C938E931197228313820E94597C0F90B2
:1056B0000F900F900F9088E10FB6F89480936000E0
:1056C000109260000FBE0C94007CEBC60E94334C1D
:1056D000E8C66091A1047091A20480E090E00E946D
:1056E000C37B1C016CEF72E00E94D87B009749F4E9
:1056F0000E94E0528091B9049091BA0481608D7F3C
:1057000096C6C1016FEF72E00E94D87B009741F40A
:105710000E9442528091B9049091BA048C7F87C64E
:1057200006E313E0C101B8010E94D87B009749F459
:105730000E9442528091B9049091BA048E7F826097
:1057400076C68091B90481FF0BC000D000D081EFF4
:1057500095E0EDB7FEB7928381831483038398C6E7
:1057600080FF03C08CEF92E002C08FEF92E000D088
:1057700000D02DEE35E082C600D081E394E0EDB795
:10578000FEB7928381830E94597C8DB79EB7409764
:105790000FB6F8949EBF0FBE8DBFEDB7FEB7319622
:1057A00083E194E0ADB7BEB712969C938E931197A8
:1057B00080914D2090914E20A0914F20B09150208B
:1057C00082839383A483B58380914120909142206A
:1057D000A0914320B091442086839783A087B1870E
:1057E0008091452090914620A0914720B09148207B
:1057F00082879387A487B5878091492090914A201A
:10580000A0914B20B0914C2086879787A08BB18BBD
:105810000E94597C20919C04EDB7FEB772960FB69A
:10582000F894FEBF0FBEEDBF222309F43AC600D0A4
:1058300000D0EDB7FEB7319680E194E0A2CDF894A8
:1058400081E090E00E948308182F80E090E00E94A1
:105850008308082F7894F89483E090E00E948308EE
:10586000F82E82E090E00E948308E82E789400D021
:1058700000D000D026E034E0EDB7FEB732832183BC
:105880002091EE173091EF174091F0175091F117DA
:10589000ADB7BEB713962D933D934D935C9316977A
:1058A0000E94597C00D000D0EDB7FEB731962FEDA5
:1058B00033E0ADB7BEB712963C932E931197E282B8
:1058C0001382F482158206831782108711860E9444
:1058D000597CEDB7FEB73A960FB6F894FEBF0FBEEF
:1058E000EDBF0E944C1A2091660000D000D0EDB7A9
:1058F000FEB7319683ED93E0ADB7BEB712969C9399
:105900008E931197228313820E94597C0F900F90DF
:105910000F900F900E94650C20919C04222309F4A3
:10592000C0C500D000D0EDB7FEB7319680ED93E052
:1059300028CD80E090E00E94710C81E090E00E9410
:10594000710C20919C04222309F4ABC500D000D037
:10595000EDB7FEB731968DEC93E013CD0E942F1872
:105960000E94650C20919C04222309F49AC500D062
:1059700000D0EDB7FEB731968AEC93E002CD60918E
:10598000A1047091A20480E090E00E94C37B8C018E
:105990006CEF72E00E94D87B009731F48091B904DB
:1059A0009091BA04886043C5C8016FEF72E00E940D
:1059B000D87B4091B9045091BA04009711F4477F05
:1059C00011C143FF03C08CEF92E002C08FEF92E061
:1059D00000D000D025EF35E0EDB7FEB7328321834C
:1059E0009483838355C56091A1047091A20480E0E3
:1059F00090E00E94C37B6BE373E00E94D87B00972A
:105A000041F5F89483EF96E00E9418400CC0C8015D
:105A10000D960E94644388E495E0B8010E94D23F4D
:105A2000C8010E94DE40082F192F0115110579F7D2
:105A300004C083EF96E00E94594083EF96E00E94F5
:105A4000BE400097B1F783EF96E00E94144078942F
:105A50004BC083EF96E00E941840482F592F7A01DF
:105A600001E413E03DC08DB79EB70C970FB6F894D4
:105A70009EBF0FBE8DBFEDB7FEB73196ADB7BEB7B7
:105A800012961C930E931197D70112968C91129730
:105A90008283138213968C911397848315821896B0
:105AA0008C9118978683178214968D919C911597E7
:105AB0009187808716968D919C91179793878287FF
:105AC0000E94477CEDB7FEB73C960FB6F894FEBF38
:105AD0000FBEEDBFC7010E94DE40482F592F7A014B
:105AE000E114F10409F0BFCF20919C04222309F4B2
:105AF000D8C400D000D0EDB7FEB7319687EC93E064
:105B000040CC0E94351BCDC46091A1047091A204C9
:105B100080E090E00E94C37B8C016CEF72E00E94F9
:105B2000D87B009751F48091B9049091BA049460A5
:105B30009093BA048093B90410C0C8016FEF72E06B
:105B40000E94D87B4091B9045091BA04009771F437
:105B50005B7F5093BA044093B90489EB94E064E10D
:105B600070E042E050E00E94A97D17C052FF03C0E0
:105B70008CEF92E002C08FEF92E000D000D029EFCE
:105B800035E0EDB7FEB732832183948383830E948F
:105B9000597C0F900F900F900F9081E00E94740A33
:105BA00080C46091A1047091A20480E090E00E9402
:105BB000C37B8C016EE073E00E94D87B009731F4C8
:105BC0008091B9049091BA049D7F31C4C80163E00B
:105BD00073E00E94D87B4091B9045091BA040097B9
:105BE00031F452605093BA044093B90424C451FF75
:105BF00003C083E093E002C08EE093E000D000D0C9
:105C000028E633E0ADB7BEB712963C932E931197BA
:105C100014969C938E9313970E94477C3BC460918B
:105C2000A1047091A20480E090E00E94C37B0097E1
:105C3000A9F160E070E040E150E00E94A879609333
:105C4000B3047093B4048093B5049093B60400D069
:105C500000D000D024EB33E0EDB7FEB732832183D0
:105C6000ADB7BEB713966D937D938D939C931697A6
:105C70000E94597CEDB7FEB736960FB6F894FEBF7A
:105C80000FBEEDBF83EB94E06EE070E044E050E0C7
:105C90000E94A97D81E00E94D81B03C480E00E947D
:105CA000D81B0E94650C00D000D000D08FE993E093
:105CB000ADB7BEB712969C938E9311978091B304A3
:105CC0009091B404A091B504B091B604EDB7FEB7BD
:105CD00083839483A583B6830E94597C8DB79EB736
:105CE00006960FB6F8949EBF0FBE8DBF81E00E944E
:105CF000D81B0E94650C20919C04222309F4D1C377
:105D000000D000D0EDB7FEB731968CE993E039CBE7
:105D10006091A1047091A20480E090E00E94C37B96
:105D2000009741F160E070E04AE050E00E94A879FD
:105D30007093B8046093B70400D000D0EDB7FEB7FD
:105D400031962FE733E0ADB7BEB712963C932E9352
:105D50001197738362830E94597C0F900F900F906C
:105D60000F9087EB94E062E170E042E050E00E9427
:105D7000A97D14C000D000D08EE593E0EDB7FEB74A
:105D8000928381838091B7049091B8049483838334
:105D90000E94597C0F900F900F900F9020919C04BF
:105DA000222309F47EC300D000D0EDB7FEB73196B0
:105DB0008BE593E0E6CA0E94A14320919C04222334
:105DC00009F46FC300D000D0EDB7FEB7319688E577
:105DD00093E0D7CA00D088E493E0EDB7FEB7928392
:105DE00081830E94597C0F900F900E94A41900D0CB
:105DF00084E493E0ADB7BEB712969C938E9311974F
:105E00000E94597C0F900F9080E00E94FB1A00D0F6
:105E10008EE393E0EDB7FEB7928381830E94597CB5
:105E20000F900F900E94181080913B1C80FF05C0BE
:105E300081E061E041E00E9458110E94A91900D060
:105E400000D0EDB7FEB7319681E393E0ADB7BEB7B2
:105E500012969C938E9311978091D306828313821E
:105E60000E94597C89E193E0EDB7FEB7928381836C
:105E700080E490E0948383830E94597C00D0EDB746
:105E8000FEB7319686E093E0ADB7BEB712969C930D
:105E90008E9311978091B724828313828091B824C6
:105EA000848315820E94597C0F900F9081EF92E0BD
:105EB000EDB7FEB7928381838091B7049091B804C7
:105EC000948383830E94597C00D08DED92E0ADB71E
:105ED000BEB712969C938E9311978091B3049091C4
:105EE000B404A091B504B091B604EDB7FEB78383B6
:105EF0009483A583B6830E94597C8DB79EB706967E
:105F00000FB6F8949EBF0FBE8DBF81E00E94D81BD4
:105F10000E94520B00D000D000D020ED32E0ADB78F
:105F2000BEB712963C932E931197EDB7FEB76383DD
:105F30007483858396830E94597C8DB79EB706969D
:105F40000FB6F8949EBF0FBE8DBF0E94890B0E94B2
:105F5000660B00D000D000D022EC32E0ADB7BEB767
:105F600012963C932E931197EDB7FEB7638374831B
:105F7000858396830E94597C8DB79EB706960FB68F
:105F8000F8949EBF0FBE8DBF1D9B03C083E193E0BD
:105F900002C08FEF92E000D000D026EB32E0ADB728
:105FA000BEB712963C932E93119714969C938E93A2
:105FB00013970E94597C2091922430919324409110
:105FC0009424509195248091962490919724A091A7
:105FD0009824B091992400D000D000D00DB71EB7FE
:105FE0000F5F1F4F68E972E0EDB7FEB77283618300
:105FF000F801228333834483558386839783A08764
:10600000B1870E94597CEDB7FEB7319686E792E0E2
:10601000ADB7BEB712969C938E93119780919F2433
:106020009091A024A091A124B091A2248283938373
:10603000A483B5838091A3249091A424A091A52446
:10604000B091A62486839783A087B1870E94597C4C
:10605000EDB7FEB738960FB6F894FEBF0FBEEDBF92
:106060008CE692E0928381830E94597C8091B904EE
:106070000F900F9081FF0EC000D086E692E0ADB782
:10608000BEB712969C938E9311970E94597C0F90E5
:106090000F9017C080FF03C08CEF92E002C08FEF1B
:1060A00092E000D000D022E632E0EDB7FEB73283B6
:1060B0002183948383830E94597C0F900F900F90CB
:1060C0000F908091B90483FF03C08CEF92E002C06F
:1060D0008FEF92E000D000D02FE432E0ADB7BEB732
:1060E00012963C932E93119714969C938E9313972C
:1060F0000E94597C8091B9049091BA040F900F903E
:106100000F900F9092FF03C08CEF92E002C08FEFD0
:1061100092E000D000D022E432E0EDB7FEB7328347
:106120002183948383830E94597C8091CE06909131
:10613000CF0625E332E0ADB7BEB712963C932E935F
:10614000119714969C938E9313970E94597C0F90ED
:106150000F900F900F90779903C08CEF92E002C0E0
:106160008FEF92E000D000D02CE232E0EDB7FEB726
:1061700032832183948383830E94597C8091B90464
:106180009091BA040F900F900F900F9091FF03C061
:1061900083E093E002C08EE093E000D000D028E6D8
:1061A00033E0ADB7BEB712963C932E931197149679
:1061B0009C938E9313970E94477C20919C040F9090
:1061C0000F900F900F90222309F46BC100D000D0E4
:1061D000EDB7FEB7319689E292E0D3C80E94711AFA
:1061E00020919C04222309F45CC100D000D0EDB7BB
:1061F000FEB7319686E292E0C4C80E9475170097F8
:10620000B9F500D000D000D08BE192E0EDB7FEB739
:10621000928381838091371890913818A091391812
:10622000B0913A1883839483A583B6830E94597CE6
:106230008EE092E0ADB7BEB712969C938E93119705
:106240008091B3249091B424A091B524B091B62448
:10625000EDB7FEB783839483A583B6830E94597CF0
:106260008DB79EB706960FB6F8949EBF0FBE8DBF32
:106270000E94650C20919C04222309F412C100D0D5
:1062800000D0EDB7FEB731968BE092E07AC883E09C
:1062900061E048E021E00E94F21200D000D000D07E
:1062A00084E092E0EDB7FEB79283818380912A1853
:1062B00090912B18A0912C18B0912D188383948362
:1062C000A583B6830E94597C00D000D0EDB7FEB7FD
:1062D000319683EF91E0ADB7BEB712969C938E9343
:1062E000119780912E1890912F18A0913018B0918D
:1062F000311882839383A483B5838091321890915F
:106300003318A0913418B091351886839783A087ED
:10631000B1870E94597CEDB7FEB73A960FB6F89454
:10632000FEBF0FBEEDBF0E94650C20919C0422238E
:1063300009F4B7C000D000D0EDB7FEB7319680EFBA
:1063400091E01FC86091A1047091A20480E090E0E8
:106350000E94C37B61E773E00E94D87B0097B1F491
:106360006091A1047091A20480E090E00E94C37B40
:10637000009709F496C00E94BA7A803108F091C063
:1063800090915201982B909352018BC080915201B1
:1063900000D000D02DEF35E0EDB7FEB7328321837A
:1063A00090E08F709070948383830E94597C0F904B
:1063B0000F900F900F900E94650C73C06091A10424
:1063C0007091A20480E090E00E94C37B8C016CEF8E
:1063D00072E00E94D87B009741F40E942451809182
:1063E000B9049091BA04986022C0C8016FEF72E0BE
:1063F0000E94D87B009741F5F8940E94325188E1C1
:106400000FB6F89480936000109260000FBE84B7BE
:10641000877F84BF809160008861809360001092C4
:10642000600078948091B9049091BA04977F90931A
:10643000BA048093B90489EB94E064E170E042E02F
:1064400050E00E94A97D2DC0C80166E773E00E945C
:10645000D87B4091B9045091BA04009721F453FFBE
:1064600020C0F894FFCF53FF03C08CEF92E002C02E
:106470008FEF92E000D000D02AE036E0ADB7BEB793
:1064800012963C932E93119714969C938E93139788
:106490000E94597C0F900F900F900F9002C00E94A5
:1064A0009918E981FA811182108283E00F900F9090
:1064B000CF91DF911F910F91FF90EF90DF90CF90E0
:1064C000BF90AF909F908F907F906F905F904F9014
:1064D0003F902F900895F89491E2E0E0F0E09093DF
:1064E00057008491E2E0F0E0909357002491E4E0BB
:1064F000F0E090935700E49190E0A0E0B0E0DC0180
:106500009927882730E040E050E0542F432F322F66
:106510002227820F931FA41FB51F8E0F911DA11D4F
:10652000B11D8093EE179093EF17A093F017B093DF
:10653000F11778940895DF93CF93CDB7DEB72797FF
:106540000FB6F894DEBF0FBECDBFCE0104966EE04D
:1065500070E044E050E00E948B7D8C819D81AE8193
:10656000BF818F3F2FEF92072FEFA2072FEFB207C8
:1065700049F483EB94E06EE070E044E050E00E9468
:10658000A97D08C08093B3049093B404A093B5048C
:10659000B093B604CE01029662E170E042E050E0B2
:1065A0000E948B7D8A819B812FEF8F3F920779F428
:1065B0008CE390E09093B8048093B70487EB94E069
:1065C00062E170E042E050E00E94A97D04C0909337
:1065D000B8048093B704CE01029664E170E042E013
:1065E00050E00E948B7D8A819B812FEF8F3F920725
:1065F00079F48AE090E09093BA048093B90489EB2F
:1066000094E064E170E042E050E00E94A97D04C0A3
:106610009093BA048093B904CE01029660E070E0D2
:1066200042E050E00E948B7D8A819B812FEF8F3F5B
:10663000920769F41092CF061092CE068EEC96E087
:1066400060E070E042E050E00E94A97D04C09093B9
:10665000CF068093CE0687EA94E267E170E049E0D6
:1066600050E00E948B7D0E94D40DCE01049666E01E
:1066700070E044E050E00E948B7D8C819D81AE8172
:10668000BF818F3F2FEF92072FEFA2072FEFB207A7
:1066900049F484E994E066E070E044E050E00E9450
:1066A000A97D08C084E994E066E070E044E050E031
:1066B0000E948B7DCE0104966AE070E044E050E0D9
:1066C0000E948B7D8C819D81AE81BF818F3F2FEF9A
:1066D00092072FEFA2072FEFB20749F488E994E061
:1066E0006AE070E044E050E00E94A97D08C088E9BB
:1066F00094E06AE070E044E050E00E948B7DCE01BF
:10670000049662E070E044E050E00E948B7D8C8152
:106710009D81AE81BF818F3F2FEF92072FEFA207A0
:106720002FEFB20749F480E994E062E070E044E0C2
:1067300050E00E94A97D08C080E994E062E070E02A
:1067400044E050E00E948B7DCE01019666E170E04E
:1067500041E050E00E948B7D89818F3F49F483EDB9
:1067600096E066E170E041E050E00E94A97D08C03B
:1067700083ED96E066E170E041E050E00E948B7DA1
:1067800027960FB6F894DEBF0FBECDBFCF91DF9135
:1067900008950E9418516C9A6B9A6A9A6F9A729A2D
:1067A000749A739A779A809880B3897F80BB839814
:1067B000849887E080937E00549A0E946B320E94F6
:1067C0009B3281E00E94740A80E090E00E94E80D14
:1067D0000E94A14A8091B90486FD239A0895CF931F
:1067E000DF93EC0188819981009731F02AE08033B2
:1067F000920709F08CC082C00E94C9338091B9040D
:1068000080FD06C081FF02C01D9902C00E94425255
:10681000809170008C7F809370008091B6008062C0
:106820008093B6001092B20082E08093B100809114
:10683000B60090E0877090700097C9F78091700063
:1068400081608093700080E090E06AE878E00E94C8
:10685000FB500E94A41980E00E94FB1A00D08AEE2F
:1068600091E0ADB7BEB712969C938E9311970E949C
:10687000597C0F900F900E94181080913B1C86FF4E
:1068800002C00E94DE4B80E090E00E9489550E9489
:10689000FE538093010700D000D000D0EDB7FEB7C3
:1068A00031962BE733E0ADB7BEB712963C932E93EB
:1068B0001197828313828091D306848315820E946C
:1068C000477C109200071092FF06EDB7FEB7369690
:1068D0000FB6F894FEBF0FBEEDBF87EC94E0909327
:1068E000B1248093B02483E290E09093F8068093E3
:1068F000F70680E39AE0998388830DC0633259F4E8
:106900008FEF96E060E070E00E94311FE6CF1982C1
:10691000188283E001C081E0DF91CF910895853630
:10692000910564F12091CE063091CF0620FF10C072
:1069300000D000D02DE833E0EDB7FEB732832183DD
:10694000948383830E94477C0F900F900F900F9049
:1069500080914D2090914E20A0914F20B0915020D9
:106960000196A11DB11D80934D2090934E20A093C0
:106970004F20B093502021E030E002C020E030E012
:10698000C90108954F925F926F927F928F929F926A
:10699000AF92BF92CF92DF92EF92FF920F931F932D
:1069A000DF93CF93CDB7DEB7CB58D0400FB6F89476
:1069B000DEBF0FBECDBF2C01633871F48FED96E0C2
:1069C000C557DF4F6883CB58D0400E94583DC5570C
:1069D000DF4F6881CB58D040D2018D919C911197A7
:1069E000B9E0863E9B0709F48FC7E9E0873E9E0722
:1069F00040F4009789F0F8E0803F9F0709F0C5C791
:106A000016C029E0873F920709F499C739E08E3F05
:106A1000930709F0BAC7ABC78FED96E061E870E065
:106A200044E455E00E943D3D80EF98E068C7623144
:106A300009F0B1C78091B3049091B404A091B5045A
:106A4000B091B60497FD8C9A0E94890B8091B30493
:106A50009091B404A091B504B091B60493FF02C024
:106A60000E9475178091B3049091B404A091B5046D
:106A7000B091B60494FF0AC00E94520B60939A240E
:106A800070939B2480939C2490939D248091B304C5
:106A900080FF5DC042E1C42ED12CCC0EDD1E00D0A3
:106AA00000D000D0EDB7FEB73196ADB7BEB71296A5
:106AB000DC92CE92119788E790E09383828381EAFB
:106AC00093E0958384830E94B77C082F192F37EABF
:106AD000E32E34E2F32EEDB7FEB736960FB6F894F8
:106AE000FEBF0FBEEDBF28E7A22EB12C9FE8892E76
:106AF00092E0992ED7012D917D01EDB7FEB7389721
:106B00000FB6F894FEBF0FBEEDBF3196C601800FE1
:106B1000911FADB7BEB712969C938E931197B38217
:106B2000A28295828482268317820E94B77C080FF6
:106B3000191FEDB7FEB738960FB6F894FEBF0FBE1B
:106B4000EDBFFFEAEF16F4E2FF06A1F602C000E097
:106B500010E08091B30481FF6EC082E1C82ED12C79
:106B6000CC0EDD1E00D000D000D0EDB7FEB73196C0
:106B7000C601800F911FADB7BEB712969C938E933E
:106B8000119788E790E09383828385EA93E0958369
:106B900084830E94B77C080F191F7E010894E11CB2
:106BA000F11C80E1F70111928A95E9F72DB73EB704
:106BB0002A5F3F4F0FB6F8943EBF0FBE2DBF80EB4C
:106BC00068E9A70128E00E941011B8E0AB2EB12CB3
:106BD000AC0EBD1EA8E78A2E912CFFE86F2EF2E0C6
:106BE0007F2ED7012D917D01EDB7FEB738970FB6F7
:106BF000F894FEBF0FBEEDBF3196C601800F911F06
:106C0000ADB7BEB712969C938E93119793828282F2
:106C100075826482268317820E94B77C080F191F31
:106C2000EDB7FEB738960FB6F894FEBF0FBEEDBFB6
:106C3000EA14FB04B1F68091B3049091B404A091DE
:106C4000B504B091B6040097A105B10581F12DB747
:106C50003EB7285030400FB6F8943EBF0FBE2DBF50
:106C6000EDB7FEB73196CE014296800F911FADB7BA
:106C7000BEB712969C938E93119788E790E093830A
:106C800082838AEA93E0958384838091D1069091F0
:106C9000D206978386830E94B77C080F191FEDB731
:106CA000FEB738960FB6F894FEBF0FBEEDBF8091C9
:106CB000B30482FF50C089E290E06BE270E04AE2E8
:106CC00050E027E00E94B74787EA94E20E94274AF3
:106CD0002DB73EB72A5030400FB6F8943EBF0FBED6
:106CE0002DBFEDB6FEB60894E11CF11C9E012E5E90
:106CF0003F4F200F311FADB7BEB712963C932E9376
:106D0000119728E730E0F7013383228321EB33E04A
:106D1000358324839C01B901882777FD8095982FBE
:106D20000E94157620E030E048EC52E40E94AB75FA
:106D3000D70116966D937D938D939C9319970E941E
:106D4000B77C080F191FEDB7FEB73A960FB6F89447
:106D5000FEBF0FBEEDBF8091B30483FF56C089E232
:106D600090E06BE270E04AE250E026E00E94B74714
:106D700081E090E00E94D90B8093D50686EA97E1E6
:106D80000E94274A2DB73EB72A5030400FB6F894DC
:106D90003EBF0FBE2DBFEDB6FEB60894E11CF11C40
:106DA0009E012E5E3F4F200F311FADB7BEB712962A
:106DB0003C932E93119728E730E0F7013383228329
:106DC0002BEB33E0358324839C01B901882777FDC1
:106DD0008095982F0E94157620E030E048EC52E430
:106DE0000E94AB75D70116966D937D938D939C93FE
:106DF00019970E94B77C080F191FEDB7FEB73A9696
:106E00000FB6F894FEBF0FBEEDBF8091B30484FFB0
:106E100036C02DB73EB72A5030400FB6F8943EBF6B
:106E20000FBE2DBFEDB7FEB73196CE014296800F53
:106E3000911FADB7BEB712969C938E93119788E7BA
:106E400090E09383828386EC93E0958384838091A2
:106E5000921790919317A0919417B09195178683EC
:106E60009783A087B1870E94B77C080F191FEDB7E1
:106E7000FEB73A960FB6F894FEBF0FBEEDBF8091F5
:106E8000B30485FF31C00E94660B2DB73EB72A5070
:106E900030400FB6F8943EBF0FBE2DBFEDB7FEB722
:106EA00031969E012E5E3F4F200F311FADB7BEB70A
:106EB00012963C932E93119728E730E03383228378
:106EC00024ED33E03583248366837783808791873D
:106ED0000E94B77C080F191FEDB7FEB73A960FB6A0
:106EE000F894FEBF0FBEEDBF8091B30486FF3AC099
:106EF000F8948091922490919324A0919424B0913D
:106F0000952478942DB73EB72A5030400FB6F894A8
:106F10003EBF0FBE2DBF4DB75EB74F5F5F4F9E01A7
:106F20002E5E3F4F200F311FEDB7FEB73283218316
:106F300028E730E0FA013383228322EE33E0358301
:106F4000248386839783A087B1870E94B77C080F2C
:106F5000191F2DB73EB7265F3F4F0FB6F8943EBFBF
:106F60000FBE2DBF8091B30487FF92C08091B704FC
:106F70009091B804009709F48BC0F894C0909224C3
:106F8000D0909324E0909424F0909524789480916C
:106F90009E1790919F17A091A017B091A117A701DC
:106FA0009601281B390B4A0B5B0BCA01B9010E94E1
:106FB0001376862EA72E682EB92E6091B704709195
:106FC000B80480E090E00E9413769B01AC01682D2C
:106FD0007A2D862D9B2D0E94AB755C014DB75EB757
:106FE0004A5050400FB6F8945EBF0FBE4DBFEDB78C
:106FF000FEB73196CE014296800F911FADB7BEB756
:1070000012969C938E93119788E790E093838283E6
:107010008BEE93E095838483262F372F4A2D5B2DAB
:107020002683378340875187C557DF4F6883CB5806
:10703000D040C657DF4F7883CA58D0400E94B77CF3
:10704000080F191FC557DF4F6881CB58D040C6576E
:10705000DF4F7881CA58D040862F972FAA2DBB2D9D
:1070600080939F249093A024A093A124B093A22462
:10707000C0929E17D0929F17E092A017F092A1178E
:10708000EDB7FEB73A960FB6F894FEBF0FBEEDBF50
:107090008091B3049091B404A091B504B091B6046A
:1070A00090FF40C0F8948091962490919724A091ED
:1070B0009824B091992478942DB73EB72A50304047
:1070C0000FB6F8943EBF0FBE2DBF4DB75EB74F5FF2
:1070D0005F4F9E012E5E3F4F200F311FEDB7FEB771
:1070E0003283218328E730E0FA013383228328EFBB
:1070F00033E03583248386839783A087B1870E94FA
:10710000B77C080F191F2DB73EB7265F3F4F0FB64C
:10711000F8943EBF0FBE2DBFC8010E948F34009768
:1071200009F082CC8091B3049091B404A091B5048D
:10713000B091B60491FF92C08091B7049091B804C9
:10714000009709F48BC0F894C0909624D0909724AF
:10715000E0909824F090992478948091A2179091CF
:10716000A317A091A417B091A517A7019601281BFA
:10717000390B4A0B5B0BCA01B9010E941376862EAC
:10718000A72E682EB92E6091B7047091B80480E0E4
:1071900090E00E9413769B01AC01682D7A2D862D1C
:1071A0009B2D0E94AB755C014DB75EB74A505040B5
:1071B0000FB6F8945EBF0FBE4DBFEDB7FEB7319668
:1071C000CE014296800F911FADB7BEB712969C9329
:1071D0008E93119788E790E09383828381E094E017
:1071E00095838483262F372F4A2D5B2D2683378363
:1071F00040875187C557DF4F6883CB58D040C6576B
:10720000DF4F7883CA58D0400E94B77C080F191FFF
:10721000C557DF4F6881CB58D040C657DF4F7881C4
:10722000CA58D040862F972FAA2DBB2D8093A32418
:107230009093A424A093A524B093A624C092A2174F
:10724000D092A317E092A417F092A517EDB7FEB75E
:107250003A960FB6F894FEBF0FBEEDBF8091B3040F
:107260009091B404A091B504B091B60492FF3EC0D1
:1072700080913D2090913E20A0913F20B0914020F0
:107280002DB73EB72A5030400FB6F8943EBF0FBE20
:107290002DBF4DB75EB74F5F5F4F9E012E5E3F4FD4
:1072A000200F311FEDB7FEB73283218328E730E08E
:1072B000FA01338322832EE034E0358324838683EE
:1072C0009783A087B1870E94B77C080F191F2DB73D
:1072D0003EB7265F3F4F0FB6F8943EBF0FBE2DBF9F
:1072E000C8010E948F34009709F09ECB8091B304AF
:1072F0009091B404A091B504B091B60493FF3CC042
:107300004DB75EB74A5050400FB6F8945EBF0FBEFF
:107310004DBFEDB7FEB73196CE014296800F911F5B
:10732000ADB7BEB712969C938E93119788E790E005
:107330009383828387E194E09583848380913718D7
:1073400090913818A0913918B0913A188683978394
:10735000A087B1870E94B77C080F191FEDB7FEB751
:107360003A960FB6F894FEBF0FBEEDBFC8010E945B
:107370008F34009709F058CB8091B3049091B404F6
:10738000A091B504B091B60494FF3CC02DB73EB7B0
:107390002A5030400FB6F8943EBF0FBE2DBFEDB758
:1073A000FEB73196CE014296800F911FADB7BEB7A2
:1073B00012969C938E93119788E790E09383828333
:1073C00082E294E09583848380919A2490919B2417
:1073D000A0919C24B0919D2486839783A087B18738
:1073E0000E94B77C080F191FEDB7FEB73A960FB68B
:1073F000F894FEBF0FBEEDBFC8010E948F34009706
:1074000009F012CB8091B3049091B404A091B5041B
:10741000B091B60495FF48C081E00E94040B2DB7DF
:107420003EB72A5030400FB6F8943EBF0FBE2DBF76
:10743000EDB6FEB60894E11CF11C9E012E5E3F4F96
:10744000200F311FADB7BEB712963C932E93119704
:1074500028E730E0F701338322832FE234E03583DD
:107460002483209194043091950440919604509186
:1074700097040E94F176D70116966D937D938D93B4
:107480009C9319970E94B77C080F191FEDB7FEB7A0
:107490003A960FB6F894FEBF0FBEEDBFC8010E942A
:1074A0008F34009709F0C0CA8091B3049091B4045E
:1074B000A091B504B091B60496FF48C082E00E9446
:1074C000040B2DB73EB72A5030400FB6F8943EBF9C
:1074D0000FBE2DBFEDB6FEB60894E11CF11C9E0157
:1074E0002E5E3F4F200F311FADB7BEB712963C93B3
:1074F0002E93119728E730E0F701338322832CE3A2
:1075000034E035832483209198043091990440918C
:107510009A0450919B040E94F176D70116966D93C0
:107520007D938D939C9319970E94B77C080F191F28
:10753000EDB7FEB73A960FB6F894FEBF0FBEEDBF9B
:10754000C8010E948F34009709F06ECA8091B3047D
:107550009091B404A091B504B091B60497FF39C0DE
:1075600083E00E94040B2DB73EB72A5030400FB67F
:10757000F8943EBF0FBE2DBFEDB7FEB731969E010A
:107580002E5E3F4F200F311FADB7BEB712963C9312
:107590002E93119728E730E03383228329E434E0E7
:1075A0003583248366837783808791870E94B77CA5
:1075B000080F191F8C98EDB7FEB73A960FB6F894DE
:1075C000FEBF0FBEEDBFC8010E948F34009709F0C7
:1075D0002BCA8091B3049091B404A091B504B091EA
:1075E000B604A0FF06C083E061E046E020E00E9410
:1075F000F2128091B3049091B404A091B504B091BB
:10760000B604A1FF06C083E061E046E021E00E94ED
:10761000F2128091B3049091B404A091B504B0919A
:10762000B604A0FF3CC02DB73EB72A5030400FB67D
:10763000F8943EBF0FBE2DBFEDB7FEB73196CE0119
:107640004296800F911FADB7BEB712969C938E9352
:10765000119788E790E09383828386E594E0958391
:10766000848380912E1890912F18A0913018B0919A
:10767000311886839783A087B1870E94B77C080F53
:10768000191FEDB7FEB73A960FB6F894FEBF0FBEBE
:10769000EDBFC8010E948F34009709F0C5C98091E1
:1076A000B3049091B404A091B504B091B604A1FFC5
:1076B0003CC02DB73EB72A5030400FB6F8943EBFBD
:1076C0000FBE2DBFEDB7FEB73196CE014296800FAB
:1076D000911FADB7BEB712969C938E93119788E712
:1076E00090E0938382838EE594E0958384838091F8
:1076F000321890913318A0913418B09135188683C0
:107700009783A087B1870E94B77C080F191FEDB738
:10771000FEB73A960FB6F894FEBF0FBEEDBFC80194
:107720000E948F34009709F07FC9779A8091CE0626
:107730009091CF0693FD749A8091CE069091CF06DA
:1077400082FD08C08091B90480FD04C081FF31C072
:107750001D9B2FC000D000D089E694E0ADB7BEB726
:1077600012969C938E931197CE01429614969C93F9
:107770008E9313970E94477C20919C040F900F904A
:107780000F900F902223A9F000D000D0EDB7FEB7E4
:10779000319684EE91E0ADB7BEB712969C938E936E
:1077A0001197228313820E94597C0F900F900F90A3
:1077B0000F908091F206898BFE01E00FF11F128A73
:1077C00068010894C11CD11C8091CE069091CF060F
:1077D00080FF12C000D000D080E794E0EDB7FEB784
:1077E00092838183C6010196948383830E94477CA0
:1077F0000F900F900F900F9076010894E11CF11CF0
:107800008E010F5E1F4FC801B7010E94B5468091DF
:10781000B90482FF42C083EA94E0B801A70122E9DB
:1078200030E20E943A4B8091CE069091CF0692FFB3
:1078300034C002E910E2E1E8AE2EE4E0BE2ED80149
:107840008D918D0100D000D0EDB7FEB73196ADB768
:10785000BEB71296BC92AE921197828313820E9499
:10786000477C0F900F900F900F90B0E2023A1B07E9
:1078700031F78AE090E00E94797C00D000D086E861
:1078800094E0EDB7FEB792838183F482E3820E9495
:10789000477C0F900F900F900F908091CE069091A3
:1078A000CF0682FD73980E94E0528FED96E00E9411
:1078B0005B3D2AC01092B8041092B704739889E116
:1078C00090E00E9401548091F2068F5F8093F2064F
:1078D000898BB6016F5F7F4FCE0141960E94B546FE
:1078E0008FED96E00E945B3D8091880E9091890E0D
:1078F00065E840E050E00E94213F86EE99E0D20129
:1079000011969C938E9347C08091B9049091BA04CC
:1079100090FDD0CF8091D1069091D206009711F0C2
:107920000E9442528091F2068F5F8093F20680910E
:10793000CE069091CF0682FF77C8739A75C88AEEFB
:1079400096E00E940242009731F10E94E05280913D
:10795000B90487FD2B988AEE96E060E470E00E94FF
:10796000D7418EEF99E0F2019183808314C08AEEB3
:1079700096E00E940242009771F00E94425280916C
:10798000B90487FF51C82B9A4FC8D20111961C9297
:107990001E9283E001C081E0C557DF4F0FB6F89417
:1079A000DEBF0FBECDBFCF91DF911F910F91FF9032
:1079B000EF90DF90CF90BF90AF909F908F907F908F
:1079C0006F905F904F9008950895FC01DB018C91BA
:1079D000808311968C91119781830895FC01DB01BE
:1079E00090818C91981741F421E030E091811196BB
:1079F0008C911197981711F020E030E0C90108959B
:107A0000FC0180818093B72481818093B8240895FC
:107A1000DC011996ED91FC911A970280F381E02D1B
:107A2000309709F009950895EF92FF920F931F93F5
:107A3000DF93CF9300D0CDB7DEB78C0188E10E94F1
:107A40003047BC017E010894E11CF11CC7010E9473
:107A5000E53CD8011996ED91FC911A970190F081BF
:107A6000E02DC801B70109950F900F90CF91DF91DC
:107A70001F910F91FF90EF900895EF92FF920F9357
:107A80001F93CF93DF93EC018B017A0144E555E01E
:107A90000E94693DFA86E986C80168E575E00E94A2
:107AA000C83DDF91CF911F910F91FF90EF90089506
:107AB0000E94823D0895CF93DF93EC0188E167EB4C
:107AC00074E20E942647CE010E94853DDF91CF914E
:107AD0000895EF92FF920F931F93CF93DF93EC01E2
:107AE0008B017A010E94A13DF886EF82C8016CE506
:107AF00075E00E94C83DDF91CF911F910F91FF90DB
:107B0000EF9008950E94AA3D08950E94B7580895E5
:107B1000FC01A781B0852D913C91F901099508954B
:107B2000DC011796ED91FC9118970280F381E02D0E
:107B3000309709F00995089584E89EE00E9414406A
:107B40000895FC017383628384E89EE0BF010E9474
:107B50009F400895BC0184E89EE00E94664008951D
:107B6000CF93DF93EC0184E89EE00E94184008C0A8
:107B7000828193818C179D0739F0CF010E94DE40EE
:107B8000E82FF92F3097A1F7CF01DF91CF9108951A
:107B90000F931F93CF93DF938B010E94B03DEC01B5
:107BA000009731F01D830C83C8010E940F5B8E8308
:107BB000DF91CF911F910F9108951F93CF93DF9382
:107BC000EC01162F888580FF1DC0EC81FD81309768
:107BD000C9F0D093890EC093880E82E08887CE01C9
:107BE00006960995992787FD909502978230910511
:107BF00010F0133829F4CE01BE010E94063E02C0E7
:107C000081E08887DF91CF911F910895CF92DF9215
:107C1000EF92FF920F931F93CF93DF93EC017B01C1
:107C2000C090880ED090890E0091860E1091870E1C
:107C3000F80103C00190F081E02DEC17FD0719F069
:107C40003097C1F746C0209709F443C08885882340
:107C500009F118860BC0C017D10729F0C80167E8E1
:107C6000AE010E94DD3DF801008111810115110571
:107C700091F7EC81FD81309769F0CE15DF0551F069
:107C8000D093890EC093880ECE01069663E840E03B
:107C900050E00995E091860EF091870ECE17DF0730
:107CA00091F4888199819093870E8093860E0DC000
:107CB000808191818C179D0729F488819981918316
:107CC000808303C0FC01309799F7D092890EC0924F
:107CD000880EDF91CF911F910F91FF90EF90DF9071
:107CE000CF9008951F93CF93DF9310928A0EC09187
:107CF000860ED091870E11E00EC08985882341F051
:107D000018871986CE0162E840E050E00E94DD3D10
:107D10000990D881C02D209781F7DF91CF911F91D5
:107D200008958091350F982F9F5F9093350F089598
:107D30006091880E7091890E0E94063E08958AE82F
:107D40008093350F10928C0E10928B0E1092870E2E
:107D50001092860E1092890E1092880E08958091CE
:107D60008A0E882311F00E94723E70918B0E772349
:107D700009F455C020918C0E30E0F901EE0FFF1F81
:107D8000EE0FFF1FE20FF31FE357F14F6081609387
:107D9000340F418152815093330F4093320F8381CE
:107DA00094819093310F8093300F2F5F3F4F2F714D
:107DB000307020938C0E715070938B0E009741F5AC
:107DC0008091860E9091870E18C080918A0E88232C
:107DD00011F00E94723E4091320F5091330F80910A
:107DE0002E0F90912F0F6091340F0E94DD3DE09196
:107DF0002E0FF0912F0F8081918190932F0F809300
:107E00002E0F80912E0F90912F0F0097F1F607C043
:107E1000613819F421E0FC0120870E94DD3D80914A
:107E20008A0E20918B0E30E0280F311DC901089574
:107E300080918A0E20918B0E30E0280F311DC901F0
:107E4000089570918B0E7032D9F020918C0E270F0F
:107E50002F7120932D0F30E0F901EE0FFF1FEE0F71
:107E6000FF1FE20FF31FE357F14F608352834183FB
:107E7000948383837F5F70938B0E20E030E002C099
:107E800021E030E0C9010895CF93DF93C091880EBF
:107E9000D091890E0E94DD3DD093890EC093880E4B
:107EA000DF91CF910895FC01AB019091860E8091F6
:107EB000870E9C01A32FB22F03C00D90BC91A02D63
:107EC000AE17BF0791F01097C1F7309771F090830C
:107ED0008183F093870EE093860E81E0808717827E
:107EE0001682CF0161E80E94443F0895FC0100978B
:107EF00041F080858150823020F481E08187809339
:107F00008A0E089521E030E0FC018085882311F479
:107F100020E030E0C9010895CF93DF93EC014A815E
:107F20005B818C819D8160E070E00E94D17B4A8101
:107F30005B8188819981489F9001499F300D589FAE
:107F4000300D11248E819F8160E070E0A9010E94B4
:107F5000D17BDF91CF910895FC018281938120E054
:107F600030E019C0A481B581A20FB31F4C91442306
:107F700081F481E08C9340815181249FC001259F31
:107F8000900D349F900D112426813781280F391FC1
:107F900007C02F5F3F4F2817390720F320E030E05C
:107FA000C9010895FC01268137814281538180E017
:107FB00090E018C02617370781F4A481B581A80F77
:107FC000B91F2C91121614F421502C930480F581C2
:107FD000E02DE80FF91F80810895A081B1812A0F5B
:107FE0003B1F01968417950728F38FEF0895FC0136
:107FF000CB01268137816217730790F0A081B18190
:1080000062817381A69FA001A79F500DB69F500D5E
:108010001124420F531F21E030E08417950710F020
:1080200020E030E0C9010895FC011182108208951A
:10803000FC01808191810895FB0120813181FC0147
:10804000318320830895FC01208131812115310580
:1080500011F407C09C01F901808191810097D1F74B
:1080600002C020E030E0C9010895CF93DF93DC0126
:108070002D913C91119721153105A9F0F9018081CD
:108080009181009729F411961C921E920EC0F9015D
:1080900020813181D9018D919C9111970097B9F779
:1080A0001182108202C020E030E0C901DF91CF913F
:1080B0000895DC01ED91FC911197309729F08081B2
:1080C000918111969C938E93CF010895CF93DF9366
:1080D000FC01A081B1811097D9F0C0E0D0E016C0BA
:1080E000A617B70771F48D919C911197209719F4F9
:1080F0009183808302C09983888311961C921E927B
:1081000007C0ED0198818981A92FB82F109741F7F9
:10811000DF91CF9108950F931F93CF93DF938C013D
:10812000EB010E946640F8018081918199838883E8
:10813000D183C083DF91CF911F910F910895EF926A
:10814000FF920F931F93CF93DF93EC017B010E946B
:108150006640F70111821082CE010E942340FC018B
:10816000009719F4E882F98202C0F182E082DF917F
:10817000CF911F910F91FF90EF900895DC01ED9149
:10818000FC91119720E030E005C02F5F3F4F019038
:10819000F081E02D3097C9F7C9010895FB013097B0
:1081A00021F4BA010E948B400895DA018081918107
:1081B00011969C938E93518340830895009721F0EC
:1081C000FC012081318102C020E030E0C901089526
:1081D0008091360F9091370F009729F41092390F44
:1081E0001092380F08950E94A44FE091360FF0913D
:1081F000370F2281338140815181240F351F281B85
:10820000390B0CC04281538160817181460F571F29
:10821000481B590B4217530708F49A010480F58153
:10822000E02D309779F7280F391F3093390F2093BD
:10823000380F08958AE695E00E94763F0895CF9220
:10824000DF92EF92FF920F931F93CF93DF937C0106
:10825000FC0180819181009729F08A35910509F010
:108260006EC00BC01092370F1092360F8AE590E067
:10827000F7019183808381E066C0673849F5CA01C0
:10828000E091360FF091370F03C00480F581E02DA7
:10829000309741F32681378128173907B1F3E093EE
:1082A000360FF093370F0FC016962D913C9117970C
:1082B0002817390739F414962D913C911597358379
:1082C0002483DF01FD01A481B581109769F7CECF2A
:1082D000623861F6C091360FD091370F00E010E0A0
:1082E0002BC0CE010E94075F0097F1F08E819F8125
:1082F00068E8AE010E94213F0097A1F41F821E8210
:108300008C819D810115110521F0F80195838483ED
:1083100004C09093370F8093360F1D821C820E94F9
:10832000E840D8CF0E941A418E019C818D81C92ED0
:10833000E6016E01D82EE601209799F697CFF70156
:108340001182108283E0DF91CF911F910F91FF90F6
:10835000EF90DF90CF900895CF93DF93EC010E94D0
:108360001A418E819F81009769F0E091360FF0915C
:10837000370F06C0EC17FD07A9F00480F581E02D4A
:108380003097C1F78091880E9091890E9F838E83DC
:108390008091360F9091370F9D838C83D093370F48
:1083A000C093360F0E94E840DF91CF910895CF939C
:1083B000DF93EC010E94E75ECE010E94AC41DF91A9
:1083C000CF910895CF93DF93EC010E94F35ECE012D
:1083D0000E94AC41DF91CF910895CF93DF93EC01E0
:1083E0000E94FD5ECE010E94AC41DF91CF910895C5
:1083F000FC0180819181860F971F918380830E9469
:10840000E840089521E030E0FC01868197810097E3
:1084100011F020E030E0C9010895FC012281338190
:1084200080819181280F391FC9010895FC01808145
:108430009181089521E030E08091360F9091370FBF
:10844000009711F420E030E0C90108958091360FC3
:108450009091370F009729F02091380F3091390F04
:1084600002C020E030E0C9010895CF93DF93EC0112
:10847000E091360FF091370F8E179F0741F48C81F2
:108480009D819093370F8093360F14C0FC01309775
:1084900031F0848195818C179D07C1F707C01D823B
:1084A0001C821F821E82DF91CF9108958C819D8155
:1084B000958384830E94E840F2CFCF92DF92EF92BF
:1084C000FF920F931F93CF93DF938C017A01FC01EE
:1084D00080819181009729F08B34910509F051C07A
:1084E0001EC08BE39FE00E941840C82EE6017E016B
:1084F000F92EE70109C06C817D81CE0102960E94B0
:10850000D7410990D881C02D2097A9F781E08093A9
:108510003A0F8BE490E0F8019183808337C068388C
:10852000A9F58BE39FE00E941840C82EE6016E017A
:10853000D92EE60123C0CE010296E816F906D9F439
:108540008BE39FE0BE010E946640E090880EF090B1
:10855000890E8A859B859093890E8093880EEC8581
:10856000FD85309719F08E859F850995F092890ECB
:10857000E092880ECECF0990D881C02D2097D9F6F1
:10858000C8CFF8011182108283E001C081E0DF9141
:10859000CF911F910F91FF90EF90DF90CF900895B2
:1085A00010923A0F8BE39FE00E94144083E895E01D
:1085B00060E070E00E94533F08950F931F93CF93A4
:1085C000DF93EC010091880E1091890E1B870A87BA
:1085D0005D874C873F872E8780913A0F882379F0FB
:1085E00083E895E09093890E8093880ECE010296E1
:1085F0000E94D7411093890E0093880E02C07D839C
:108600006C838BE39FE0BE010E9466408BE39FE09A
:10861000BE010E949F40DF91CF911F910F9108955D
:108620000F931F93CF93DF93EC0180913A0F882330
:1086300091F00091880E1091890E83E895E0909357
:10864000890E8093880ECE0102960E94E24110931B
:10865000890E0093880E8BE39FE0BE010E94664066
:108660008BE39FE0BE010E949F40DF91CF911F915D
:108670000F9108950F931F93CF93DF93EC01809197
:108680003A0F882391F00091880E1091890E83E8AB
:1086900095E09093890E8093880ECE0102960E94F9
:1086A000ED411093890E0093880E8BE39FE0BE018D
:1086B0000E9466408BE39FE0BE010E949F40DF91D5
:1086C000CF911F910F910895CF93DF93EC0180918B
:1086D0003A0F882329F0CE0102960E94354204C049
:1086E0001F821E82198618868BE39FE0BE010E94BE
:1086F0006640DF91CF910895CF93DF93EC01809195
:108700003A0F882331F0CE0102960E9402429C016A
:1087100014C08BE39FE00E941840E82FF92F06C099
:10872000EC17FD0741F00190F081E02D3097C1F783
:1087300021E030E002C020E030E0C901DF91CF91BC
:1087400008950F931F930091B7241091B8240E94AD
:10875000D14F2DB73EB7225530400FB6F8943EBFEB
:108760000FBE2DBFEDB7FEB7319621ED3DE0ADB7A1
:10877000BEB712963C932E931197028313821483F3
:10878000158266837783808791878091AA2690914E
:10879000AB26A091AC26B091AD2682879387A487A3
:1087A000B5878091AE269091AF26A091B026B0916A
:1087B000B12686879787A08BB18B8091B226909146
:1087C000B326A091B426B091B526828B938BA48B4F
:1087D000B58B8091B6269091B726A091B826B0911E
:1087E000B926868B978BA08FB18F8091BA269091F6
:1087F000BB26A091BC26B091BD26828F938FA48FFB
:10880000B58F8091BE269091BF26A091C026B091D1
:10881000C126868F978FA0A3B1A38091C226909185
:10882000C326A091C426B091C52682A393A3A4A376
:10883000B5A38091C6269091C726A091C826B09175
:10884000C92686A397A3A0A7B1A78091CA26909115
:10885000CB26A091CC26B091CD2682A793A7A4A722
:10886000B5A78091CE269091CF26A091D026B09129
:10887000D12686A797A7A0ABB1AB8091D2269091C5
:10888000D326A091D426B091D52682AB93ABA4ABCE
:10889000B5AB8091D6269091D726A091D826B091DD
:1088A000D92686AB97ABA0AFB1AF8091DA26909175
:1088B000DB26A091DC26B091DD2682AF93AFA4AF7A
:1088C000B5AFEDB7FEB7FF968091DE269091DF261B
:1088D000A091E026B091E12680839183A283B383A7
:1088E000EDB7FEB7ED5BFF4F8091E2269091E32656
:1088F000A091E426B091E52680839183A283B3837F
:10890000EDB7FEB7E95BFF4F8091E6269091E72631
:10891000A091E826B091E92680839183A283B38356
:10892000EDB7FEB7E55BFF4F8091EA269091EB260D
:10893000A091EC26B091ED2680839183A283B3832E
:10894000EDB7FEB7E15BFF4F8091EE269091EF26E9
:10895000A091F026B091F12680839183A283B38306
:108960000E94597C0091B7241091B8242DB73EB7CE
:108970002E5A3F4F0FB6F8943EBF0FBE2DBF0E9438
:10898000D14FADB7BEB7D2970FB6F894BEBF0FBEEA
:10899000ADBFEDB7FEB7319622E63DE012963C93AF
:1089A0002E93119702831382148315826683778333
:1089B000808791878091F2269091F326A091F426EA
:1089C000B091F52682879387A487B5878091F62694
:1089D0009091F726A091F826B091F926868797877F
:1089E000A08BB18B8091FA269091FB26A091FC265A
:1089F000B091FD26828B938BA48BB58B8091FE2644
:108A00009091FF26A0910027B0910127868B978B2C
:108A1000A08FB18F8091022790910327A091042706
:108A2000B0910527828F938FA48FB58F80910627F1
:108A300090910727A0910827B0910927868F978FDB
:108A4000A0A3B1A380910A2790910B27A0910C2796
:108A5000B0910D2782A393A3A4A3B5A380910E2761
:108A600090910F27A0911027B091112786A397A36B
:108A7000A0A7B1A780911A2790911B27A0911C272E
:108A8000B0911D2782A793A7A4A7B5A780911E2701
:108A900090911F27A0912027B091212786A797A703
:108AA000A0ABB1AB0E94597C2DB73EB72E5C3F4FB7
:108AB0000FB6F8943EBF0FBE2DBF1F910F910895C2
:108AC00080E380933D0F0895EF92FF92CF93DF9361
:108AD00020913D0F30E0C0E3D0E0C21BD30B2E5BF2
:108AE000304FB901AE010E94C87BCE01DF91CF911A
:108AF000FF90EF900895AF92BF92CF92DF92EF92E6
:108B0000FF920F931F93CF93DF937C01C0903E0F92
:108B1000D0903F0F20913D0F30E08601005D1F4F48
:108B2000021B130B01381105E0F4C0E3D0E0C21BB7
:108B3000D30B2E5B304FB901AE010E94C87BCE0D26
:108B4000DF1D2091400F3091410F8091F40F9091E3
:108B5000F50F280F391FCE01B901A6010E94C87B6D
:108B600002C000E010E0C801DF91CF911F910F918A
:108B7000FF90EF90DF90CF90BF90AF9008959091CD
:108B80003D0F980F90933D0F089540913E0F5091E7
:108B90003F0F9C014817590798F08091F40F90916E
:108BA000F50F820F931F9093F50F8093F40F421BE4
:108BB000530B50933F0F40933E0F21E030E002C033
:108BC00020E030E0C901089590933F0F80933E0F5D
:108BD00008952091F40F3091F50F2E58304FC901B0
:108BE000089520913D0F30E02E5B304FC90108956C
:108BF00021E030E08091400F9091410F4FE08237AB
:108C0000940711F420E030E0C90108950E94F8456E
:108C1000009771F022E73FE06091400F7091410FA3
:108C200040913E0F50913F0FC9010E94C87B0895AB
:108C3000A091F40FB091F50F1097B9F020913E0F6D
:108C400030913F0F205D3F4FAE58B04FE2E7FFE05D
:108C500080E390E003C04D91419301968217930702
:108C6000D4F31092F50F1092F40F08958091400FF5
:108C70009091410F089580913E0F90913F0F08957C
:108C800090913D0F80E3891B089580E390913D0F03
:108C9000891B20913E0F30913F0F280F311DC901D4
:108CA00008951F93CF93DF93EC0110913D0F812F17
:108CB00090E08C179D076CF00E9445468C0F9D1F1D
:108CC0008138910530F41C1B10933D0F21E030E0FA
:108CD00002C020E030E0C901DF91CF911F910895DB
:108CE000CF93DF93E1ECF4E21192119284E2E13F41
:108CF000F807D1F7C0E0D0E0CE01880F991F875464
:108D00009B4D62E575E00E94E53C2196C430D1059B
:108D100099F7DF91CF9108951092F50F1092F40F0B
:108D200010923F0F10923E0F80E380933D0F82E739
:108D30009FE09093410F8093400F0E9470460895EA
:108D40000F931F93CF93DF93EC018B010E948C460E
:108D5000D093410FC093400F10933F0F00933E0FED
:108D6000DF91CF911F910F910895CF92DF92EF92F3
:108D7000FF920F931F93DF93CF9300D0CDB7DEB751
:108D80008C0169837A830E948C4669817A81C62E20
:108D9000D72E21E8C216D10418F030E8C32ED12C0A
:108DA0008091400F9091410FB801A6010E94C87BAD
:108DB000D0923F0FC0923E0FC6010F900F90CF91FF
:108DC000DF911F910F91FF90EF90DF90CF9008956A
:108DD000282F392FD901E1ECF4E280E301900D92C4
:108DE0008150E1F7862F972FDC01E9EBF4E288E070
:108DF00001900D928150E1F70895E1ECF4E2282F03
:108E0000392FD90180E30D9001928150E1F7A9EB50
:108E1000B4E2862F972FFC0188E001900D928150DB
:108E2000E1F70895E82FF0E0EE0FFF1FEF53FB4D41
:108E30007183608381E090E00895E82FF0E0EE0F09
:108E4000FF1FEF53FB4D80819181089590E0880FC3
:108E5000991F87579B4D0E94E53C81E090E0089563
:108E6000282F30E0220F331F27573B4DC9010895AB
:108E70008115910511F00197F1F70895E091F4241F
:108E8000F091F52490818091F32489230895E09155
:108E9000F124F091F22480819091F324892B808336
:108EA000E091F624F091F72480819091F324892BAE
:108EB00080830895E091F124F091F22490818091D3
:108EC000F324809589238083E091F624F091F724A0
:108ED00090818091F3248095892380830895FF9267
:108EE0000F931F93E091F124F091F22490818091EF
:108EF000F324809589238083E091F624F091F72470
:108F000080819091F324892B80838FEB93E00E94E2
:108F10003847FFB6F894E091F624F091F724908159
:108F20008091F32480958923808383E890E00E94D8
:108F30003847E091F424F091F52400811091F32456
:108F4000FFBE78948BE393E00E943847E091F424CD
:108F5000F091F52480819091F324892319F0802FDA
:108F6000812301C081E01F910F91FF9008955093DC
:108F7000F7244093F6247093F2246093F1249093A5
:108F8000F5248093F42481E090E002C0880F991FBB
:108F90002A95E2F78093F3240E946F4708950F9378
:108FA0001F93182F0FB7F894E091F624F091F7244F
:108FB00080819091F324892B808383E090E00E944C
:108FC0003847112351F0E091F624F091F724908175
:108FD0008091F32480958923808387E190E00E942B
:108FE0003847E091F424F091F52480819091F324A6
:108FF000892309F410E089E590E00E943847E09168
:10900000F624F091F72490818091F32480958923B0
:1090100080830FBF8BE390E00E943847812F1F9120
:109020000F9108950F931F93182F08E0812F8170DF
:109030000E94CF471695811110680150B9F7812F12
:109040001F910F9108958FEF0E9412480895DF92AB
:10905000EF92FF920F931F93CF93DF93182FEB01A3
:109060000E946F47882389F580EF0E941248EE2402
:1090700000E498EFD92ED00E81E00E94CF47F82E61
:1090800081E00E94CF47882319F0FF2069F020C0BB
:10909000FF2051F4011728F0888180FF05C01017C8
:1090A00019F0E02EFF24F3948F2D0E94CF47888182
:1090B00086958883FF2011F08068888301500D1504
:1090C000D9F6002339F02196D4CFEE24EA9402C0D9
:1090D0008EEFE82E8E2DDF91CF911F910F91FF9093
:1090E000EF90DF9008950F931F93CF93DF93182F86
:1090F000EB010E946F47209751F085E50E941248CE
:1091000008E089910E9412480150D9F703C08CEC05
:109110000E941248812F0E941248DF91CF911F9127
:109120000F9108950F931F93CF93DF93FB01DA0103
:10913000E801408150E0718160E0462B572B80317F
:1091400071F4BA016E7F13E0660F771F1A95E1F78D
:1091500096814CE050E0491B5109460F571F57FFBD
:1091600006C091E09C93509541955F4F01C01C92C1
:10917000883289F4848190E0BC016076707060363A
:10918000710549F086FF02C04E7F05C085FF02C011
:109190004C7F01C0487FCA0154E0969587955A9547
:1091A000E1F7F90180834F70488380E0DF91CF9130
:1091B0001F910F9108950F931F93CF93DF938C010D
:1091C000EB01F8018081BE010E942748F8018083ED
:1091D00081508D3F28F48881883211F0803189F7E1
:1091E000DF91CF911F910F9108951F93CF93DF933C
:1091F000EC010E946F4784EBBE010E94734881E03E
:109200000E94CF47182F0E946F4781E0112309F475
:1092100080E0DF91CF911F9108951F93CF93DF934B
:10922000182FEB010E946F470E943E47882349F0A8
:1092300084E4BE010E947348113029F00E94474720
:1092400002C082E001C080E0DF91CF911F910895BC
:109250006F927F928F929F92AF92BF92CF92DF9246
:10926000EF92FF920F931F93DF93CF93CDB7DEB7AB
:1092700029970FB6F894DEBF0FBECDBF7C014B011E
:109280003A0159010E946F478EEBB7010E94734863
:109290008E010F5F1F4F8AE0C82ED12CCC0EDD1E31
:1092A0000E942348F80181938F01EC15FD05C1F759
:1092B0008E010F5F1F4FC80169E070E00E94B86324
:1092C000882351F4F7018081B801A401930185013D
:1092D0000E94924880E001C083E029960FB6F8947E
:1092E000DEBF0FBECDBFCF91DF911F910F91FF90D9
:1092F000EF90DF90CF90BF90AF909F908F907F9036
:109300006F9008957F928F929F92AF92BF92CF926B
:10931000DF92EF92FF920F931F93DF93CF93CDB71E
:10932000DEB729970FB6F894DEBF0FBECDBF782EFB
:109330005B014A0179018EEB60E070E00E947348A6
:109340008E010F5F1F4F9AE0C92ED12CCC0EDD1E6F
:109350000E942348F80181938F01EC15FD05C1F7A8
:109360008E010F5F1F4FC80169E070E00E94B86373
:10937000882349F4872DB801A501940187010E9433
:10938000924880E001C083E029960FB6F894DEBFD2
:109390000FBECDBFCF91DF911F910F91FF90EF9046
:1093A000DF90CF90BF90AF909F908F907F90089567
:1093B0000F931F93DF93CF93CDB7DEB728970FB6E8
:1093C000F894DEBF0FBECDBF182F062FDE01119619
:1093D000E5E9F5E088E001900D928150E1F7242F56
:1093E000332727FD309541E752E0249FC001259F98
:1093F000900D349F900D112464E670E00E94C378B4
:10940000AB0164E6069FB0011124460F571FFE0111
:109410003196CE010996619170E02617370719F44D
:109420004F5F5F4F03C0E817F907A9F7112319F041
:10943000509541955F4FCA0128960FB6F894DEBF4C
:109440000FBECDBFCF91DF911F910F9108950F9364
:109450001F93DF93CF93CDB7DEB72B970FB6F8945A
:10946000DEBF0FBECDBF182F092F885F612F792F68
:109470000E940D49882309F049C066E471E48FE039
:1094800090E00E94944A812F902FBE016F5F7F4F22
:10949000AE014E5F5F4F9E012D5F3F4F0E942849F6
:1094A0008823A1F5DE011496EDE8F5E088E001904F
:1094B0000D928150E1F74B81642F70E021E732E09B
:1094C000629FC001639F900D729F900D112464E60E
:1094D00070E00E94C3789A8184E6989FC0011124AD
:1094E000680F791FFE013496CE010C962191421728
:1094F00019F46F5F7F4F03C0E817F907B9F7898147
:10950000882331F0709561957F4F02C064E371E26A
:10951000CB012B960FB6F894DEBF0FBECDBFCF9117
:10952000DF911F910F910895DC01CB018115910509
:10953000A105B10529F081509040A040B040D9F775
:1095400008951092B90080E28093B800089594EADB
:109550009093BC0020EA36E841E050E005C021507D
:10956000304040405040F1F09091BC0097FFF7CF61
:109570001DC09031B9F48093BB0084E88093BC0097
:1095800080EA96E8A1E0B0E004C00197A109B10922
:1095900059F02091BC0027FFF8CF0EC081E0903435
:1095A00021F40FC081E0089581E008959091B90001
:1095B000987F9830F1F6DFCF9091B900987F98317D
:1095C00069F780E0089544EA34E824E94093BC0058
:1095D0009091BC0097FFFCCF9091B900987F983094
:1095E00011F0903199F78093BB003093BC009091BB
:1095F000BC0097FFFCCF9091B900987F903211F09A
:10960000983539F42093BC009091BC0094FDFCCFB8
:10961000DDCF08950E94A74A089584E98093BC0095
:109620008091BC0084FDFCCF08958093BB0084E84A
:109630008093BC008091BC0087FFFCCF9091B90063
:10964000987F81E0983209F480E0089584EC80935B
:10965000BC008091BC0087FFFCCF8091BB000895C7
:1096600084E88093BC008091BC0087FFFCCF809190
:10967000BB000895E82FF92F80E1919190933F016D
:109680008150D9F780913C018F7D80933C0180917E
:109690003C01877F80933C01862F972FFC0180E15E
:1096A000919190933E018150D9F780913C0180685F
:1096B00080933C0180913D0180FFFCCF40515040A0
:1096C00080913C01806280933C0180913C01877FC6
:1096D00080933C0114C0862F972FFC0180E191916B
:1096E00090933E018150D9F780913C01806880932E
:1096F0003C0180913D0180FFFCCF40515040141649
:1097000015064CF3822F932FFC0180E190913E01CE
:1097100091938150D9F781E090E008950F931F93C2
:10972000CF93DF938C018CE70E94E34A8CE70E9481
:10973000154BC0E0D0E0F80181918F010E94154BDC
:109740002196C031D105B9F70E940D4BDF91CF9121
:109750001F910F910895813039F48CE790E060E01B
:1097600070E040E050E006C08CE790E060E070E020
:1097700040EC50E00E94F8100895813039F48CE7F5
:1097800090E060E070E04EE050E006C08CE790E0D2
:1097900060E070E048E050E00E94F81008958CE727
:1097A00090E060E070E041E050E00E94F8106AE66E
:1097B0007AE080E090E00E94944A08958CE790E07F
:1097C00060E070E048E350E00E94F8108CE790E021
:1097D00060E070E049E350E00E94F8108CE790E010
:1097E00060E070E044E150E00E94F8108CE790E007
:1097F00060E070E048E750E00E94F8108CE790E0ED
:1098000060E070E04EE550E00E94F8108CE790E0D8
:1098100060E070E04DE650E00E94F8106CE17AE103
:1098200086E090E00E94944A8CE790E060E070E06F
:109830004CE050E00E94F8108CE790E060E070E0AF
:1098400041E050E00E94F8108CE790E060E070E0AA
:1098500046E050E00E94F8106AE67AE080E090E08E
:109860000E94944A0895DF93CF93CDB7DEB7A297B5
:109870000FB6F894DEBF0FBECDBFDE011196EDE945
:10988000F5E081E101900D928150E1F7DE01529601
:10989000EEEAF5E081E101900D928150E1F70E943E
:1098A000DE4BCE0101960E948E4B82E00E94AB4BB4
:1098B0006AE67AE080E090E00E94944ACE01429607
:1098C0000E948E4B60E17EEA88E290E00E94944A1A
:1098D00080E00E94BD4B60E17EEA88E290E00E9459
:1098E000944A81E00E94BD4BA2960FB6F894DEBF69
:1098F0000FBECDBFCF91DF910895E6E4F1E0808106
:1099000020819081308182958695869583702295FD
:109910002F70822B832B92959F70892B0895DF9255
:10992000EF92FF920F931F93DF93CF9300D0CDB7A9
:10993000DEB780E06CE046E00E94655089E18093EC
:10994000C4001092C50082E08093C00080E00E94B5
:109950000F510E94944F84B784B784B784B784B7FB
:10996000E8E7FDE222E432E4318320833A968DB7C2
:109970009EB70A97E817F907B8F300D000D08EE138
:109980009FE0ADB7BEB712969C938E9311978FEB65
:1099900095E014969C938E9313970E94597C0F9098
:1099A0000F900F900F900E94D15F0E949F3E8AE619
:1099B00095E060E070E00E94533F0E94D042E09149
:1099C0000A06F0910B0609950E947D4C90E00E94DA
:1099D0000F60CE0101960E94C24E882359F000D03C
:1099E0008EEF9EE0EDB7FEB7928381830E94597C93
:1099F0000F900F908E010F5F1F4FC8010E94003D16
:109A00000E94CC4E7C010E94D14EBC01C701A8012E
:109A10000E941C540E942A4E0E9401540E94D64E5D
:109A20000E94895500D081EF9EE0ADB7BEB7129677
:109A30009C938E9311970E94597C00D0EDB7FEB78E
:109A400031960DEE1EE0ADB7BEB712961C930E9385
:109A500011978A81828313820E94597CEDB7FEB7E9
:109A60003196ADB7BEB712961C930E9311978981AC
:109A7000828313820E94597C0F900F908BEE9EE0A0
:109A8000EDB7FEB7928381830E94597C0F900F90AF
:109A90000E941560E0918D06F0918E060995E09187
:109AA0007406F09175060995E0913606F091370637
:109AB0000995E0907206F090730600918B06109164
:109AC0008C060E94FE53D82E0E9491552DB73EB7AA
:109AD0002A5030400FB6F8943EBF0FBE2DBFEDB7F1
:109AE000FEB7319620ED3EE0ADB7BEB712963C937F
:109AF0002E931197F382E28215830483D682178214
:109B0000808711860E94597CE0919706F091980613
:109B10002DB73EB7265F3F4F0FB6F8943EBF0FBE3E
:109B20002DBF3097D1F00995BC0100D000D08DEB4E
:109B30009EE0ADB7BEB712969C938E93119780E8C6
:109B400090E00E94AF78EDB7FEB7748363830E9404
:109B5000597C0F900F900F900F9000D08BEB9EE0F0
:109B6000ADB7BEB712969C938E9311970E94597C05
:109B70000F900F9086EB96E060E070E00E94533FFC
:109B800088E395E00E94BB5E00D083EB9EE0EDB7DA
:109B9000FEB7928381830E94597C0F900F900F90A3
:109BA0000F90CF91DF911F910F91FF90EF90DF9079
:109BB0000895EF92FF920F931F9380E880936100C6
:109BC000109261000E948F4C0E94AF3E0E94305163
:109BD0008091F8249091F924009729F001979093AF
:109BE000F9248093F824E090FA24F090FB2400916B
:109BF000FC241091FD240E94D14FE616F7060807B9
:109C0000190711F30E94D14F6093FA247093FB243B
:109C10008093FC249093FD24D7CF00D000D000D0B7
:109C2000EDB7FEB731962DEA3EE0ADB7BEB712965E
:109C30003C932E93119793838283758364830E9450
:109C4000597C8DB79EB706960FB6F8949EBF0FBE8F
:109C50008DBF08950F931F93DF93CF93CDB7DEB7DA
:109C6000A2970FB6F894DEBF0FBECDBF82E490E09E
:109C70000E94A37D89839A83982F9B50903108F08E
:109C80008A839A819095891709F470C000D089E57C
:109C90009FE0ADB7BEB712969C938E9311970E942A
:109CA000597C8E010D5F1F4F0F900F90D80180E0FF
:109CB00090E0FC01E75CF04FE491ED930196883071
:109CC0009105B9F7F894CE01039660E270E048E0A0
:109CD00050E00E94A97DD80180E090E0FC01EF5B9C
:109CE000F04FE491ED9301968E309105B9F7CE01D6
:109CF000039668E270E04EE050E00E94A97D80E0AB
:109D000090E0FC01E15BF04FE491D801ED938D010F
:109D100001968A309105A9F7CE01039666E370E0BB
:109D20004AE050E00E94A97D84E490E06DEC7BEA7B
:109D30000E94C17D86E490E060E070E00E94C17DF9
:109D400088E490E060E00E94B37D80E490E060E011
:109D500070E00E94C17D8AE1898385EE8A836981F2
:109D60007A8182E490E00E94C17D78948981A296F4
:109D70000FB6F894DEBF0FBECDBFCF91DF911F911C
:109D80000F910895F89460E270E042E050E00E9484
:109D90008B7D789480E0089584E490E00E94A37D18
:109DA000089586E490E00E94A37D089588E490E001
:109DB0000E949B7D089520910625309107254091B2
:109DC00008255091092590E0A0E0B0E0280F391F48
:109DD0004A1F5B1F209306253093072540930825D3
:109DE00050930925209102253091032540910425A7
:109DF00050910525280F391F4A1F5B1F209302250C
:109E00003093032540930425509305252091A626E1
:109E10002223A1F02091FE243091FF2440910025BF
:109E200050910125280F391F4A1F5B1F2093FE24E4
:109E30003093FF24409300255093012508951F92ED
:109E40000F920FB60F920BB60F9211242F933F93E0
:109E50004F935F936F937F938F939F93AF93BF9332
:109E6000EF93FF938091F60F9091F70F01969093E7
:109E7000F70F8093F60F8091F80F8F5F8093F80FA4
:109E80008091F80F8038A9F41092F80F8091062580
:109E900090910725A0910825B09109250196A11D53
:109EA000B11D8093062590930725A0930825B093B4
:109EB00009258091A6268823F1F08091F90F8F5F04
:109EC0008093F90F8091F90F8038A9F41092F90F5F
:109ED0008091FE249091FF24A0910025B09101254E
:109EE0000196A11DB11D8093FE249093FF24A093A1
:109EF0000025B09301250E941A42009711F00E949C
:109F00001A41FF91EF91BF91AF919F918F917F91F6
:109F10006F915F914F913F912F910F900BBE0F90DA
:109F20000FBE0F901F901895F8941092B60016BCB3
:109F300083EF87BD82E084BD94E095BD95B395BB6A
:109F400080936E00789408952091F60F3091F70F6A
:109F50008091F60F9091F70F28173907A9F7C901DB
:109F6000089507C022E330E0000021503040E1F7BF
:109F700001970097B9F708950F931F93CF93DF933D
:109F80008C010E94A44FEC010E94A44F8C1B9D0BDE
:109F900080179107C8F3DF91CF911F910F9108951A
:109FA000089520910625309107254091082550916C
:109FB00009258091062590910725A0910825B0914B
:109FC0000925281739074A075B0759F7B901CA015C
:109FD00008951F920F920FB60F9211241092E3056D
:109FE0000F900FBE0F901F9018951F920F920FB6F3
:109FF0000F920BB60F9211242F933F934F935F93C1
:10A000006F937F938F939F93AF93BF93EF93FF9340
:10A01000E091D905F091DA058081E091E405F091B5
:10A02000E505309709F00995FF91EF91BF91AF9148
:10A030009F918F917F916F915F914F913F912F9160
:10A040000F900BBE0F900FBE0F901F9018951F9290
:10A050000F920FB60F9211241092F0050F900FBEC1
:10A060000F901F9018951F920F920FB60F920BB67C
:10A070000F9211242F933F934F935F936F937F938E
:10A080008F939F93AF93BF93EF93FF93E091E60578
:10A09000F091E7058081E091F105F091F2053097AC
:10A0A00009F00995FF91EF91BF91AF919F918F9129
:10A0B0007F916F915F914F913F912F910F900BBEC8
:10A0C0000F900FBE0F901F90189590E02DE030E09C
:10A0D000829FF001839FF00D929FF00D1124E752B3
:10A0E000FA4FA281B3811C92A481B5816C93A681A1
:10A0F000B78188ED8C93A085B1854C931286148628
:10A100001386089590E02DE030E0829FF001839F58
:10A11000F00D929FF00D1124E752FA4F81E08287F3
:10A12000A081B1816C933A9680818823E9F70895E4
:10A130001F93182F8A3031F48091FA0F6DE00E943E
:10A14000825002C08D3029F08091FA0F612F0E9459
:10A15000825080E090E01F910895EF92FF921F934C
:10A16000CF93DF93182FE62EE7017E01F72EE7014C
:10A170000CC08A3021F4812F6DE00E9482506991D9
:10A180006D3019F0812F0E9482508881882389F7D1
:10A19000DF91CF911F91FF90EF9008950F931F9340
:10A1A000DF93CF93CDB7DEB7FE013A960BEF1FE0FA
:10A1B000C80160E470E0488559859F010E94F57CE4
:10A1C0008F81B8010E94AD50CF91DF911F910F9107
:10A1D00008951F93CF93DF93182FEB0104C0812FB5
:10A1E0000E9482502196FE0164916623C1F7DF919F
:10A1F000CF911F91089590E02DE030E0829FF00113
:10A20000839FF00D929FF00D1124E752FA4F74874F
:10A2100063870895682F80E00E948250089580939C
:10A22000FA0F8BEC95E09093732D8093722D089527
:10A2300084B7877F84BF88E10FB6F894809360006D
:10A24000109260000FBE08952FE088E190E00FB6F5
:10A25000F894A895809360000FBE20936000089545
:10A26000A895089588E10FB6F89480936000109245
:10A2700060000FBE0895F89428E088E190E00FB6E2
:10A28000F894A895809360000FBE20936000FFCFE4
:10A290008091192590E0FC01EE0FFF1F9695982FF5
:10A2A000882797958795E80FF91FE65EFA4D10828B
:10A2B0000895809111258091112590E00895809155
:10A2C000390181FD0CC081E491E06FE140E00E9422
:10A2D0003257813039F021E030E0813129F020E03F
:10A2E00030E002C021E030E0C901089580913901D9
:10A2F00081FD12C081E491E06FE140E00E9432579D
:10A30000982F8151823050F09F3141F0913041F0CF
:10A3100081E0923031F402C081E0089580E0089538
:10A3200080E008950E9476518823E1F3089581E446
:10A3300091E06FE140E00E9432570895E9E3F1E0D7
:10A34000808180818D7F80838DE090E00197F1F79F
:10A3500082E491E06FE140E023E00E943C5783E01B
:10A3600090E00197F1F708950E9492511092A6266D
:10A370000E949E51809139018260809339018091C1
:10A3800029278823E9F180919400909195002091EC
:10A390003A2730913B2782179307A0F48091062734
:10A3A00090910727A0910827B09109278C57914ECB
:10A3B000AF4FBF4F8093062790930727A09308279E
:10A3C000B09309278091940090919500821B930B84
:10A3D000A0E0B0E0209106273091072740910827A0
:10A3E00050910927820F931FA41FB51F8093062742
:10A3F00090930727A0930827B09309271092292745
:10A4000080912B278823E9F1809194009091950009
:10A4100020913E2730913F2782179307A0F4809127
:10A420000E2790910F27A0911027B09111278C57DC
:10A43000914EAF4FBF4F80930E2790930F27A0935D
:10A440001027B09311278091940090919500821B62
:10A45000930BA0E0B0E020910E2730910F274091A0
:10A46000102750911127820F931FA41FB51F8093AF
:10A470000E2790930F27A0931027B09311271092C7
:10A480002B2708958091A626882381F080913B1088
:10A49000882321F40E947651882331F481E080934F
:10A4A000BE1021E030E004C00E94B45120E030E052
:10A4B000C90108950F931F93182F883049F08630F3
:10A4C00039F0893029F0863119F0893109F041C01D
:10A4D0008091390181FD40C00E9492510E949751A4
:10A4E000082F181709F43BC0183019F40E949E5128
:10A4F00029C0193141F48631A9F482E491E06FE179
:10A5000040E029E009C0163169F4893159F482E448
:10A5100091E06FE140E026E00E943C57E3E0F0E08C
:10A520003197F1F782E491E06FE140E0212F0E9442
:10A530003C57083019F4E9E6F1E002C0E3E0F0E04E
:10A540003197F1F70E949751811749F023E430E0E9
:10A5500008C022E430E005C024E430E002C020E47A
:10A5600030E0C9011F910F9108958091940090915E
:10A57000950090933F2780933E2721E020932B273F
:10A580008091390181FF15C02093A5268091940008
:10A590009091950090933B2780933A272093292709
:10A5A000809139018D7F809339018091A526882380
:10A5B000E1F786E10E945A5281E08093A626089531
:10A5C0008091A626882351F480913B10882321F0A6
:10A5D00081E08093BD1002C00E94B55281E090E0FE
:10A5E00008951F93DF93CF930F92CDB7DEB78FB748
:10A5F000898380913B10882331F5F8948091A626B9
:10A60000882351F08091390181FD1BC00E94765151
:10A610008823B9F080E003C00E94E05281E090916D
:10A6200047019E3010F010E001C01FEF882311F0A9
:10A630000E94425216FF05C089818FBF21E030E0A1
:10A6400004C089818FBF20E030E0C9010F90CF9115
:10A65000DF911F9108958091BD10882321F00E9401
:10A66000B5521092BD108091BE10882321F00E9437
:10A67000B4511092BE1010923B100895EF92FF92C9
:10A68000CF93DF93B82FA92FF62FE72F81E0809388
:10A690003B102091EA263091EB264091EC26509118
:10A6A000ED262F5F3F4F4F4F5F4F2093EA263093A9
:10A6B000EB264093EC265093ED26862F8E5F87FF86
:10A6C0000CC08091A3269091A42601969093A42675
:10A6D0008093A326CFEFDFEF0BC02CE330E1C9015D
:10A6E0006B2F7A2F4F2F5E2F0E94C87BC0E0D0E0E7
:10A6F0000E942B53CE01DF91CF91FF90EF900895F0
:10A700009091390191FD0AC0282F803108F02FE087
:10A7100085E491E06FE040E00E943C57089580930B
:10A72000C01008950E9497518250813130F4E82F73
:10A73000F0E0E25EF94F8081089581E00895089588
:10A740008FEF80934E018CE691E060EF44E022E0D1
:10A750000E943C578CE290E06EE041E025E00E94D0
:10A760003C5780E880936F018091460180936D0192
:10A7700084E491E060E245E021E00E943C570895C6
:10A78000CF93DF93CDEFD3E0CE010197F1F70E9495
:10A79000285710921A2510929C2510921E2610926E
:10A7A000192510921825E9E3F1E080818E7F8083DE
:10A7B00080818D7F80838DE090E00197F1F780812B
:10A7C0008160808382E491E06FE140E023E00E94B9
:10A7D0003C572197F1F780915D0180915E010E94C5
:10A7E000A05380E096E060E070E00E94533F0E943A
:10A7F000B55281E090E0DF91CF9108958091BF1034
:10A800000895DF93CF930F92CDB7DEB789830E946F
:10A81000925129812093BF1088E491E06FE140E0DC
:10A820000E943C570F90CF91DF9108950E940154F0
:10A8300086E00E945A5208958093620190936301CA
:10A8400060936001709361014115510531F1FA0186
:10A85000819180936B01DA0111968C9180936A014A
:10A86000DF011196818180936901FD013196119676
:10A870008C9180936801DF0111968181809367013B
:10A88000FD01319611968C9111978093660181811B
:10A8900080936501828180936401089580E096E051
:10A8A0000E94763F81E0809311258091122590913E
:10A8B00013250196909313258093122581E090E053
:10A8C0000895EF92FF92CF93DF9350911925252F92
:10A8D00030E0F901EE0FFF1F3695322F2227379512
:10A8E0002795E20FF31FE65EFA4D4081442309F4F9
:10A8F000CEC02091390121FDCAC02091A626222375
:10A9000009F4C5C047FF16C00E9448518091DA265D
:10A910009091DB26A091DC26B091DD260196A11D49
:10A92000B11D8093DA269093DB26A093DC26B093AA
:10A93000DD26ADC04330B0F40E9448518091D62648
:10A940009091D726A091D826B091D9260196A11D25
:10A95000B11D8093D6269093D726A093D826B09386
:10A96000D92695C0C42FD0E022976C177D07B0F48C
:10A970000E9448518091D2269091D326A091D4264E
:10A98000B091D5260196A11DB11D8093D22690933A
:10A99000D326A093D426B093D52679C0652F70E036
:10A9A0009B01220F331F7695762F66277795679543
:10A9B000260F371F255E3A4DB90150E00E94C87B33
:10A9C00020911925822F90E0FC01EE0FFF1F969534
:10A9D000982F882797958795E80FF91FE656FA4D27
:10A9E000808180930A25822F90E0FC01EE0FFF1FEB
:10A9F0009695982F882797958795E80FF91FE65E1B
:10AA0000FA4D10822F5F20931925233010F01092F9
:10AA100019258091192590E0FC01EE0FFF1F9695F6
:10AA2000982F882797958795E80FF91FE65EFA4DCE
:10AA30008081882311F00E944E54609147016093F9
:10AA40000B2580911025882311F0681710F460936E
:10AA5000102584E070E00E94124760910A2583E08F
:10AA600070E00E9412478091EE269091EF26A0910F
:10AA7000F026B091F1260196A11DB11D8093EE261E
:10AA80009093EF26A093F026B093F12602C0C0E089
:10AA9000D0E0CE01DF91CF91FF90EF900895CF935A
:10AAA000DF93EC0188819981009729F024E08B3FA6
:10AAB000920739F505C08BEF94E09983888325C010
:10AAC000623819F5109211250E948C460E94E945C2
:10AAD00060E870E00E9461541816190644F40E9460
:10AAE000E445E0919106F09192060995E4CF8091BA
:10AAF0000E2590910F25019690930F2580930E259A
:10AB0000DACF1982188283E001C081E0DF91CF9112
:10AB1000089591E090933B100E9480530E942B5324
:10AB200008958091390181FD07C085E491E06FE0CF
:10AB300040E00E943257089580E10895CF92DF925D
:10AB4000EF92FF920F931F93CF93DF93182F21E083
:10AB500020933B100091A6268091390181FF16C0F9
:10AB6000809194009091950090933B2780933A2791
:10AB7000209329272093A526809139018D7F8093EA
:10AB800039018091A5268823E1F700E00E949251C7
:10AB90008091A626882309F441C080912B27882321
:10ABA000E9F1209194003091950080913E27909199
:10ABB0003F2728173907A0F420910E2730910F273F
:10ABC00040911027509111272C57314E4F4F5F4F16
:10ABD00020930E2730930F2740931027509311276F
:10ABE0002091940030919500281B390B40E050E0F3
:10ABF000C0900E27D0900F27E0901027F0901127DB
:10AC00002C0D3D1D4E1D5F1D20930E2730930F27E9
:10AC1000409310275093112710922B2789E10E940F
:10AC20005A5286E00E941D47009751F00E949155AC
:10AC3000C82F86E00E941D4781500E94805302C0A9
:10AC4000C0E0D0E0809194009091950090933D27D2
:10AC500080933C2781E080932A27F89480913901E2
:10AC6000826080933901809139018D7F8093390111
:10AC7000612F6E5F8CE390E10E946D577894809114
:10AC8000A0269091A12601969093A1268093A026BC
:10AC90000E94925182E491E060EE45E00E943257BA
:10ACA000182F86E00E941D47009719F08C2F0E94F4
:10ACB0008053002319F00E94B55202C00E94B45183
:10ACC00080912A278823E9F1809194009091950042
:10ACD00040913C2750913D2784179507A0F480911F
:10ACE0000A2790910B27A0910C27B0910D278C5724
:10ACF000914EAF4FBF4F80930A2790930B27A0939D
:10AD00000C27B0930D272091940030919500241BBF
:10AD1000350B40E050E080910A2790910B27A091DD
:10AD20000C27B0910D27280F391F4A1F5B1F209356
:10AD30000A2730930B2740930C2750930D2710922E
:10AD40002A278091A626882361F080919400909113
:10AD5000950090933F2780933E2781E080932B2797
:10AD600007C082E491E06FE140E023E00E943C579D
:10AD70000E942B531130E1F01330A9F48091E226A8
:10AD80009091E326A091E426B091E5260196A11DBD
:10AD9000B11D8093E2269093E326A093E426B0931E
:10ADA000E52612E00AC0153029F0173031F404C04E
:10ADB00010E003C013E001C011E0812F90E0DF91AB
:10ADC000CF911F910F91FF90EF90DF90CF9008955A
:10ADD000CF93DF93EB010E943E539C01009731F427
:10ADE000CE010E949E559C01009749F08091A326B8
:10ADF0009091A42601969093A4268093A326C9013E
:10AE0000DF91CF9108950F931F938091A6268823F9
:10AE100021F40E94E05211E001C010E00E9497511D
:10AE2000863111F0813119F40091470109C086E49F
:10AE300091E06FE140E00E943257082F000F080FA9
:10AE4000112311F00E944252802F1F910F910895FB
:10AE50001092C2101092C110EFE6F0E08081806283
:10AE600080830895FC018081862390E002C095953F
:10AE700087954A95E2F70895F894FC019081862F12
:10AE80008095892330E002C0220F331F4A95E2F7F4
:10AE90002623282B208378940895DC011196209195
:10AEA0007B01FC012083215030E0A9014F575E4F08
:10AEB000E0E8F1E061916D93E417F507D9F7FC0143
:10AEC000E058FF4F2F573E4FD9012C9120838F57C9
:10AED0009F4F21E0FC0120830895FC0160938001D5
:10AEE00001966350860F911DA1E8B1E021912D9349
:10AEF000E817F907D9F708951F920F920FB60F922E
:10AF00000BB60F9211242F933F934F935F936F9340
:10AF10007F938F939F93AF93BF93EF93FF93809112
:10AF2000470180930B252091182530E0C901880F37
:10AF3000991F3695322F222737952795820F931F19
:10AF4000865E9A4D0E944D57809118258F5F8093A1
:10AF50001825833010F0109218250E944E54FF914E
:10AF6000EF91BF91AF919F918F917F916F915F9181
:10AF70004F913F912F910F900BBE0F900FBE0F90EE
:10AF80001F9018951F920F920FB60F9211240F90D9
:10AF90000FBE0F901F9018951F920F920FB60F9231
:10AFA00011240F900FBE0F901F9018951F920F92B3
:10AFB0000FB60F9211240F900FBE0F901F9018958F
:10AFC0001F920F920FB60F9211241092A5260F9088
:10AFD0000FBE0F901F9018951F920F920FB60F92F1
:10AFE00011241092A5260F900FBE0F901F90189558
:10AFF0001F920F920FB60F9211248F9381E08093CE
:10B0000011258F910F900FBE0F901F9018951F92D2
:10B010000F920FB60F9211241092A5260F900FBE1B
:10B020000F901F9018951F920F920FB60F92112438
:10B030008F939F938091C1109091C210019690932D
:10B04000C2108093C1109F918F910F900FBE0F90EF
:10B050001F9018950F931F93CF93DF938091AE2687
:10B060009091AF26A091B026B091B1260196A11D76
:10B07000B11D8093AE269093AF26A093B026B093D7
:10B08000B1260E94DB5AEC0183EC90E10E9418404B
:10B090000BC0D8011296ED91FC911397309709F0EF
:10B0A0000995C8010E94DE40082F192F01151105CE
:10B0B00081F7209719F0CE010E94883DDF91CF9152
:10B0C0001F910F9108950E9415600E948C460E9466
:10B0D000E55882E796E09093A9268093A8260E94DF
:10B0E000D85A82E090E060E074E040E05EE12FEF4B
:10B0F00031E00E94995A0895CF92DF92EF92FF9229
:10B100000F931F93CF93DF936C01EB018A0183ECC4
:10B1100090E10E9418400CC0D7011496ED91FC916B
:10B120001597309711F0CE010995C7010E94DE40B6
:10B13000E82EF92EE114F10479F7C601BE01A80149
:10B140000E94903DDF91CF911F910F91FF90EF9062
:10B15000DF90CF900895BC0183EC90E10E949F4066
:10B160000895BC0183EC90E10E9466400895CF935E
:10B17000DF93EC018091AA269091AB26A091AC269A
:10B18000B091AD260196A11DB11D8093AA26909382
:10B19000AB26A093AC26B093AD26CE010E94F25A06
:10B1A000009769F00E940646E0917606F0917706D6
:10B1B0008CE798E5BE01099521E030E002C020E06F
:10B1C00030E0C901DF91CF91089585EC90E10E94B4
:10B1D000144008950F93CF93DF93EC017B836A8330
:10B1E00018865F834E8385EC90E1BE010E949F40EC
:10B1F000E091C710F091C810309749F04C815D8103
:10B200008A819B81688520E030E001E00995DF912B
:10B21000CF910F910895BC0185EC90E10E946640AA
:10B2200008950F93DC0118961C921897E091C710AF
:10B23000F091C810309759F012968D919C91139708
:10B2400060E040E050E020E030E000E009950F9140
:10B2500008950F93DC01AB0114962D913C91159745
:10B2600081E018968C93189715967C936E9314979B
:10B27000E091C710F091C810309739F012968D9177
:10B280009C91139761E000E009950F9108950F9349
:10B29000DC01E091C710F091C810309769F0149666
:10B2A0002D913C91159712968D919C91139718961C
:10B2B0006C91A90101E009950F910895E091C910E1
:10B2C000F091CA10309709F0099508959093CA102B
:10B2D0008093C91008959093C8108093C710089563
:10B2E00085EC90E10E9418400895EF92FF920F9331
:10B2F0001F93CF93DF938C01EB017A0185EC90E1F2
:10B300000E94184015C0DC0112962D913C911397B4
:10B310002C173D0759F41696ED91FC91179730972D
:10B3200061F0B801AE019701099507C00E94DE40A7
:10B33000282F392FC901009731F7DF91CF911F9145
:10B340000F91FF90EF9008950895AF92BF92CF9222
:10B35000DF92EF92FF920F931F93DF93CF9300D072
:10B36000CDB7DEB75B010E94E945FC010081118188
:10B370001A8309830C30110518F4EE24FF242EC023
:10B3800000D000D08AE396E0EDB7FEB792838183C8
:10B39000148303830E94477C0F900F900F900F90AF
:10B3A00020C00E94E945F701EE0FFF1FEE0FFF1FBF
:10B3B000E80FF91FC280D3800E94E9450894E11C80
:10B3C000F11CF701EE0FFF1FEE0FFF1FE80FF91F33
:10B3D00040815181C501B6010E947559E016F10600
:10B3E00000F30F900F90CF91DF911F910F91FF907D
:10B3F000EF90DF90CF90BF90AF900895CF93DF9301
:10B40000C6EED0E16091FC107091FD10CE0140E3DA
:10B410005AE520E030E00E94DD420E941260609117
:10B42000FC107091FD100E94AF78BC01CE014097D6
:10B4300045E45AE520E030E00E94DD42DF91CF9103
:10B4400008950F93013051F48091F6109091F71008
:10B450009093FD108093FC100E94FE590F91089567
:10B460008091FC109091FD102091FA103091FB100A
:10B47000880F991F2817390708F4C9019093FD1008
:10B480008093FC100E94FE590895EF92FF92CF9393
:10B49000DF930E948C460E94E945E82EE7017E0179
:10B4A000F92EE701198218820E94705926C028815E
:10B4B0003981F901EE0FFF1FEE0FFF1FEC0FFD1F8B
:10B4C000DC0112964D915C911397538342832F5F59
:10B4D0003F4FF901EE0FFF1FEE0FFF1FEC0FFD1F97
:10B4E00014964D915C91159751834083398328833D
:10B4F0000E94DE40282F392FC901009721F0FC015E
:10B5000020852223A1F688819981880F991F880FB1
:10B51000991F02960E94E44588819981009721F045
:10B520008BEC90E10E945B3DDF91CF91FF90EF901B
:10B530000895EF92FF920F931F93CF93DF93FC0137
:10B540008B017A01E9018BEC90E1BF0147E556E000
:10B550000E943D3D1093F7100093F610F092F91001
:10B56000E092F810D093FB10C093FA1081E29AE5B4
:10B570000E946B59DF91CF911F910F91FF90EF9037
:10B580000895CF93DF93C6EED0E1CE010E946443CD
:10B59000CE0140970E946443CE014B970E94583DD4
:10B5A000DF91CF9108958091FC109091FD10089546
:10B5B0000E949C3D0895EF92FF92CF93DF93E0911C
:10B5C0005B06F0915C060995EC01009729F06A8111
:10B5D0007B8181E00E941247CE01DF91CF91FF90E5
:10B5E000EF9008950F931F93CF93DF938C01E09119
:10B5F0005D06F0915E060995EC01F80162817381A8
:10B6000081E00E94124721E030E0209711F420E011
:10B6100030E0C901DF91CF911F910F910895E09122
:10B620005F06F091600609950895FC0120E030E086
:10B6300004C08181280F311D329680818823C9F78B
:10B64000C9010895FC01818190E0308120E0822BC6
:10B65000932B02C0880F991F6A95E2F7892F9927CB
:10B66000FA01EF59F94F208130E08223932328E03B
:10B6700030E0241B350B02C0969587952A95E2F79A
:10B6800008956F927F928F929F92AF92BF92CF92C6
:10B69000DF92EF92FF920F931F93CF93DF936C0192
:10B6A0007B015A0189012830310544F4CB01BA01EC
:10B6B000A9010E94225BF601808341C0390133E079
:10B6C000759467943A95E1F74115510521F04C01C5
:10B6D000C0E0D0E016C0DB01FC01C0E0D0E08D91FD
:10B6E00081932196C615D705D4F3A80147705070F1
:10B6F0004115510521F1C7018C0F9D1F60E070E0DD
:10B7000019C0C7018C0F9D1FB50148E050E00E9491
:10B71000225BF40181934F012196C615D7058CF366
:10B72000A801477050704115510549F0C7018C0FB1
:10B730009D1FB5010E94225BCC0DDD1D8883DF912A
:10B74000CF911F910F91FF90EF90DF90CF90BF901E
:10B75000AF909F908F907F906F9008954F925F92DF
:10B760006F927F928F929F92AF92BF92CF92DF9211
:10B77000EF92FF920F931F93DF93CF9300D000D0EF
:10B78000CDB7DEB70E94E945E82E092F82E090E0B0
:10B790000E94C545009709F464C0EE2DF02F9181F9
:10B7A00080E02081820F911D0E94B03D7C010097B6
:10B7B00009F459C00E94E9453C01F7014681242F54
:10B7C00030E02770307081E090E02115310511F4F0
:10B7D00080E090E0469546954695840F911D0E9425
:10B7E000C5450097F1F1F70104811581CC24DD24D2
:10B7F00053E0452E512C4C0E5D1E4E010894811CC9
:10B80000911C2AC0F801A180BB24B60143E07595C4
:10B8100067954A95E1F7660D771DA6014770507050
:10B82000883150F0C40195010E94415BF80180818C
:10B83000B4010E9426470CC01C821B82C2019501E4
:10B840000E94415B6B817C81F80180810E941247DC
:10B85000CA0CDB1C0E5F1F4FF8018081882391F614
:10B8600002C0EE24FF24C7010F900F900F900F909D
:10B87000CF91DF911F910F91FF90EF90DF90CF90CC
:10B88000BF90AF909F908F907F906F905F904F9000
:10B890000895FC0150E080E190E0861B970B821B2D
:10B8A000930B02C0440F551F8A95E2F78081852BC8
:10B8B00080838181842B818308956F927F928F9200
:10B8C0009F92AF92BF92CF92DF92EF92FF920F932F
:10B8D0001F93CF93DF938C015B016A0179012830BC
:10B8E000310524F4C801FA01408156C0390163E0F2
:10B8F000759467946A95E1F7A114B10421F04A01A7
:10B90000C0E0D0E021C0DA01F80180E090E02D91A4
:10B910002193019686159705D4F39701277030700F
:10B9200021153105D9F1F601E80FF91F408150E0EA
:10B9300068E070E0621B730B02C0559547956A95ED
:10B94000E2F7800F911F26C0F40141914F01C80119
:10B950008C0F9D1FB50128E030E00E94495C2196C4
:10B96000C615D7058CF39701277030702115310566
:10B97000A9F0F601EC0FFD1F408150E0C5010896CB
:10B98000821B930B02C0559547958A95E2F7C80133
:10B990008C0F9D1F60E070E00E94495CDF91CF91A9
:10B9A0001F910F91FF90EF90DF90CF90BF90AF90DD
:10B9B0009F908F907F906F9008954F925F926F92BB
:10B9C0007F928F929F92AF92BF92CF92DF92EF922F
:10B9D000FF920F931F93DF93CF9300D0CDB7DEB7C5
:10B9E0008C01DC0116964C911697842F90E087709D
:10B9F000907021E030E0009711F420E030E04695AF
:10BA0000469546957901E40EF11CC70102960E9405
:10BA10005146009709F453C00E94F145FC01D8013A
:10BA200012968C911297808313968C9181830E9439
:10BA3000F145F2E06F2E712C680E791EC30160E0B3
:10BA400070E0A7010E94D17BF801C480D58000E09E
:10BA500010E02E010894411C511C2AC0D6011196F9
:10BA60008C90119799247801E3E0F594E794EA9596
:10BA7000E1F7E60CF71C77E0A72EB12CA022B1224B
:10BA8000883130F00E943047AC01C701B50107C0D2
:10BA90000E941D479A838983C701B501A2019401C1
:10BAA0000E945D5C080D191DE2E0F0E0CE0EDF1E85
:10BAB000D6018C91882391F621E030E002C020E08D
:10BAC00030E0C9010F900F90CF91DF911F910F913E
:10BAD000FF90EF90DF90CF90BF90AF909F908F90AE
:10BAE0007F906F905F904F900895E0918F06F09156
:10BAF000900609950895E0913806F0913906099568
:10BB00000895E0919306F091940609950895E091C7
:10BB10009506F09196060995089580E090E00895C5
:10BB20000895E0911A06F0911B0609950895009773
:10BB300031F0E0911A06F0911B0609950895E09105
:10BB40001C06F0911D060995089580E090E0089587
:10BB50000F931F93DF93CF93CDB7DEB7E0970FB668
:10BB6000F894DEBF0FBECDBF0E943B468C010E9401
:10BB7000E945602FAE014F5F5F4F0E94DB65882370
:10BB800009F445C088A99801281B3109C9010E9400
:10BB9000C5450097E1F12E81222371F18A859B85AD
:10BBA0003BEA8D3C930721F03FEF8F3F930779F5F8
:10BBB000223041F088E090E007C0019722912F3FAA
:10BBC00041F00BC082E090E0FE01E80FF91F3C96C7
:10BBD000F4CF181619068CF30FC089E1BE01645F1B
:10BBE0007F4F0E94264789E10E94304767EB74E24D
:10BBF0000E94EE3C009759F088E1BE016A5E7F4FDB
:10BC00000E942647E0917806F09179060995E09622
:10BC10000FB6F894DEBF0FBECDBFCF91DF911F915D
:10BC20000F910895AF92BF92CF92DF92EF92FF9261
:10BC30000F931F93DF93CF93CDB7DEB7E0970FB687
:10BC4000F894DEBF0FBECDBF6C018B01FE013196B3
:10BC500080E3DF011D928A95E9F781E089838CE01A
:10BC60000E941D478C831D821F828091001189874D
:10BC70008F5F8093001183E0E82EE8868DEC9BEACD
:10BC80009B878A8789E10E94304762E575E00E94C0
:10BC9000EE3C009731F082E08E838FEF8C878D87AA
:10BCA00009C089E10E943047BC01CE010C960E9478
:10BCB000E53CEE828DEC9BEA9D8B8C8BCE0146960B
:10BCC00067EB74E20E94E53C0E94E9459FA78EA7BE
:10BCD0000E943B4688AB7E010894E11CF11CC70121
:10BCE0000E94D264A82E90E00E945146009741F134
:10BCF0000E94F145BC01C7014A2D0E94F064A0904A
:10BD00001006B09011060E94F1457C010E94454644
:10BD1000BC01C701F5010995C114D10489F0009750
:10BD200021F08130910561F404C0C80160E070E049
:10BD300003C0C80164E070E041E050E0F6010995FD
:10BD4000E0960FB6F894DEBF0FBECDBFCF91DF9166
:10BD50001F910F91FF90EF90DF90CF90BF90AF9029
:10BD600008950E94126080930011E0911A06F091EC
:10BD70001B0609950895EF92FF92CF93DF93E82E6B
:10BD8000E7017E01F92EE70104C060E070E00E9447
:10BD9000533F899199910097C1F7DF91CF91FF901F
:10BDA000EF900895EF92FF92CF93DF93E82EE70193
:10BDB0007E01F92EE70102C00E94983E8991999177
:10BDC0000097D1F7DF91CF91FF90EF900895CF9337
:10BDD000DF93EC017B836A830E94A44F998388835D
:10BDE000DF91CF910895FC0180819181228133817F
:10BDF000820F931F918380830895CF93DF93EC018B
:10BE00000E94A44F99838883DF91CF910895CF93A7
:10BE1000DF93EC010E94A44F28813981821B930B90
:10BE2000019621E030E04A815B814817590710F004
:10BE300020E030E0C901DF91CF910895EF92FF92A9
:10BE4000CF93DF93FC01C281D38180819181C80FA0
:10BE5000D91F0E94A44FC81BD90BCE01DF91CF91EF
:10BE6000FF90EF900895CF93DF93E0E3F7E2C2EF06
:10BE7000D6E2A4E2B7E211921192199219921992A4
:10BE800019921D9287E2E834F807A9F7DF91CF9164
:10BE900008950F931F93CF93DF93FC01DC01AC5DFA
:10BEA000B84D8C91882339F1009194001091950040
:10BEB000EF01CC0FDD1FCC0FDD1FCE50D94DDF01C0
:10BEC000AA0FBB1FA05DB84D8D919C911197980151
:10BED000281B390B40E050E0688179818A819B8181
:10BEE000260F371F481F591F288339834A835B83D6
:10BEF00011961C930E93EE0FFF1FEE0FFF1FEE50D7
:10BF0000F94D6081718182819381DF91CF911F9181
:10BF10000F91089560E070E0CB010895FC01EE0FF1
:10BF2000FF1FEE0FFF1FEE50F94D408351836283D8
:10BF300073830895EF92FF920F931F93CF93DF9334
:10BF400024E237E2C2EFD6E2E0E3F7E2D9018D91D5
:10BF50009D018823C9F04091940050919500808103
:10BF600091817A01E81AF90A00E010E0888199814C
:10BF7000AA81BB818E0D9F1DA01FB11F888399834D
:10BF8000AA83BB835183408324963296B7E2203341
:10BF90003B07E1F6DF91CF911F910F91FF90EF905A
:10BFA00008950E944F6408950F931F93FC01CB01E5
:10BFB0004091011150910211338322831583048330
:10BFC00071836083F0930211E093011141155105D3
:10BFD00011F40E94696480E090E01F910F91089530
:10BFE00080910111909102110097C1F010920211FD
:10BFF00010920111DC0114966D917C9115971296A7
:10C00000ED91FC9113970995E0910111F0910211C6
:10C01000309721F0808191810E94696408950E9487
:10C020009D7908950E949879089589E996E00E9483
:10C030008C3F81EA96E00E948C3F0895EF92FF9238
:10C04000CF93DF930E94F8450097C9F081EA96E00C
:10C050000E94AC3FE82EE7017E01F92EE701209710
:10C0600031F10E943B46998388830E9436469B8328
:10C070008A83C70104960E9464458CAB18C089E985
:10C0800096E00E94AC3FEC017E01F92EE70120977B
:10C0900071F0C70102960E947B4599838883B7019E
:10C0A0006E547F4FC7018E579F4F0E94E846CE01C6
:10C0B000DF91CF91FF90EF900895BC016E547F4FB8
:10C0C0008E579F4F0E94E8460895CF93DF93EC016F
:10C0D00089E996E0BE010E94F73F009719F089E9CF
:10C0E00096E009C081EA96E0BE010E94F73F009702
:10C0F00029F081EA96E0BE010E94D23FDF91CF9104
:10C100000895EF92FF92CF93DF93EC0189E996E0D7
:10C11000BE010E94F73F009779F068817981CE01D6
:10C1200002960E94B546BE016E547F4FCE018E57D7
:10C130009F4F0E94FD461BC081EA96E0BE010E940F
:10C14000F73F0097A1F00E948C46688179818A812F
:10C150009B810E94B5468CA990E00E9451460E94A6
:10C16000F1454CA92496BE0150E00E94C87BDF91A6
:10C17000CF91FF90EF900895EF92FF92CF93DF93CE
:10C18000EC0189E996E0BE010E94F73F009711F0AB
:10C1900022960DC081EA96E0BE010E94F73F00970B
:10C1A00021F00A80DB81C02D02C0C0E0D0E0CE01CA
:10C1B000DF91CF91FF90EF900895FC0180819181F4
:10C1C000089570E06F5B7F4F660F771F680F791FD0
:10C1D000CB010895E62FF0E0EF5BFF4FEE0FFF1F5E
:10C1E000E80FF91F808191810895089589E597E10D
:10C1F0000E940242009721F089E597E10E94ED41FB
:10C200000895E0916617F0916717309711F009953E
:10C21000089580E00895EF92FF920F931F93CF93BC
:10C22000DF93EC018A0188819981009731F023E046
:10C230008C30920709F006C12BC080E00BC0E82FBC
:10C24000F0E0EE0FFF1FEE0FFF1FE95BF84E1182CB
:10C2500010828F5F843098F3809361178091880EED
:10C260009091890E90935817809357170E94913E92
:10C270008093482789E597E160E470E00E94D74108
:10C280000E946A678CE093E09983888381E0DDC037
:10C29000623009F4B9C0633030F4662309F489C010
:10C2A000613081F79CC0673819F0683859F741C090
:10C2B0001092621747E4E42E47E1F42E18C0F7010C
:10C2C000828193818017910749F4808191810E9436
:10C2D000B168F701118210821382128284E090E02B
:10C2E000E80EF91E809162178F5F8093621780912C
:10C2F0006217843020F3E8E5FCE2848D958D801789
:10C30000910719F4158E148E118EB0969CE2E83DBB
:10C31000F90799F7EEEEFCE2818592858017910787
:10C3200011F4158214823D962DE2E037F207A1F751
:10C33000A9CF87E14935580709F0A4CFCA010E9467
:10C340000242009709F49ECF109262172DC0F0E0D0
:10C3500035E0EE0FFF1F3A95E1F7E85AF34D818D76
:10C360008823E9F089E597E10E94ED418091621709
:10C3700090E025E0880F991F2A95E1F7885A934DA0
:10C380009093572C8093562C82E00E94E568809110
:10C39000492790914A27009711F00E9401618091EE
:10C3A00062178F5F80936217E0916217E43078F232
:10C3B00069CF4115510509F465CF5093572C40932F
:10C3C000562C83E00E94E5688091492790914A2786
:10C3D000009711F00E9401610E94F66053CF411551
:10C3E000510509F44FCF5093532C4093522C85E0C4
:10C3F0000E94E5688091492790914A27009709F4A7
:10C4000041CF0E9401613ECF8091492790914A27F8
:10C41000009709F437CF80915A27863031F4809104
:10C42000722781FF02C00E94F66081E00E94E568E9
:10C430008091492790914A27009709F423CF0E94C1
:10C44000346320CF1982188283E0DF91CF911F914E
:10C450000F91FF90EF900895909367178093661760
:10C4600008952091880E3091890E60E0E7E4F7E1AD
:10C4700013C0408151814817590761F442815381AB
:10C480004217530739F460936517118210820E9496
:10C49000B168089534966F5F643058F36093651700
:10C4A000089540E0E7E4F7E116C0542F5F5F208174
:10C4B00031812115310569F440936417918380839C
:10C4C0002091880E3091890E338322830E94CB689D
:10C4D00008953496452F443040F3409364170895EF
:10C4E000FC018091880E9091890E958F848F778FB3
:10C4F000668F0895FC018091880E9091890E928735
:10C500008187748763870895CF93DF93EA010E9440
:10C510002D68FC01009741F08091880E9091890E62
:10C5200092878187D487C387CF01DF91CF91089508
:10C530000F931F93DF93CF9300D000D0CDB7DEB71A
:10C540008C01AB018FEF89838A838B838C83CE012F
:10C550000196B8010E948462FC01009711F01583D6
:10C560000483CF010F900F900F900F90CF91DF9128
:10C570001F910F91089586EB96E062E040E050E055
:10C580000E94443F10924A27109249270895AC0117
:10C5900086EB96E061E00E94213F0895AC0186EBB6
:10C5A00096E060E00E94213F08950F931F93CF9380
:10C5B000DF93EA010E94A3678C01009761F08091EC
:10C5C000880E9091890EF801958F848FD78FC68F32
:10C5D000C8010E94CE62C801DF91CF911F910F91D7
:10C5E0000895CF93DF93A091562CB091572C1097BC
:10C5F00019F0ED016C9605C0C091522CD091532CCE
:10C6000029968091512C86FF22C01092631740E03A
:10C61000E7E4F7E116C02081318114968D919C9159
:10C6200015972817390759F482819381009739F0BB
:10C6300040936317998388831B821A8206C03496BD
:10C640004F5F443040F3409363170E94F660888147
:10C650009981009731F04A815B81609148270E945F
:10C66000443FDF91CF9108950F931F93CF93DF93B2
:10C6700080915A27863009F074C0809149279091A3
:10C680004A2725E08030920709F06BC0C4E9D2E068
:10C69000D0934A27C093492702E00093532714E917
:10C6A0001093542710927627109275270E94626784
:10C6B00080959095909376278093752710925C27AC
:10C6C00010925B270E9451678095909590935C270C
:10C6D00080935B270E940161D0934A27C09349272A
:10C6E00000935327109354279091542C8091552CEC
:10C6F000E92FF82FDF01A459BD4F8CE692E00D9091
:10C7000001920197E1F789E697E26CE672E00E94F8
:10C71000F56680914D278093692780914E278093FD
:10C720006A2780914F2780936B27809150278093B1
:10C730006C2710927627109275270E946267809569
:10C740009095909376278093752710925C2710928E
:10C750005B270E9451678095909590935C2780930A
:10C760005B270E940161DF91CF911F910F91089586
:10C77000282F392FF90120E030E080E0A8E112C035
:10C78000419198E0542F5827B52FB17050FD8A275A
:10C790008695B13009F48068915011F04695F2CF3A
:10C7A0002F5F3F4F2617370759F708951F920F92B3
:10C7B0000FB60F920BB60F9211242F933F934F9306
:10C7C0005F936F937F938F939F93AF93BF93EF93F9
:10C7D000FF938091940090919500909335278093DA
:10C7E000342781E08093262780917100807D80939B
:10C7F00071000E94F05F809126278823E9F18091E3
:10C80000940090919500209134273091352782171C
:10C810009307A0F48091FA269091FB26A091FC2624
:10C82000B091FD268C57914EAF4FBF4F8093FA26A3
:10C830009093FB26A093FC26B093FD268091940054
:10C8400090919500821B930BA0E0B0E02091FA2616
:10C850003091FB264091FC265091FD26820F931FBC
:10C86000A41FB51F8093FA269093FB26A093FC2665
:10C87000B093FD2610922627FF91EF91BF91AF91C3
:10C880009F918F917F916F915F914F913F912F91E8
:10C890000F900BBE0F900FBE0F901F9018959FB773
:10C8A000F894E1E7F0E08081807D808388B38F6237
:10C8B00088BB10929000E1E9F0E0108210929200A3
:10C8C00010929500109294008081856080839FBFB4
:10C8D00008952FB7F894909399008093980088B3A7
:10C8E0008F6288BBE1E7F0E08081826080832FBFA8
:10C8F0000895EF92FF92CF93DF93FC01DB0185E077
:10C90000EB0119928A95E9F7858190E08370907028
:10C91000009711F082E08C93878190E08370907093
:10C92000009721F082E012968C931297858190E017
:10C9300083709070009799F0878190E08370907079
:10C94000009769F0238934898185928528173907F2
:10C9500031F481E0848312961C92129701C01482F4
:10C96000858183708250823030F4C82FD0E0C0546B
:10C97000D94F888101C080E011968C931197E7818F
:10C98000E370E250E23028F4F0E0E054F94F8081A7
:10C9900001C080E013968C931397DF91CF91FF90A5
:10C9A000EF900895DF93CF9300D000D00F92CDB7D2
:10C9B000DEB7BE016F5F7F4F0E94796489819A81E3
:10C9C000890F8D5F9B81890F9C81890F9D81890FC4
:10C9D0000F900F900F900F900F90CF91DF910895CF
:10C9E000AF92BF92CF92DF92EF92FF920F931F937D
:10C9F000DF93CF9300D000D000D0CDB7DEB78C014D
:10CA00007B01BE016F5F7F4F4E830E947964C980B6
:10CA10009A81A92EBB24DB808C81682F70E0950160
:10CA20002C0D311D2D5F3F4F2D0D311D260F371F52
:10CA30005D81250F311D4E8150E0421753070CF4E4
:10CA4000A8C0D80111964C91119750E041705070D8
:10CA5000E3E0440F551FEA95E1F712962C911297E7
:10CA600030E02170307054E0220F331F5A95E1F707
:10CA7000242B3C913770232B13963C911397E32F73
:10CA8000F0E0E170F07045E0EE0FFF1F4A95E1F72E
:10CA90002E2B14963C911497E32FF0E0E170F07088
:10CAA00036E0EE0FFF1F3A95E1F72E2BF7012083BA
:10CAB00015964C91159750E043705070440F551FD8
:10CAC000440F551F16962C91169730E02370307046
:10CAD00054E0220F331F5A95E1F7242B17963C910F
:10CAE00017973295330F330F307C322B31831896E2
:10CAF0002C9118972283FC2DF23069F419962C9111
:10CB0000D70113962C931397F801228514962C9332
:10CB1000149745E001C043E0E92FF0E03B96E00FB9
:10CB2000F11F542F0AC09701250F311DC290D90162
:10CB3000CC925F5F0894A108B108A114B10499F7E1
:10CB4000940FBD2DB23089F4F701E90FF11DD80122
:10CB500053962C91539720839F5FF701E90FF11DA6
:10CB600054962C91549720839F5FE82FF0E07596A0
:10CB7000E00FF11F292F08C0D701A20FB11D32917C
:10CB80003C932F5F6150704061157105A9F7890FC3
:10CB900001C080E026960FB6F894DEBF0FBECDBF71
:10CBA000CF91DF911F910F91FF90EF90DF90CF9089
:10CBB000BF90AF900895BF92CF92DF92EF92FF9215
:10CBC0000F931F93CF93DF937C01D62EEA0163303E
:10CBD00008F4ADC0FC018081B82EB294B694B6942E
:10CBE000B3E0BB22F1E0BF22F7019181292F269506
:10CBF00026952370C92EC294C694C694A3E0CA2277
:10CC0000382F37703883382F3695369536953170F2
:10CC10003983382F329531703A83829586958170A9
:10CC20008B83BC822D83892F829583708E83CF82E4
:10CC30008281888787010D5F1F4F222361F1F801F0
:10CC4000918180E0F7013381830F911D9A87898755
:10CC500087010B5F1F4F223081F4CA010B9662E5FA
:10CC600075E00E94E53CF80181818B87F7018581A1
:10CC70008C878701095F1F4F16C02330A1F4F7018D
:10CC80003D96DA011B9682918D93E017F107D9F753
:10CC9000085F1F4F08C0CA010B9662E575E00E944D
:10CCA000E53C1A861986CC2089F1BB2059F4F8019D
:10CCB000918180E02081820F911D9C8B8B8B0E5F78
:10CCC0001F4F04C089859A859C8B8B8BFC2DF2307D
:10CCD00071F4CE01459662E575E00E94E53CF801ED
:10CCE00081818D8B80818E8B0E5F1F4F17C0FC2D35
:10CCF000F330A1F4085F1F4FD801FE01759680E064
:10CD00009E9191938F5F8830D9F708C0CE014596E8
:10CD100062E575E00E94E53C1C8A1B8A802F8E1913
:10CD20009D2D981B9FA71EA70DA7D81608F480E07D
:10CD3000DF91CF911F910F91FF90EF90DF90CF90F7
:10CD4000BF9008959C0141505040460F571FDB0192
:10CD500010C0FC91E0E011968C911197BF01680F13
:10CD6000711D260F371F2617370710F42F5F3F4F0F
:10CD70001296A417B50768F3A417B50749F49C9158
:10CD800080E0280F391F2817390710F42F5F3F4F15
:10CD9000C9010895CF93DF9390915427C92FD0E014
:10CDA00064973091532720E0C20FD31F9E01280FB4
:10CDB000311DC9016DE577E248E050E00E94A266AE
:10CDC00065E677E2AE010E94A266009719F0382F5F
:10CDD000292F02C02FEF3FEFC901DF91CF910895B6
:10CDE00090937717809376170895FC014381460F3F
:10CDF00040935027872F99272281280F20934F2770
:10CE0000A181A0934E27508150934D2730E02817E1
:10CE1000390748F48A2F8F5F80934E27882319F4AF
:10CE20005F5F50934D27842F90E0707086179707AF
:10CE300098F480914F278F5F80934F27882361F468
:10CE400080914E278F5F80934E27882329F480910D
:10CE50004D278F5F80934D270895BC018091562CFC
:10CE60009091572C08960E94F566E091562CF0910F
:10CE7000572C80914D27808780914E278187809104
:10CE80004F27828780915027838708959C01AB01AB
:10CE900080E090E0B9010E94A266382F292FC901D5
:10CEA000089580E090E061E577E244E150E00E947F
:10CEB000A266009719F0382F292F02C02FEF3FEFFD
:10CEC000C901089586E00E94CA66089581E10E9422
:10CED000CA66089580E009C0E82FF0E0EE0FFF1F5A
:10CEE000E852F34D118210828F5F8430A8F380E006
:10CEF0000BC0E82FF0E095E0EE0FFF1F9A95E1F7E9
:10CF0000E85AF34D118E8F5F843098F380E094E0FF
:10CF1000909379178093781740E08DE090E00EC0F1
:10CF2000242F30E0289FF001299FF00D389FF00D4D
:10CF30001124E251F34D158214824F5F4A3080F381
:10CF400040937417089520917817309179172F5FC7
:10CF50003F4F4DE72030340710F020E030E1522FF2
:10CF6000432FA0E013C0EA2FF0E0B5E0EE0FFF1F63
:10CF7000BA95E1F7E85AF34DB18DBB2331F0048047
:10CF8000F581E02DE417F50711F3AF5FA43059F7F1
:10CF900030937917209378171092741720E0E0E00F
:10CFA000F0E01EC0A22FB0E035E0AA0FBB1F3A95FB
:10CFB000E1F7A85AB34D59963C915997332321F480
:10CFC00020937417FD0110C0373049F4309731F0C9
:10CFD0005A964C915A97328D341708F4FD012F5F01
:10CFE000243000F3209374173097A9F122E0218FA9
:10CFF00020916E17248720916F1725872091701735
:10D00000268720917117278728ED34E0338B228BF8
:10D01000358B248B21E030E0318B208B138E21E087
:10D02000228F23E0208F168A20E1278B209178170A
:10D03000309179173227232732273583248377834A
:10D040006683DC012D913D914D915C911397208376
:10D05000318342835383CF0108950F931F93CF935E
:10D06000DF9320917817309179174DE050E02F5FD2
:10D070003F4FADE720303A0710F020E030E1B22F0B
:10D08000A32F10E012C0C12FD0E0C49FF001C59FB4
:10D09000F00DD49FF00D1124E251F34D0480F58181
:10D0A000E02DEA17FB0719F31F5F1A3061F7309381
:10D0B00079172093781710E02DE030E01AC0012F87
:10D0C0000F5FC12FD0E0C29FF001C39FF00DD29F30
:10D0D000F00D1124E251F34DDF0114964481558186
:10D0E0004115510529F410937417309749F433C052
:10D0F000102F1A3020F310937417E0E0F0E02BC0EB
:10D1000020917817309179173227232732271196EB
:10D110003C932E9377836683009729F410821182C3
:10D120001282138209C0DC012D913D914D915C91D9
:10D1300020833183428353838DE090E0C89FD001E8
:10D14000C99FB00DD89FB00D1124A251B34D80E4FA
:10D1500018968C931897CF01DF91CF911F910F9163
:10D16000089540E013C0E42FF0E0542F5F5FEE0F0E
:10D17000FF1FE852F34D208131812817390729F428
:10D1800040937417118210820895452F443058F34C
:10D1900040937417089540E013C0E42FF0E0542F3B
:10D1A0005F5FEE0FFF1FE852F34D208131812115A3
:10D1B000310529F440937417918380830895452F96
:10D1C000443058F3409374170895EF92FF920F93F1
:10D1D0001F93CF93DF93C091562CD091572C84305E
:10D1E00009F4F7C109E717E21093552C0093542C6A
:10D1F00010934C2700934B27833071F4898D90E076
:10D200008F7090708330910509F074C08889998976
:10D21000009709F02FC78DC0823009F08EC0809131
:10D2200071178F5F80937117882399F4809170171D
:10D230008F5F80937017882361F480916F178F5FE1
:10D2400080936F17882329F480916E178F5F8093E6
:10D250006E1710924A27109249271092ED2C1092C7
:10D26000EC2C898D873011F0853041F48A8D8F5FE9
:10D270008A8F843109F0FEC6198EFCC6882309F412
:10D28000F9C6288939892115310509F44EC09A8DCE
:10D29000292F21502A8F992309F0ECC69B8D9830B5
:10D2A00031F0282F2150223048F4953039F4198E6E
:10D2B00080E88093512C0E94F16295C5953048F426
:10D2C00023E030E0092E02C0220F331F0A94E2F758
:10D2D00001C020E32A8F9F5F9B8F90E08F7090703A
:10D2E00083309105E1F0843091054CF48130910553
:10D2F00009F461C38230910509F0BCC60DC08630C7
:10D30000910509F40CC58830910509F408C58430ED
:10D31000910509F0AFC603C5109272274FC384E090
:10D320008093512C0E94F16290C58F70833009F078
:10D33000A1C688E08093512C4BC5853019F5E0914A
:10D34000522CF091532C84819581009709F492C658
:10D350001092572C1092562C0C5010401093552CB4
:10D360000093542C10934C2700934B271092ED2CD4
:10D370001092EC2C10924A271092492788E0809353
:10D38000512C25C10852104080915127853409F055
:10D3900071C69091532780E0209154277C01E20EC2
:10D3A000F11C8091492790914A278E159F0508F41A
:10D3B00061C6F0924A27E09249278091572790E072
:10D3C0008F739070009709F055C680915827882375
:10D3D00009F050C68091E82C9091E92CC091C606C6
:10D3E000D091C7068C179D0759F44091EA2C5091B3
:10D3F000EB2C2091C8063091C90642175307A1F0C3
:10D4000020916127309162272817390709F032C629
:10D4100020916327309164278091EA2C9091EB2C26
:10D420002817390709F026C60E9451672FEF8F3F52
:10D43000920709F01FC680915A27863009F431C13E
:10D440008131E9F1813009F015C680916527883076
:10D4500009F010C610926527809167279091682780
:10D460004FEF873F940710F0099601C008969093FC
:10D4700068278093672780915D2790915E27A09110
:10D480005F27B09160278093612790936227A093D4
:10D490006327B09364278091E82C9091E92CA091A8
:10D4A000EA2CB091EB2C80935D2790935E27A0939C
:10D4B0005F27B093602780E4F8018087B8C5C70173
:10D4C0004C9790934A27809349278DE697E2909353
:10D4D000552C8093542C80916B2790916C2700974A
:10D4E00039F00E946667FFEF8F3F9F0709F0C2C5C2
:10D4F00020916727309168272115310509F4BAC5B5
:10D500008EEE9CE29093532C8093522C6091C8062F
:10D510007091C9064091C2065091C3060091C4069D
:10D520001091C50639C084819581009781F1281733
:10D53000390769F586819781009739F0A0916527B1
:10D54000B0916627A817B90711F5808191818C17D2
:10D550009D0729F4A281B381A617B70739F1841773
:10D56000950729F4A281B381A017B107F9F0A09122
:10D570005D27B0915E27A817B90749F4A0915F27EE
:10D58000B091602782819381A817B90779F03D9601
:10D59000F093532CE093522CE091522CF091532CA9
:10D5A0008DE2E037F80708F4BECF64C51092572C1F
:10D5B0001092562C82E08093512C8DE697E2909346
:10D5C0004C2780934B271092ED2C1092EC2C0E944C
:10D5D000F1628091EC2C9091ED2C009709F44AC5F2
:10D5E0009C01245E3F4F30934A2720934927309374
:10D5F000532720935427E091522CF091532C2085EF
:10D600002093592721E120935A27089698278927A4
:10D61000982790936A278093692710926C2710921D
:10D620006B278481958190936627809365278681F7
:10D63000978190936827809367278091E82C909139
:10D64000E92CA091EA2CB091EB2C80935D2790936C
:10D650005E27A0935F27B093602780819181A2818C
:10D66000B3818093612790936227A0936327B0933F
:10D67000642789E797E29093552C8093542C0E945D
:10D6800066678095909590936C2780936B270097A1
:10D6900009F0CDC48FEF9FEF90936C2780936B2799
:10D6A000C6C40E946267EFEF8F3F9E0709F0E2C495
:10D6B0008091672790916827009709F4DBC4209137
:10D6C0006527309166272115310509F4D3C4C8E5D3
:10D6D000DCE2498D4423E9F06C817D818617970750
:10D6E000C1F46E817F812617370799F4E0915D2799
:10D6F000F0915E2768817981E617F70751F4E09190
:10D700005F27F09160276A817B81E617F70709F4AC
:10D710006DC1A096FCE2C83DDF07D9F620917227C3
:10D720002F732230B9F4909373178093721740E0EF
:10D730000DC0E42FF0E0EE0FFF1FE852F34D208103
:10D7400031814F5F8217930709F46EC0443088F32C
:10D75000409374178091722782FD8CC484E1F80194
:10D7600081A388E290E090934A278093492780E53F
:10D7700080A380916C2790917027938F30916B27B5
:10D7800090916F27928F368F20916A2790916E2704
:10D79000918F258F909169279093741740916D27F1
:10D7A000408F948F8F5F878F882361F4832F8F5FE3
:10D7B000868F882339F4822F8F5F858F882311F419
:10D7C0009F5F948F80916527909166279093731740
:10D7D000809372172091672730916827F801358B65
:10D7E000248B978B868B80915D2790915E27A091EB
:10D7F0005F27B09160278093612790936227A09361
:10D800006327B09364278091E82C9091E92CA09134
:10D81000EA2CB091EB2C80935D2790935E27A09328
:10D820005F27B0936027E8C31092741780E0C0E0D0
:10D83000D0E022C0E82FF0E075E0EE0FFF1F7A95F0
:10D84000E1F7E85AF34D918D992321F480937417F1
:10D85000EF0116C0973079F4209721F0228D9A8D30
:10D86000921748F4C82FD0E065E0CC0FDD1F6A9511
:10D87000E1F7C85AD34D8F5F8430E0F2809374177C
:10D88000209709F4F7C3D093572CC093562C83E00C
:10D890008A8F888F1E8A84E08F8B1B8E80916727EA
:10D8A000909168279D838C8380916527909166274E
:10D8B0009F838E8380915D2790915E27A0915F2743
:10D8C000B091602788839983AA83BB8381E0898F85
:10D8D00080916E178C8780916F178D87809170175C
:10D8E0008E87809171178F8781E090E0998B888B6C
:10D8F00080916C278B8780916B278A8780916A271C
:10D90000898780916927888781E090E00E942D6750
:10D9100080917127282F30E0207F3070213531052C
:10D920000CF449C082958F7090E00597880F991F7D
:10D93000880F991F5091751740E034C0F901EF5AD4
:10D94000F84D50A5552329F440937417109275177C
:10D9500032C0513011F44F5F25C05230E1F461A55F
:10D960006430C9F4409374175093751732A520E0C2
:10D9700083A590E0822B932B90937317809372175B
:10D98000F4E0893D9F0710F088ED94E09B8B8A8B33
:10D990009D8B8C8B10C02F5A384DF90121A5222365
:10D9A00031F0420F242F30E0281739073CF2409322
:10D9B00074175093751780E18093722780917227B6
:10D9C00082608093722782E08093792784E080933D
:10D9D0007A2780937B2788ED80937C278CE290E0E8
:10D9E00090934A278093492780E6B3C2D093572C5F
:10D9F000C093562C1092512C8091722790E082FF98
:10DA000003C0198E80E24EC22091712722952F709B
:10DA1000220F220F20937417B701621B71099B011B
:10DA20002451304030934A272093492750E04F70CB
:10DA300050704230510539F4AC014F73507042318F
:10DA4000510551F42AC04130510531F4AC014F73F6
:10DA500050704230510509F12115310531F49C0116
:10DA60002370307021153105C1F030916927288568
:10DA7000321709F064C230916A272985321709F0FC
:10DA80005EC230916B272A85321709F058C2309157
:10DA90006C272B85321709F052C284FF4AC068896F
:10DAA00079896115710509F444C0CE010C960E9474
:10DAB000F56630916D2780914D273817D1F520916B
:10DAC0006E2780914E272817A1F590916F2780919E
:10DAD0004F27981771F58091702740915027841730
:10DAE00041F53C872D879E878F878B8D8823D1F4C6
:10DAF0002E89888D9A8D891B922F9695969596954D
:10DB0000891B280F2E8B87FD81959F89392F36958C
:10DB10003695931B980F9F8B822F869586958695B9
:10DB2000890F888F81E08093512C888D8A8F198A84
:10DB3000188A298D30E0C9018F709070843091056A
:10DB400009F4B5C18530910564F482309105C9F1BD
:10DB5000833091050CF0B9C08130910509F08AC27B
:10DB600011C08630910509F4E2C1863091050CF4AC
:10DB7000BEC18730910509F4E2C18830910509F0F2
:10DB800079C28AC18091512C80FF14C083E0898FB3
:10DB900080E48093512C198A188A809149279091AA
:10DBA0004A27009709F410C122E42093512C0E94C7
:10DBB0002D670AC1809172278F73823009F05AC293
:10DBC000FACE8091512C80FF75C0809172278F739F
:10DBD000823109F06FC080917127282F30E0207FBB
:10DBE0003070213531050CF449C082958F7090E07A
:10DBF0000597880F991F880F991F5091751740E05E
:10DC000034C0F901EF5AF84D50A5552329F440933B
:10DC100074171092751732C0513011F44F5F25C040
:10DC20005230E1F461A56430C9F440937417509305
:10DC3000751732A520E083A590E0822B932B90935B
:10DC400073178093721774E0893D970710F088ED81
:10DC500094E09B8B8A8B9D8B8C8B10C02F5A384DF8
:10DC6000F90121A5222331F0420F242F30E028179B
:10DC700039073CF2409374175093751783E0898FEE
:10DC800080916927888780916A27898780916B278F
:10DC90008A8780916C278B8781E090E00E942D67B6
:10DCA00082E48093512C198A188A10924A27109284
:10DCB00049278AC080E28093512C0E94F162E09152
:10DCC000562CF091572C118E45CD8091722780FFF4
:10DCD0002AC024FD28C088899989009709F0CAC103
:10DCE0008091492790914A2701960E942D672091A3
:10DCF000512C822F80618093512C809149279091E3
:10DD00004A27009719F022612093512C0E94F1625A
:10DD100081E090E0998B888B88E0898F1B8E81E170
:10DD2000809372270FC185FF1CC05091772740E078
:10DD30008091782790E0842B952B4091542C509122
:10DD4000552C480F591F5093552C4093542C4091FB
:10DD5000492750914A27481B590B50934A27409313
:10DD600049278091492790914A27009749F024FD3F
:10DD700007C02091512C22602093512C0E942D67C6
:10DD80009091732780E020917427820F911D9093CA
:10DD90007317809372172C893D892817390710F063
:10DDA000009721F4309373172093721780917217A4
:10DDB000909173179B8B8A8B8091512C90E083708C
:10DDC0009070009709F456C11092ED2C1092EC2C33
:10DDD0000E94F1628091512C85FF07C01092ED2CBA
:10DDE0001092EC2C198E84E19BCF84FF0AC0109214
:10DDF000ED2C1092EC2C81E090E0998B888B84E0E4
:10DE00008CCF2091EC2C3091ED2C21153105E1F0D7
:10DE100080FF02C0198A188A88899989009781F43D
:10DE20008A899B898217930720F49093ED2C809325
:10DE3000EC2C8091EC2C9091ED2C998B888B04C06C
:10DE40009093ED2C8093EC2C1B8E80914B2790911E
:10DE50004C279093552C8093542C8091EC2C9091CE
:10DE6000ED2C009759F088899989009739F08896A8
:10DE700090934A278093492788E10BC08091512CC9
:10DE800081FFF8C088E290E090934A278093492769
:10DE900080E1809372275CC08091512C80FFEAC0A2
:10DEA000198E80E18093512C0E94F162E3C0809131
:10DEB000492790914A27009711F00E942D67909171
:10DEC00072278091512C90FF0BC080FF06C087E025
:10DED000898F1A8E198A188A19C086E0898F16C010
:10DEE00080FF1EC085E0898F198A188AC3C080917F
:10DEF000492790914A27009711F00E942D67809141
:10DF0000722780FF0DC087E0898F1A8E81E090E034
:10DF10000E942D6780E18093512C0E94F1620FC016
:10DF20008091492790914A27009749F4A3C0809196
:10DF3000512C80FF9FC087E0898F1A8E9BC080E1A3
:10DF4000F80181A388E290E090934A2780934927C3
:10DF500080E580937127888580936D2789858093DC
:10DF60006E278A8580936F278B85809370278C8599
:10DF7000809369278D8580936A278E8580936B2790
:10DF80008F8580936C2786E080935A278C819D81B2
:10DF900090936627809365278E819F819093682751
:10DFA000809367278091E82C9091E92CA091EA2C2E
:10DFB000B091EB2C80935D2790935E27A0935F2711
:10DFC000B093602788819981AA81BB818093612762
:10DFD00090936227A0936327B0936427898D84FF71
:10DFE00005C0109274271092732706C084E08093B6
:10DFF000732788ED8093742780E48093592780915C
:10E00000492790914A279093532780935427109241
:10E0100078271092772710927627109275270E9402
:10E02000626780959095909376278093752785E415
:10E0300080935127109252271092582710925727F9
:10E040008091761790917717019690937717809328
:10E050007617909355278093562710925C2710923D
:10E060005B270E9451678095909590935C278093E1
:10E070005B2704C010924A27109249271092512C16
:10E08000DF91CF911F910F91FF90EF900895382F5E
:10E09000292FC9010895382F292F40E050E0762715
:10E0A0006727762780E090E0CB0177276627262B2D
:10E0B000372B482B592BB901CA010895AC01E091C7
:10E0C0004B27F0914C27222733272E1B3F0B2F5A2B
:10E0D000334D621773070CF49B011216130664F498
:10E0E0002093EC2C3093ED2C4E175F0729F0CF01D5
:10E0F000BA01A9010E94C87B08950F93DF93CF93C3
:10E10000CDB7DEB760970FB6F894DEBF0FBECDBFB8
:10E11000002309F459C029833A834B835C836D83C0
:10E120007E838F839887E0E2E01B29813A814B81CF
:10E130005C811E16BCF019861A861B861C868E2FE3
:10E14000992787FD9095909581959F4F04C0220F48
:10E15000331F441F551F8A95D2F72D873E874F875F
:10E16000588B2AC0CA01B901002E04C0660F771F60
:10E17000881F991F0A94D2F769877A878B879C87B3
:10E18000DA01C90104C0B695A79597958795EA95D8
:10E19000D2F72D813E814F81588504C0220F331F55
:10E1A000441F551F0A95D2F7822B932BA42BB52B16
:10E1B0008D879E87AF87B88B29853A854B855C858F
:10E1C0006D857E858F85988960960FB6F894DEBF41
:10E1D0000FBECDBFCF91DF910F910895A0E1B0E0C8
:10E1E000E4EFF0E70C941B7929833A834B835C833B
:10E1F0006D837E838F839887A986BA86CB86DC86DB
:10E20000ED86FE860F87188B2D813E814F815885C4
:10E210008D859E85AF85B889281739074A075B0722
:10E22000C8F082179307A407B50790F029813A81B7
:10E230004B815C8189859A85AB85BC852817390718
:10E240004A075B0738F082179307A407B50720F445
:10E2500082E003C080E001C081E06096EAE00C94B7
:10E2600037792F923F924F925F926F927F928F9267
:10E270009F92AF92BF92CF92DF92EF92FF920F9355
:10E280001F93DF93CF93CDB7DEB763970FB6F894A4
:10E29000DEBF0FBECDBF6C017F876E87FC0117828A
:10E2A0001682838181FD04C06FC34C855D8504C0E7
:10E2B0001E010894211C311CF6019381EE85FF8517
:10E2C00093FD859193FF8191FF87EE87882309F461
:10E2D00057C3853241F493FD859193FF8191FF8768
:10E2E000EE87853259F490E0B6014A8B5B8B0E9431
:10E2F0001B7C4A895B895D874C87D7CF10E0FF2460
:10E3000000E00032B0F48B3269F08C3228F48032B5
:10E3100051F0833271F40BC08D3239F0803349F4FF
:10E3200001602CC00260046029C0086027C0006141
:10E3300025C007FD2EC0282F20532A3098F406FF51
:10E3400008C0812F880F182F110F110F180F120FEF
:10E3500015C08F2D880FF82EFF0CFF0CF80EF20E53
:10E3600000620CC08E3221F406FD0AC3006406C0B0
:10E370008C3611F4006802C0883659F4EE85FF85AA
:10E3800093FD859193FF8191FF87EE87882309F0A4
:10E39000B8CF982F9554933018F40061805E06C072
:10E3A000982F9556933008F09BC10F7E06FF16E01C
:10E3B0006FE3E62EE022853619F4F0E4EF2A07C079
:10E3C000863619F420E8E22A02C011111150E7FE46
:10E3D00006C01C3340F4912E939427E00BC01830F4
:10E3E00030F4212F06C027E03CE3932E03C027E042
:10E3F00017E09924CA0104969D878C87FA016081F1
:10E40000718182819381A101092D0E94D87A5C01DA
:10E410006980262D30E0398B288B60FE03C0388957
:10E4200033FF06C0E1FC06C0E2FE06C000E205C004
:10E430000DE203C00BE201C000E0888999898C706D
:10E4400090700097C1F1002311F084E001C083E0D7
:10E450008F1558F4F81AE3FC09C080E290E0B60189
:10E460000E941B7CFA94C9F701C0FF24002329F005
:10E47000802F90E0B6010E941B7C888983FD03C039
:10E480000AE81FE00EC006E81FE00BC0A114B104AB
:10E4900009F0805290E0B6010E941B7C0F5F1F4F75
:10E4A00005C0AE2CBB2490E1A922BB24F8018491C5
:10E4B000882361F762C2E7FE0EC09A0CF889F4FF68
:10E4C00004C08A81813309F49A94191454F5292DD2
:10E4D000293050F52DC0E6FC2BC0812F90E08A1525
:10E4E0009B054CF03CEFA3163FEFB30624F080E809
:10E4F000E82A01C01150112349F0E2E0F0E0EC0FEE
:10E50000FD1FE10FF11D80818033A1F3E7FE10C0F4
:10E51000912E9394812F90E0A816B90644F41A190D
:10E5200007C09924939404C098E0992E01C010E08C
:10E53000E7FE07C01A141B043CF495012F5F3F4F00
:10E5400005C025E030E002C021E030E0002311F0FA
:10E550002F5F3F4F112329F0812F90E00196280F64
:10E56000391F8F2D90E02817390714F4F21A01C0D3
:10E57000FF244E2C5524C20189709070009749F4F5
:10E5800006C080E290E0B6010E941B7CFA94FF2056
:10E59000C1F7002329F0802F90E0B6010E941B7C78
:10E5A00043FC09C006C080E390E0B6010E941B7CDA
:10E5B000FA94FF20C1F7E7FE46C03501B7FE02C05E
:10E5C0006624772425010894411C511C46185708DD
:10E5D000420C531CF501E919F1094F01812F90E01C
:10E5E00000271127081B190BFFEF6F16FFEF7F069F
:10E5F00029F48EE290E0B6010E941B7CA614B704B9
:10E6000034F0861497041CF4F201808101C080E389
:10E610000894610871080894411C511C6016710629
:10E620002CF090E0B6010E941B7CDECF6A147B04C4
:10E6300041F49A81963320F4953319F4F889F4FF64
:10E6400081E390E049C08A81813311F02FEE62228C
:10E6500090E0B6010E941B7C112389F08EE290E0CD
:10E66000B6010E941B7C02E0F101E00FF11D0F5F7B
:10E67000808190E0B6010E941B7C1150A9F744FEF6
:10E6800003C085E490E002C085E690E0B6010E94F8
:10E690001B7CB7FC05C0A114B10441F464FE06C0A4
:10E6A000B094A194B108B3948DE201C08BE290E0E4
:10E6B000B6010E941B7C80E305C08F5FE6EFFFEF91
:10E6C000AE0EBF1EFAE0AF16B104BCF790E0B60183
:10E6D0000E941B7CC501C096B6010E941B7C4DC1E7
:10E6E000833631F0833789F0833509F059C022C071
:10E6F0009A012E5F3F4F3D872C87FA0180818983E5
:10E70000310181E0A82EB12C13C09A012E5F3F4F3A
:10E710003D872C87FA016080718006FF03C0612F5E
:10E7200070E002C06FEF7FEFC3010E94E17B5C01EC
:10E730000F7714C09A012E5F3F4F3D872C87FA0157
:10E740006080718006FF03C0612F70E002C06FEF30
:10E750007FEFC3010E94B87B5C01006803FD1CC011
:10E7600006C080E290E0B6010E941B7CFA948F2DD7
:10E7700090E0A816B906A8F30FC0F30107FD859134
:10E7800007FF81913F0190E0B6010E941B7CF110D0
:10E79000FA940894A108B108A114B10471F7EDC06E
:10E7A000843611F0893661F507FF0BC09A012C5FA2
:10E7B0003F4F3D872C87FA0160817181828193816F
:10E7C0000CC09A012E5F3F4F3D872C87FA01608174
:10E7D0007181882777FD8095982F0F7697FF08C065
:10E7E00090958095709561957F4F8F4F9F4F0068F2
:10E7F000A1012AE030E00E942D7D982E921841C0A0
:10E80000853721F40F7E2AE030E020C0097F8F3663
:10E81000A9F0803720F4883509F0B2C00BC08037EA
:10E8200021F0883709F0ACC001C0006104FF09C0C5
:10E83000046007C004FF08C0066006C028E030E09E
:10E8400005C020E130E002C020E132E007FF0AC04D
:10E85000CA0104969D878C87FA016081718182814B
:10E86000938109C0CA0102969D878C87FA01608155
:10E87000718180E090E0A1010E942D7D982E921878
:10E880000F7706FF09C00E7F911630F404FF06C013
:10E8900002FD04C00F7E02C0E92C01C0E12E802FD2
:10E8A00090E004FF0CC0FE01E90DF11D2081203332
:10E8B00011F4097E09C0E39402FF06C004C0867803
:10E8C0009070009709F0E394A02EBB2403FD14C0C0
:10E8D00000FF0FC0EF1428F4192D1F0D1E19EF2C87
:10E8E00008C0192D06C080E290E0B6010E941B7C92
:10E8F000E394EF14C0F304C0EF1410F4FE1801C049
:10E90000FF24A4FE0FC080E390E0B6010E941B7CB0
:10E91000A2FE1FC0A1FE03C088E590E010C088E7FA
:10E9200090E00DC0C50186789070009791F0A1FC31
:10E9300002C080E201C08BE207FD8DE290E0B601EB
:10E940000E941B7C06C080E390E0B6010E941B7C05
:10E9500011509116C0F39A94F101E90DF11D8081D7
:10E9600090E0B6010E941B7C9920A9F706C080E2C6
:10E9700090E0B6010E941B7CFA94FF20C1F795CC71
:10E98000F6012681378102C02FEF3FEFC901639660
:10E990000FB6F894DEBF0FBECDBFCF91DF911F91B0
:10E9A0000F91FF90EF90DF90CF90BF90AF909F902E
:10E9B0008F907F906F905F904F903F902F90089531
:10E9C0005058BB27AA270ED0CBC1BCD130F0C1D143
:10E9D00020F031F49F3F11F41EF48CC10EF4E09549
:10E9E000E7FB82C1E92FCDD180F3BA176207730725
:10E9F0008407950718F071F49EF5E5C10EF4E095D3
:10EA00000B2EBA2FA02D0B01B90190010C01CA01E8
:10EA1000A0011124FF27591B99F0593F50F4503E93
:10EA200068F11A16F040A22F232F342F4427585F85
:10EA3000F3CF469537952795A795F0405395C9F79D
:10EA40007EF41F16BA0B620B730B840BBAF0915055
:10EA5000A1F0FF0FBB1F661F771F881FC2F70EC0F4
:10EA6000BA0F621F731F841F48F4879577956795C7
:10EA7000B795F7959E3F08F0B3CF9395880F08F0B0
:10EA80009927EE0F9795879508955CD158F080E807
:10EA900091E009F49EEF5DD128F040E851E059F48F
:10EAA0005EEF09C027C18FC1E92FE0786AD168F312
:10EAB000092E052AC1F3261737074807590738F0EA
:10EAC0000E2E07F8E02569F0E025E0640AC0EF6348
:10EAD00007F8009407FADB01B9019D01DC01CA01C6
:10EAE000AD01EF9347D03CD10AD05F91552331F06F
:10EAF0002BED3FE049E450FD49EC63CF0895DF93EF
:10EB0000DD27B92FBF7740E85FE3161617064807E1
:10EB10005B0710F4D92F5ED19F938F937F936F93F0
:10EB20000FD2E0E2F1E0E9D01BD12F913F914F915C
:10EB30005F9163D1DD2349F09058A2EA2AED3FE0CE
:10EB400049EC5FE3D0785D274DDFDF9109C1A8D0A4
:10EB500008F481E008950CD003C1FBD040F0F2D05E
:10EB600030F021F45F3F19F0BFC051112DC1C2C078
:10EB700008D198F39923C9F35523B1F3951B550B8D
:10EB8000BB27AA2762177307840738F09F5F5F4F80
:10EB9000220F331F441FAA1FA9F333D00E2E3AF0C1
:10EBA000E0E830D091505040E695001CCAF729D0DB
:10EBB000FE2F27D0660F771F881FBB1F261737072A
:10EBC0004807AB07B0E809F0BB0B802DBF01FF275A
:10EBD00093585F4F2AF09E3F510568F085C0F4C0FE
:10EBE0005F3FECF3983EDCF3869577956795B79594
:10EBF000F7959F5FC9F7880F911D9695879597F9AF
:10EC00000895E1E0660F771F881FBB1F6217730727
:10EC10008407BA0720F0621B730B840BBA0BEE1F3C
:10EC200088F7E0950895E89409C097FB3EF4909525
:10EC30008095709561957F4F8F4F9F4F9923A9F0D5
:10EC4000F92F96E9BB279395F69587957795679564
:10EC5000B795F111F8CFFAF4BB0F11F460FF1BC0A8
:10EC60006F5F7F4F8F4F9F4F16C0882311F096E93B
:10EC700011C0772321F09EE8872F762F05C06623E9
:10EC800071F096E8862F70E060E02AF09A95660FA2
:10EC9000771F881FDAF7880F9695879597F908955B
:10ECA000990F0008550FAA0BE0E8FEEF161617069D
:10ECB000E807F907C0F012161306E407F50798F005
:10ECC000621B730B840B950B39F40A2661F0232B1E
:10ECD000242B252B21F408950A2609F4A140A6959A
:10ECE0008FEF811D811D089597F99F6780E870E07F
:10ECF00060E008959FEF80EC0895DF93CF931F931A
:10ED00000F93FF92EF92DF927B018C01689405C014
:10ED1000DA2EEF0172D0FE01E894A591259135918C
:10ED200045915591AEF3EF015DDEFE019701A8011B
:10ED3000DA9479F7DF90EF90FF900F911F91CF91C8
:10ED4000DF91089500240A9416161706180609067E
:10ED5000089500240A941216130614060506089551
:10ED6000092E0394000C11F4882352F0BB0F40F4D9
:10ED7000BF2B11F460FF04C06F5F7F4F8F4F9F4F19
:10ED8000089557FD9058440F551F59F05F3F71F09B
:10ED90004795880F97FB991F61F09F3F79F0879502
:10EDA0000895121613061406551FF2CF4695F1DF8B
:10EDB00008C0161617061806991FF1CF869571051B
:10EDC000610508940895E894BB2766277727CB014F
:10EDD00097F908959B01AC0160E070E080E89FE343
:10EDE000BACE0BD0BDCFAEDF28F0B3DF18F095233D
:10EDF00009F07ACF7FCF1124E7CFC3DFA0F3959F2F
:10EE0000D1F3950F50E0551F629FF001729FBB2711
:10EE1000F00DB11D639FAA27F00DB11DAA1F649FBD
:10EE20006627B00DA11D661F829F2227B00DA11D70
:10EE3000621F739FB00DA11D621F839FA00D611DF6
:10EE4000221F749F3327A00D611D231F849F600D17
:10EE5000211D822F762F6A2F11249F5750408AF050
:10EE6000E1F088234AF0EE0FFF1FBB1F661F771FDC
:10EE7000881F91505040A9F79E3F510570F034CF44
:10EE8000A3CF5F3FECF3983EDCF3869577956795CB
:10EE9000B795F795E7959F5FC1F7FE2B880F911DFA
:10EEA0009695879597F90895FA01EE0FFF1F309612
:10EEB0002105310599F16115710561F48038BFE3D1
:10EEC0009B0749F168949038810561F08038BFEF65
:10EED0009B0741F0992342F5FF3FE10531052105EC
:10EEE00011F1E8940894E795D901AA2329F4AB2FEE
:10EEF000BE2FF85FD0F310C0FF5F70F4A695E0F767
:10EF0000F73950F019F0FF3A38F49F779F930CD0FF
:10EF10000F9007FC905808953EF0ECCE60E070E052
:10EF200080E89FE308954FE79F775F934F933F9368
:10EF30002F9375D02F913F914F915F9152DF08C071
:10EF40009B01AC014ECF19F40EF0CECE3CCFD2CE09
:10EF500020DFC8F39638C0F707F80F92E8942BE348
:10EF60003AEA48EB5FE74BDF0F920F920F924DB7F3
:10EF70005EB70F9294D0EDE4F1E0BFDE4F915F9168
:10EF8000EF91FF91E595EE1FFF1F49F0FE57E068F6
:10EF90004427EE0F441FFA95E1F74195550B06D033
:10EFA0000F9007FE17CF08959FCEACC0F2DEE8F3B6
:10EFB0009923D9F3940F511DBBF39150504094F015
:10EFC00059F0882332F0660F771F881F9150504008
:10EFD000C1F79E3F510544F7880F911D969587957F
:10EFE00097F908955F3FACF0983E9CF0BB2786955B
:10EFF00077956795B79508F4B1609395C1F7BB0F06
:10F0000058F711F460FFE8CF6F5F7F4F8F4F9F4F2E
:10F01000E3CFDACE0EF076C06DCE689465CEB9DE61
:10F02000C8F39923D1F3C6F3DF93CF931F930F93C4
:10F03000FF92C92FDD2788232AF02197660F771FBB
:10F04000881FDAF720E030E040E85FEB9FE3883983
:10F0500020F0803E30F021968F77B3DCE5E7F1E0D9
:10F0600003C0AFDCE2EAF1E048DE8B01BE01EC0157
:10F07000FB2E6F5771097595771F880B990BD5DD9E
:10F0800028E132E741E35FE3B8DEAF2D9801AE013E
:10F09000FF900F911F91CF91DF91A4DC61CEFA0117
:10F0A000DC01AA0FBB1F9B01AC01BF5728F422272C
:10F0B0003327442750781FC0B75188F4AB2F002462
:10F0C000469537952795011CA395D2F3002069F04A
:10F0D000220F331F441FB395DAF30DD071CC61308A
:10F0E0007105A0E88A07B94630F49B01AC01662798
:10F0F000772788279078309621F0208331834283C8
:10F10000538308959F3F31F0915020F48795779570
:10F110006795B795880F911D9695879597F90895EE
:10F12000629FD001739FF001829FE00DF11D649FEB
:10F13000E00DF11D929FF00D839FF00D749FF00D77
:10F14000659FF00D9927729FB00DE11DF91F639F18
:10F15000B00DE11DF91FBD01CF0111240895AA1BB7
:10F16000BB1B51E107C0AA1FBB1FA617B70710F0B2
:10F17000A61BB70B881F991F5A95A9F780959095E4
:10F18000BC01CD01089597FB092E07260AD077FD13
:10F1900004D0E5DF06D000201AF4709561957F4F0A
:10F1A0000895F6F7909581959F4F0895A1E21A2E44
:10F1B000AA1BBB1BFD010DC0AA1FBB1FEE1FFF1F1B
:10F1C000A217B307E407F50720F0A21BB30BE40B6B
:10F1D000F50B661F771F881F991F1A9469F76095B2
:10F1E0007095809590959B01AC01BD01CF0108956C
:10F1F00097FB092E05260ED057FD04D0D7DF0AD085
:10F20000001C38F450954095309521953F4F4F4F55
:10F210005F4F0895F6F790958095709561957F4FB3
:10F220008F4F9F4F08952F923F924F925F926F9210
:10F230007F928F929F92AF92BF92CF92DF92EF9286
:10F24000FF920F931F93CF93DF93CDB7DEB7CA1B07
:10F25000DB0B0FB6F894DEBF0FBECDBF09942A8832
:10F26000398848885F846E847D848C849B84AA84DA
:10F27000B984C884DF80EE80FD800C811B81AA8167
:10F28000B981CE0FD11D0FB6F894DEBF0FBECDBF32
:10F29000ED010895AF92BF92CF92DF92EF92FF926D
:10F2A0000F931F93CF93DF93EC01688179818A815B
:10F2B0009B81611571058105910521F464E279ED69
:10F2C0008BE597E02DE133EF41E050E00E94F878C4
:10F2D00079018A0127EA31E440E050E00E94907809
:10F2E0005B016C01C801B7012CEE34EF4FEF5FEF0B
:10F2F0000E9490786A0D7B1D8C1D9D1D97FF04C098
:10F300006150704080409048688379838A839B83F2
:10F310007F77CB01DF91CF911F910F91FF90EF90FD
:10F32000DF90CF90BF90AF9008950E944A790895E2
:10F330008AEC96E00E944A790895A0E0B0E08093BC
:10F34000CA069093CB06A093CC06B093CD06089541
:10F350002F923F924F925F926F927F929F92AF92C5
:10F36000BF92CF92DF92EF92FF920F931F93CF93B2
:10F37000DF933B01EA016115710519F0FB01808300
:10F380009183209739F09E0122503040233231057D
:10F3900008F0D5C0C82ED92EF60111916F017F015A
:10F3A000812F90E00E94B07B0097B1F71D3231F4BD
:10F3B000F60111917F019924939406C01B3219F430
:10F3C000F60111917F019924209719F0C031D105E0
:10F3D000D1F4103389F4F7018081883711F0883532
:10F3E00059F4F701118182E090E0E80EF91E92E0F5
:10F3F000992AC0E1D0E007C0209729F41033B1F07A
:10F40000CAE0D0E02BC0CA30D10541F1C031D105EE
:10F4100021F0C830D105A9F409C02FEFA22E2FEF9B
:10F42000B22E2FEFC22E2FE0D22E20C0C8E0D0E0A7
:10F430009FEFA92E9FEFB92E9FEFC92E9FE1D92EE6
:10F4400015C09E01442737FD4095542F6FEF7FEF85
:10F45000CB010E94D67859016A0108C089E9A82E1B
:10F4600089E9B82E89E9C82E89E1D82E60E020E02C
:10F4700030E0A9011E01442437FC4094542C012F94
:10F4800000530A3060F0812F81548A3110F4075004
:10F4900006C0812F81568A3150F5012F0755802FE4
:10F4A00090E08C179D071CF56F3FE9F0A216B3069C
:10F4B000C406D506A8F0CA01B901A20191010E94B3
:10F4C00090789B01AC01802F90E0A0E0B0E0280F85
:10F4D000391F4A1F5B1F281739074A075B0710F4BB
:10F4E0006FEF01C061E0F70111917F01C8CF611496
:10F4F000710481F0662339F00894E108F108F30102
:10F50000F182E08207C091FE05C0C7010297F301B6
:10F510009183808390FE07C050954095309521954A
:10F520003F4F4F4F5F4F67FF0DC082E290E09093D7
:10F53000772D8093762D2FEF3FEFA90103C020E0B8
:10F5400030E0A901B901CA01DF91CF911F910F915C
:10F55000FF90EF90DF90CF90BF90AF909F907F9003
:10F560006F905F904F903F902F9008956627772778
:10F570000C94C67DFC0188279927E89421912032BC
:10F58000E9F3293010F02E30C8F32B3241F02D3240
:10F5900039F4689404C00E94137C820F911D21915C
:10F5A00020532A30C0F31EF4909581959F4F089503
:10F5B000283008F027E03327DA01990F311D87FD45
:10F5C000916000966105710539F432602E5F3D93BC
:10F5D00030E32A95E1F708959F3F30F080387105B8
:10F5E000610509F03C5F3C5F3D93913008F0806815
:10F5F000911DDF93CF931F930F93FF92EF92192FDB
:10F60000987F9695E92F96959695E90FFF27E851F3
:10F61000F04F99273327EE24FF24A701E701059037
:10F620000894079428F4360FE71EF81E491F511D51
:10F63000660F771F881F991F0694A1F705900794FE
:10F6400028F4E70EF81E491F561FC11D770F881FAB
:10F65000991F661F0694A1F70590079428F4F80EE9
:10F66000491F561FC71FD11D880F991F661F771F7F
:10F670000694A1F70590079420F4490F561FC71F61
:10F68000D81F990F661F771F881F0694A9F78491CA
:10F690001095177041F0D695C79557954795F794F3
:10F6A000E7941A95C1F7EEE8FFE06894159015917C
:10F6B00035916591959105907FE27395E118F10A76
:10F6C000430B560BC90BD009C0F7E10CF11E431FC9
:10F6D000561FC91FD01D7EF4703311F48A95E6CFF2
:10F6E000E894015030F0080F0AF40027021708F4DC
:10F6F000202F2395022F7A3328F079E37D932A95E2
:10F70000E9F710C07D932A9589F606949795679539
:10F71000379517951794E118F10A430B560BC90B4F
:10F72000D00998F023957E9173957A3308F070E3B1
:10F730007C932013B8F77E9170617D9330F08395B0
:10F7400071E37D9370E32A95E1F71124EF90FF9028
:10F750000F911F91CF91DF91992787FD9095089583
:10F760009111A2C3803219F089508550D0F70895C5
:10F77000FC010590615070400110D8F7809590957C
:10F780008E0F9F1F08954AE757E10E94EC7B089572
:10F79000FB01DC0102C001900D9241505040D8F7AE
:10F7A0000895DC0101C06D9341505040E0F7089589
:10F7B000FB01DC018D91019080190110D9F3990BA7
:10F7C0000895FC016150704001900110D8F78095B8
:10F7D00090958E0F9F1F0895FA01A191B081009717
:10F7E00019F41097E1F0CD01DC01CD010D9000205E
:10F7F00011F4C00113C0FB012191222319F020153F
:10F80000D9F7F3CFFB012191201519F41E9211961F
:10F8100006C02223C1F70D900020A1F7D001FA0104
:10F82000A193B08308957AE0979F902D879F802DB4
:10F83000910D112408950F931F93CF93DF938C01A3
:10F84000EB018B8181FF1BC082FF0DC02E813F81A8
:10F850008C819D812817390764F4E881F98101932F
:10F86000F983E88306C0E885F985802F099500971C
:10F8700031F48E819F8101969F838E8302C00FEFAA
:10F880001FEFC801DF91CF911F910F910895DF9372
:10F89000CF93CDB7DEB7FE0135966191719180911E
:10F8A000722D9091732DAF010E943171CF91DF9134
:10F8B0000895DF93CF93CDB7DEB7FE013596619102
:10F8C00071918091722D9091732DDC0113962C9182
:10F8D0001397286013962C93AF010E943171E09129
:10F8E000722DF091732D2381277F2383CF91DF9198
:10F8F00008956091722D7091732D0E941B7C089564
:10F90000EF92FF920F931F93CF93DF938C01E091BF
:10F91000722DF091732D838181FF1FC0C0E0D0E074
:10F920000AC0DB011896ED91FC9119970995009793
:10F9300011F0CFEFDFEFF80181918F016091722D0F
:10F940007091732D882369F7DB011896ED91FC9176
:10F9500019978AE00995009711F0CFEFDFEFCE01FC
:10F96000DF91CF911F910F91FF90EF9008950F932A
:10F970001F93DF93CF93CDB7DEB72E970FB6F894D2
:10F98000DEBF0FBECDBF0D891E898F89988D26E001
:10F990002C831A83098397FF02C080E090E80197C7
:10F9A0009E838D839E01255E3F4FCE010196698D1A
:10F9B0007A8DA9010E9431714D815E8157FD0AC087
:10F9C0002F813885421753070CF49A01020F131F39
:10F9D000F80110822E960FB6F894DEBF0FBECDBF91
:10F9E000CF91DF911F910F9108950F931F93DF9394
:10F9F000CF93CDB7DEB72E970FB6F894DEBF0FBE0C
:10FA0000CDBF8C01CB01BA0146E04C831A83098338
:10FA100097FF02C080E090E801979E838D83CE011E
:10FA20000196A9010E9431714D815E8157FD0AC086
:10FA30002F813885421753070CF49A01020F131FC8
:10FA4000F80110822E960FB6F894DEBF0FBECDBF20
:10FA5000CF91DF911F910F910895FA01AA272830C5
:10FA600051F1203181F1E8946F936E7F6E5F7F4F8B
:10FA70008F4F9F4FAF4FB1E03ED0B4E03CD0670F07
:10FA8000781F891F9A1FA11D680F791F8A1F911D5A
:10FA9000A11D6A0F711D811D911DA11D20D009F4AA
:10FAA00068943F912AE0269F11243019305D3193EC
:10FAB000DEF6CF010895462F4770405D4193B3E0D5
:10FAC0000FD0C9F7F6CF462F4F70405D4A3318F07C
:10FAD000495D31FD4052419302D0A9F7EACFB4E02D
:10FAE000A6959795879577956795BA95C9F70097E5
:10FAF0006105710508959B01AC010A2E0694579586
:10FB0000479537952795BA95C9F7620F731F841FDC
:10FB1000951FA01D0895DC01CB01FC01F999FECFD2
:10FB200006C0F2BDE1BDF89A319600B40D92415085
:10FB30005040B8F70895F999FECF92BD81BDF89A6B
:10FB4000992780B50895A8E1B0E042E050E00C9418
:10FB50008D7DDC01CB0103C02D910E94B47D41500D
:10FB60005040D0F70895262FF999FECF1FBA92BDC5
:10FB700081BD20BD0FB6F894FA9AF99A0FBE01968E
:10FB800008950E94B37D272F0C94B47D6F927F92CD
:10FB90008F929F92AF92BF92CF92DF92EF92FF929D
:10FBA0000F931F93DF93CF930F92CDB7DEB75B0117
:10FBB0006115710521F0DB018C9311969C93482F00
:10FBC000592F6A01F601E1906F018F018E2D90E0AF
:10FBD0000E94B07B0097B1F7FE2DFD3229F4D601CB
:10FBE000ED908D0121E007C0BE2DBB3219F4F60166
:10FBF000E1908F0120E068010894C108D108C60196
:10FC000068E870E143E050E029830E94577F298132
:10FC1000009711F572E0E72EF12CE00EF11EC701FE
:10FC20006BE870E145E050E00E94577F2981009722
:10FC300029F467E0E62EF12CE00EF11EA114B104C8
:10FC400021F0D5011196FC92EE9220FF0FC130E019
:10FC500020E090E88FEF12C1C60160E970E143E057
:10FC600050E029830E94577F2981009731F060E09E
:10FC700070E0CB01662477240AC0A114B10409F412
:10FC8000F9C00E5F1F4FF50111830083F3C03E2DB5
:10FC900030533A30A0F52260E22FF0E0AF01487017
:10FCA000507022FF07C04115510571F50894611C81
:10FCB000711C2AC04115510519F00894610871089A
:10FCC0006B017C0152E0CC0CDD1CEE1CFF1C5A9534
:10FCD000D1F76C0D7D1D8E1D9F1D660F771F881F30
:10FCE000991F630F711D811D911D6839F9E97F0707
:10FCF000F9E98F07F9E19F0738F0246005C03E3F1E
:10FD000039F423FD3FC02860D801ED908D01BFCFAD
:10FD1000353311F03531B1F5F80131913D3211F43F
:10FD2000206102C03B3241F4D80111963C911197F9
:10FD3000319642E050E002C041E050E030533A30AA
:10FD400020F08F01041B150B1DC040E050E0BCE00B
:10FD500040385B075CF4DA01AA0FBB1FAA0FBB1F78
:10FD60004A0F5B1F440F551F430F511D31913053F4
:10FD70008F013A3060F324FF03C0509541955F4FE7
:10FD8000640E751EC22EDD2421FF08C0A114B1042B
:10FD900029F001501040F501118300830E94137671
:10FDA0007B018C01F3E0CF22DD2433E0C316D104C4
:10FDB00021F417FB109517F91095C801B70120E041
:10FDC00030E0A9010E94A775882309F44AC077FE94
:10FDD00009C047EAC42E40E1D42E709461947108A2
:10FDE000739404C03FEBC32E30E1D32E26E0822E65
:10FDF000912C90E2A92EB12C0FC0F60125913591DE
:10FE000045915491C801B7010E94F176E62EF72E74
:10FE1000082F192F6A187B086A147B0474F7B594AD
:10FE2000A7940894810891088114910429F08CEF1B
:10FE30009FEFC80ED91EF0CFB701C801282F220F9F
:10FE4000292F221F2F3F39F020E030E0A9010E9426
:10FE5000A775882331F482E290E09093772D809308
:10FE6000762D3E2D2F2D902F812F08C030E020E0E1
:10FE700090E803C030E020E090EC8FE7F901AC019E
:10FE80006F2F722F852F942F0F90CF91DF911F919D
:10FE90000F91FF90EF90DF90CF90BF90AF909F9029
:10FEA0008F907F906F900895992788270895FB0180
:10FEB000DC014150504088F08D9181341CF08B352D
:10FEC0000CF4805E659161341CF06B350CF4605E5F
:10FED000861B611171F3990B0895881BFCCFF89470
:02FEE000FFCF52
:10FEE200263A202573205B414444523D252D642E41
:10FEF200252D64205345513D252D642052535349ED
:10FF02003D252D75204C51493D252D7520445250DB
:10FF12003D252D642E253032645D0A00523D252D8B
:10FF220075204C3D252D7520533D252D6420005410
:10FF3200696D656F757420414444523D252D642ED0
:10FF4200252D64205345513D252D6420525353499C
:10FF52003D252D75204C51493D252D750A0028451A
:10FF6200787450777229000065756936343D002532
:10FF720030327800253032780A00736E3D00413A03
:10FF8200202564202564202564200A00433A202588
:10FF92006420256420256420613D25352E31660AC2
:10FFA200007374617475733D3078253032780A209D
:10FFB20000312E30204669726D7761726520566578
:10FFC200722E2053322D332E3920323031332D30E0
:10FFD200352D313200656570726F6D006F6E006F86
:10FFE200666600666F7263655F69646C650064656E
:0EFFF2006570004F6E006131007265736574BA
:020000021000EC
:10000000006E6F6E6500613200765F696E003100D0
:1000100032003300340035006175746F00666C7512
:10002000736800414444523D252D642E252D6420E3
:100030005345513D252D6420525353493D252D757F
:10004000204C51493D252D750A00707772733D256E
:10005000730A007472696D00746573740043683DBF
:10006000252D642054785077723D252D640A004573
:1000700072726F72205458204C656E6774683D250B
:10008000640A0049443D004536343D002050533D4C
:1000900025640020543D252D362E32660020543133
:1000A0003D252D362E32660020545F4D43553D25AB
:1000B0002D352E31660020565F4D43553D252D349C
:1000C0002E3266002050303D252D6C5800205030D7
:1000D0005F543D252D372E3366002050313D252DB0
:1000E0006C58002050315F543D252D372E3366006B
:1000F0002055503D252D6C58002052483D252D346B
:100100002E31660020565F494E3D252D352E326634
:100110000020565F41313D252D352E326600205698
:100120005F41323D252D352E32660020565F41332A
:100130003D252D352E30660020503D252D6C640068
:100140002050413D252D372E326600263A2025735A
:100150000A00545820706B74206C656E203D202579
:10016000640A0025303258006C656E3D25640A0033
:100170000100D734EF3C22FFCC3B22FFCC3B1A20BE
:10018000090D009D046162636465666768696A6B56
:100190006C6D6E6F70269400003C000A00636D6405
:1001A0002070726F63657373000000BB04EF33004F
:1001B000000000737464696E2070726F63657373FE
:1001C000000000D104040F0000000062726F61643F
:1001D000636173742070726F63657373000000E96C
:1001E00004C23400000000536C6565702070726FAB
:1001F000636573730000000505F40F0000000050F4
:100200006572696F6469632070726F6365737300F0
:1002100000001D05F01600000000C704DF04FB0409
:100220002E0513050000A50800001D00400004076E
:10023000440710000000143D083D181000000000A5
:100240004576656E742074696D65720000005E0508
:100250001F41000000004374696D65722070726F69
:100260006365737300000074055D420000000002C6
:100270000306070A0B0E0F020306070A0B0E0F28D0
:1002800043292032303132204865726A756C66002D
:1002900055747665636B6C696E6720202020202082
:1002A00000436F6E74696B6920322E3500000000C8
:1002B0000200000000985000000000C600C500C405
:1002C00000C100C200000000CE00CD00CC00C9007B
:1002D000CA000000005246323330206472697665ED
:1002E00072000000F3054F5500000000C0533E535C
:1002F0009E55E8566154F1525F515951E0524252B5
:1003000000010101010101010101010101010101DE
:100310000052696D65002F0663582A586164617444
:10032000612E6E756D20776179206F757420746809
:100330006572653A2025640A00A559A459AE5BDDB3
:100340005C155B0080C0E0F0F8FCFEFF6E756C6C25
:100350006D6163006A06905D755D7B5D815D875DA3
:100360008D5D736963736C6F776D6163008006B137
:100370005E125EA85D915D975DA55DBA0008000301
:10038000110B1135000200DB16DD165443502F49C6
:100390005020737461636B000000A9060B610000BC
:1003A00000000208FFFFFFFF000000000100000046
:00000001FF
